:100000000C9421330C94C6330C94C6330C94C63331
:100010000C94C6330C94C6330C94C6330C94C6337C
:100020000C94C6330C94C6330C94C6330C94C6336C
:100030000C94C6330C940B360C94C6330C94C63314
:100040000C94C6330C94C6330C94C6330C94C6334C
:100050000C94C6330C94C6330C94C6330C94C6333C
:100060000C94C6330C94C6330C94C6330C94C6332C
:100070005A5501200201003808000000000000006D
:100080000000000000A440B24082415D454745B5F4
:1000900040C440D3402D45E140EF401E1C0000000D
:1000A0000000000000000000000000000000000050
:1000B0000000000000000000000000000000000040
:1000C0000000000000000000000000000000000030
:1000D0000000000000000000000000000000000020
:1000E0000000000000000102030405060708090AD9
:1000F0000B0C0000000000000000000000000000E9
:10010000000000000D0E0F10111213141516171811
:1001100000000000000000000000000000000000DF
:1001200000000000000000000000000000000000CF
:1001300000000000191A1A1A1A1A1A1A1B1C1D1D7F
:100140001D1D1D1D1D1D1D1D1D1D1D1D1D1D1E00FB
:1001500000001F20212223242520262728292A2B9E
:100160002C2D2E2F30313233343536363700000007
:100170001F383838383838382627393A3B3C3D3E26
:100180003F404142434445463636370000001F4752
:1001900048492223242526274A4B4C4D4E4F505187
:1001A0005253545556573636370000001F383838EA
:1001B00038383838262758595A5B5C5D5E5F606175
:1001C000626364653636370000001F2066256725A8
:1001D00068202627696A6B6C6D6E6F707172383695
:1001E00036363636370000001F3838383838383859
:1001F0002627737475767778797A7B7C7D363636E8
:100200003636370000001F2047487E7F49202627CA
:100210008081818181818181818236363636363690
:10022000370000001F38383838383838262783849C
:1002300085868788898A848B363636363636370007
:1002400000008C8D8D8D8D8D8D8D8E278384848F78
:100250008F8F8F84848B36363636363637000000E3
:10026000000000000000000000278390918988872B
:100270009289848B363636363636370000000000D9
:1002800000000000000000278384849387949584F5
:10029000848B3636363636363700000000000000D4
:1002A0000000000000278384968788949784848BBD
:1002B00036363636363637000000191A1A1A1A1A28
:1002C0001A1A1B27838484989984989A9A8B3636B5
:1002D00036363636370000001F9B9B9B9B9B9B9BB3
:1002E00026279C9D9D9D9D9D9D9D9D9E36363636C7
:1002F0003636370000001F9B9B9B9B9B9B9B2627B2
:10030000363636363636363636363636363636368D
:10031000370000001F9B9B9B9B9B9B9B26279FA0BE
:10032000A1A2A3A4A5A6A7363636363636363700A0
:1003300000008C8D8D8D8D8D8D8D8EA8A9A9A9A97C
:10034000A9A9A9A9A9A9A9A9A9A9A9A9AA00000017
:10035000000000000000000000AB9F9F9F9F9F9F38
:100360009F9F9F9F9F9F9F9F9F9FAC000080818129
:10037000818181818181828081818181818181816D
:10038000818182000000000000000083AD89AE89F9
:10039000AF84B0B18B83B28692898498AE89B3B4AE
:1003A0008B000000000000000083B59189888792CF
:1003B00089B68B83B4B7B88492B8AE8988B48B0001
:1003C000000000000000009C9D9D9D9D9D9D9D9DA9
:1003D0009E9C9D9D9D9D9D9D9D9D9D9D9E00000023
:1003E00000000000000B01696A6B6C6D6E6F70712C
:1003F00072380B01737475767778797A7B7C7D011E
:10040000019B09019FA0A1A2A3A4A5A6A70A0880F9
:1004100081818181818181818283848586878889A8
:100420008A848B8384848F8F8F8F84848B83909135
:100430008988879289848B83848493879495848424
:100440008B8384968788949784848B8384849899FB
:1004500084989A9A8B9C9D9D9D9D9D9D9D9D9E019E
:1004600001840101900A04808181818181818181DF
:100470008283AD89AE89AF84B0B18B83B591898811
:10048000879289B68B9C9D9D9D9D9D9D9D9D9E0C5B
:100490000480818181818181818181818283B28691
:1004A00092898498AE89B3B48B83B4B7B88492B878
:1004B000AE8988B48B9C9D9D9D9D9D9D9D9D9D9D80
:1004C0009E02022829393A02022A2B3B3C02022CC6
:1004D0002D3D3E02022E2F3F4002023031414202AA
:1004E0000232334344020234354546020236363680
:1004F0003602024A4B585902024C4D5A5B02024ED8
:100500004F5C5D020250515E5F0202525360610215
:1005100002545562630202565764654040404040B1
:1005200040404040404040404040404040404040CB
:1005300040404040404040404040404040404040BB
:1005400040404040404040404040404040404040AB
:10055000404040404040404040404040404040409B
:1005600040404040404040404F4F4F404040404F4F
:100570004F4F4F4040404F4F40404040404F404021
:10058000404040404040404040404040404040406B
:1005900040404F404040404040404F4F4F4F4F4FF2
:1005A0004040404F4F4F4F4F4F4F404F4F4F4F4F97
:1005B0004F4F4F404F4F404F4F4F4F404F404040A5
:1005C0004F4F4F4F4040404F4F4F404040404F4FA4
:1005D0004F4040404F4F4F4F4040404040404040D0
:1005E000404040404040404040404040404040400B
:1005F000404040404040404040404040404F4F40DD
:100600004F4F4F404F4F4F404F4F4F404F4F4F4036
:100610004F4F4F404F4F4F404F4F4F40404F4F4035
:10062000404040404F4F4F40404040404F4F4F4070
:10063000404040404F4F4F40404040404F4F4F4060
:100640004F4F4F404F4F4F4F4F4F4F404F4F4F4FD8
:100650004F4F4F404F4F4F40404F4F404040404022
:10066000404040404040404040404040404040408A
:100670004040404040404040404040404F4F4F404D
:100680004F4F4F4F4F4F4F404F4F4F4F4F4F4F4098
:100690004F4F4F4F4F4F4F4F4F4F4F4040404040B5
:1006A000404040404040404040404040404040404A
:1006B000404040404040404040404040404040403A
:1006C000404040404040404040404040404040402A
:1006D000404040404040404040404F40404040400B
:1006E00040404F404040404F4F4F4F4040404F4FA1
:1006F0004F4F4F40404F4F40404040404F404040A0
:100700004040404F4F4040404040404F40404040BC
:100710004040404F404040404040404F4F4F4F408E
:100720004040404F4F4F4F404040404F4F4F4F4051
:10073000404040404F4F4F4040404040404F40407D
:10074000404F4F40404F4040404F4F40404040405E
:10075000404F4F4040404040404F4F40404040405D
:100760004040404040404040404040404040404089
:1007700040404040404040404040404F404F4F404C
:10078000404F4F4F4F4F4F404F4F4F4F404F4040C4
:100790004F4F4F4F404040404F4F4F4040404040F0
:1007A0004040404040404040404040404040404049
:1007B0004040404040404040404040404F4F4F400C
:1007C00040404F404F4F4F40404F4F404F4F4F40A2
:1007D0004F4F4F404F4F4F404F4F4F404040404092
:1007E00040404F4040404040404F4F4040404040DC
:1007F000404F4F4040404040404F4F4F4F4F4F4081
:10080000404F4F4F4F4F4F40404F4F404040404070
:10081000404F4F4F4F4F4F4F404F4F4F4040404042
:100820004040404F404040404040404F40404040AA
:100830004040404F404040404040404F404F4F407C
:100840004040404F4F4F4F4F4F40404F40404F4F21
:100850004F40404F40404F4F4F404040404040404D
:10086000404F4F40404040404F4F4F40404040403D
:100870004F4F4F404F40404F404F4F4F4F4F4F40D3
:1008800040404F404F4F404040404040404040403B
:1008900040404040404040404040404F4F4040403A
:1008A0004040404F404040404040404F4F4040401B
:1008B0004040404F4F4F40404040404F4F4F4F40CF
:1008C000404040404F4F404040404040404F4040FB
:1008D0004040404040404040404040404F4F4F40EB
:1008E0004F4F4F404F4F4F404F4F4F40404F4F4F54
:1008F0004F4F4F40404040404040404040404040CB
:1009000040404040404040404040404040404040E7
:100910004040404040404040404040404F4F4F40AA
:10092000404F4F404F4F4F4F4F4F4F404F4F4F4013
:100930004F4F40404F40404040404040404040408A
:1009400040404040404040404040404040404040A7
:1009500040404040404040404040404F4F4F4F4F4C
:100960004F4F4F404F4F4F404F4F4F404F4F4040E2
:100970004F4F4F404F4040404F4F4F404F4F4040F0
:100980004F4F404F4F4F4F4F4F40404040404F4FD1
:100990004F40404040404040404040404040404048
:1009A00040404F404040404040404F404040404029
:1009B00040404F404040404040404F404040404019
:1009C0004040404040404040404040404040404027
:1009D00040404040404040404040404F4040404008
:1009E0004040404F4F4040404040404F4F4F4040BC
:1009F0004040404F4F4F4F4F4F4F404F4F4F4F4F43
:100A00004F4F4F404F4F4F4F4F4F4F4040404F4F32
:100A10004F4F4F40404040404040404040404040A9
:100A2000404F4F4040404040404F4F40404040408A
:100A300040404F40404040404040404F4F4F4F4F5C
:100A40004F40404F4F4F4F4F4040404F4F4F40401F
:100A500040404040404040404040404F4040404087
:100A60004F4F4F4F4F4040404F4F4F4F4F404040F0
:100A7000404F4F4040404040404040404040404058
:100A80004040404040404040404040404040404066
:100A90004040404040404040404040404F4F4F4029
:100AA000404F4F404F4F4F404F40404F4F4F4F40B0
:100AB000404F4F4040404040404040404040404018
:100AC0004040404040404040404040404040404026
:100AD00040404040404040404040404F4F4F4F4FCB
:100AE000404F4F40404F4F4F404F4F4F4F4F404070
:100AF000404F4F40404040404040404040404040D8
:100B000040404040404040404040404040404040E5
:100B100040404040404040404040404F40404F4FA8
:100B20004F40404F40404F4F4F40404F40404F4F4D
:100B30004F40404040404F4F40404040404F404079
:100B400040404040404040404040404040404040A5
:100B50004040404040404040404040404040404095
:100B60004040404040404040404040404040404085
:100B70004040404040404040404040404040404075
:100B800040E1E14040404040E1E1E140404040E19F
:100B9000E1E1E140404040E1E1E1E14040404040EE
:100BA0004040404040404040404040404040404045
:100BB0004040404040404040404040E1E1E1E1E110
:100BC000E1E1E1E1E1E1E1E1E1E1E1E1E1E1E1E115
:100BD000E1E1E1E1E1E1E1E1E1E1E140404040402A
:100BE0004040404040404040404040404040404005
:100BF0004040404040404040404040E1E1404040B3
:100C0000404040E1E1E14040404040E1E1E1E1407D
:100C1000404040E1E1E1E140404040404040404050
:100C200040404040404040404040404040404040C4
:100C300040404040404040404040404040404040B4
:100C400040373740404040403737374040404037DA
:100C500037373740404040373737374040404040D3
:100C60004040404040404040404040404040404084
:100C700040404040404040404040403737373737A1
:100C800037373737373737373737373737373737F4
:100C900037373737373737373737374040404040B7
:100CA0004040404040404040404040404040404044
:100CB0004040404040404040404040373740404046
:100CC0004040403737374040404040373737374063
:100CD000404040373737374040404040404040E197
:100CE000E1E1E140404040E1E1E1E140404040E1FC
:100CF000E1E1E140404040E1E1E1E140404040E1EC
:100D0000E1E1E140404040E1E1E1E140404040E1DB
:100D1000E1E1E140404040E1E1E1E19191919191D7
:100D200091919191919191919191919191919191B3
:100D300091919191919191919191919191919191A3
:100D40009191919191919191919191919191919193
:100D50009191919191919191919191919191919183
:100D60009191919191FFFFFFFF919191FFFF9191DF
:100D70009191919191FFFFFFFF91919191919191AB
:100D8000FFFF919191919191FFFF919191FFFFFF51
:100D9000FF919191919191919191919191919191D5
:100DA00091919191919191919191919191FFFFFFE9
:100DB000FF919191FFFF919191919191FFFF9191FD
:100DC00091919191FFFF91919191919191FFFFFFED
:100DD000FF91919191919191919191919191919195
:100DE00091919191919191919191919191FFFFFFA9
:100DF000FF919191FFFF9191FFFF9191FFFF9191E1
:100E0000FFFF9191FFFF9191FFFF919191FFFFFFF4
:100E1000FF91919191919191919191919191919154
:100E2000919191919191919191919191FFFFFFFFFA
:100E3000FF919191FFFF9191FFFF9191FFFF9191A0
:100E400091919191FFFF919191919191FFFF9191DA
:100E50009191919191919191919191919191919182
:100E600091919191919191919191919191FFFFFF28
:100E7000FF919191FFFF9191FFFF9191FFFFFFFF84
:100E8000FFFF9191FFFF91919191919191FFFFFF50
:100E9000FF91919191919191919191E1E1E1E140E5
:100EA000404040E1E1E1E140404040E1E1E1E1403A
:100EB000404040E1E1E1E140404040E1E1E1E1402A
:100EC000404040E1E1E1E140404040E1E1E1E1401A
:100ED000404040E1E1E1E140404040404040403797
:100EE000373737404040403737373740404040374A
:100EF000373737404040403737373740404040373A
:100F00003737374040404037373737404040403729
:100F100037373740404040373737370A0A0A0A0A1E
:100F20000A0A0A0A0A0A0A0A0A0A0A0A0A0A0A0A21
:100F30000A00000A0A0A0A0000FFFE0A0A0A00FF65
:100F4000FFFFFE0A0A0A00FFFFFFFE0A0A00FFFF7A
:100F5000FFFEFE0A0A00FEFEFEFEFE0A0A0A0A0A5A
:100F60000A0A0A0A0A0A0A0A0A0A0A00000A0A0AF5
:100F70000A0A0AFEFE00000A0A0A0AFEFEFEFE0037
:100F80000A0A0AFEFEFEFE000A0A0AFEFEFEFEFC39
:100F9000000A0AFEFEFEFCFC000A0A0A0A0A0A0A05
:100FA0000A0A0A0A0A0A0A0A0A0A0A0A0A0A0A0AA1
:100FB0000A0A000A0A0A0A0A0A00850A0A0A0A0A2A
:100FC0000A00850A0A0A0A0A0085850A0A0A0A0A24
:100FD0000085430A0A0A0A008585430A0A0A0A0AA2
:100FE0000A0A0A0A0A0A0A0A0A0A0A000A0A0A0A6B
:100FF0000A0A0A85000A0A0A0A0A0A85000A0A0A6F
:101000000A0A0A8585000A0A0A0A0A4385000A0AAA
:101010000A0A0A438585000A0A0A0A0A0A0A0A0A0B
:101020000A0A0A0A0A0A0A0A0A0A0A0A0A0A0A0A20
:101030000000000A0A0A0A00112A2A0A0A0A002ADB
:101040002A112A0A0A00112A2A112A0A0A002A1138
:101050001111110A0A002A2A2A112A0A0A0A0A0A5E
:101060000A0A0A0A0A0A0A0A0A0A0A0000000A0AFE
:101070000A0A0A2A2A11000A0A0A0A2A112A2A0036
:101080000A0A0A2A112A2A11000A0A111111112A20
:10109000000A0A2A112A2A2A000A0A0A0A0A0A0A3D
:1010A0000A0A0A0A0A0A0A0A0A0A0A0A0A0A0A0AA0
:1010B0000A0A000A0A0A0A0A0A00270A0A0A0A0091
:1010C0000027270A0A0A00272715270A0A0A0027E5
:1010D0002727150A0A0A00272715270A0A0A0A0AD3
:1010E0000A0A0A0A0A0A0A0A0A0A0A000A0A0A0A6A
:1010F0000A0A0A27000A0A0A0A0A0A272700000A17
:101100000A0A0A27152727000A0A0A15272727008F
:101110000A0A0A27152727000A0A0A0A0A0A0A0AD7
:101120000A0A0A0A0A0A0A0A0A0A0A0A0A0A0A0A1F
:101130000A0A000A0A0A0A0A0A00250A0A0A0A0A08
:101140000037250A0A0A0A003737250A0A0A003733
:101150003737250A0A0025252525250A0A0A0A0AFD
:101160000A0A0A0A0A0A0A0A0A0A0A000A0A0A0AE9
:101170000A0A0A37000A0A0A0A0A0A3737000A0A5C
:101180000A0A0A373737000A0A0A0A373737370098
:101190000A0A0A2537373737000A0A0A0A0A0A0AEA
:1011A0000A0A0A0A0A0A0A0A0A0A0A0A0A0A0A00A9
:1011B0000000000A0A0A00D0D040D00A0A00D0D0AD
:1011C00040D0D00A0A0040404040400A0A0A00D0FD
:1011D00040D0D00A0A0A00D0D040D00A0A0A0A0A2F
:1011E0000A0A0A0A0A0A0A0A0A0A0A000000000A87
:1011F0000A0A0AD040D0D0000A0A0AD0D040D0D083
:10120000000A0A4040404040000A0AD0D040D000C6
:101210000A0A0AD040D0D0000A0A0A0A0A0A0A0AB0
:101220000A0A0A0A0A0A0A0A0A0A0A0A0A0A000032
:101230000000000A0A0000070707070A0A00070063
:101240000707070A0A0007070000000A0A00070745
:101250000007070A0A0007070007070A0A0A0A0A1E
:101260000A0A0A0A0A0A0A0A0A0A0A000000000010
:101270000A0A0A0707070700000A0A070707000704
:10128000000A0A0000000707000A0A07070007070C
:10129000000A0A0707000707000A0A0A0A0A0A0AD8
:1012A0000A0A0A0A0A0A0A0A0A0A0A0A0A0A0A0A9E
:1012B0000A0A0A0A0A0A0A0A0A0A0A0A0A0A0A0A8E
:1012C0000A0A0A0A0A0A0A0A0A0A0A0A0A0A0A0A7E
:1012D0000A0A0A0A0A0A0A0A0A0A0A373737374084
:1012E0004040403737373740404040373737374046
:1012F0004040403737373740404040373737374036
:101300004040403737373740404040373737374025
:10131000404040373737374040404091919191915C
:101320009191919191484848489191914848919163
:101330004848919148489148484891914848489177
:10134000484891914848919148489191914848481E
:1013500048919191919191919191910A0A00FEFE8B
:10136000FEFEFE0A0A00FEFEFEFEFE0A0A0A00FE5D
:10137000FEFEFE0A0A0A00FEFEFEFC0A0A0A0A0037
:1013800000FCFC0A0A0A0A0A0A00000A0A0A0A0AF7
:101390000A0A0A0A0A0A0A0A0A0A0AFEFEFEFCFCED
:1013A000000A0AFEFEFCFCFC000A0AFEFCFCFC0033
:1013B0000A0A0AFCFCFCFC000A0A0AFCFC00000AFF
:1013C0000A0A0A00000A0A0A0A0A0A0A0A0A0A0A91
:1013D0000A0A0A0A0A0A0A0A0A0A0A0A0A0A0A0077
:1013E0008543850A0A0A00858543850A0A0A00851D
:1013F0004385850A0A0085854343430A0A0085859B
:101400008585850A0A0000000000000A0A0A0A0A07
:101410000A0A0A0A0A0A0A0A0A0A0A854385000A07
:101420000A0A0A85438585000A0A0A8585438500DC
:101430000A0A0A4343438585000A0A85858585850E
:10144000000A0A0000000000000A0A0A0A0A0A0A42
:101450000A0A0A0A0A0A0A0A0A0A0A0A0A002A2AB6
:101460002A112A0A0A002A111111110A0A00112A46
:101470002A112A0A0A0A002A2A112A0A0A0A0A0032
:10148000112A2A0A0A0A0A0A0000000A0A0A0A0A93
:101490000A0A0A0A0A0A0A0A0A0A0A2A112A2A2A25
:1014A000000A0A111111112A000A0A2A112A2A1106
:1014B000000A0A2A112A2A000A0A0A2A2A11000AFC
:1014C0000A0A0A0000000A0A0A0A0A0A0A0A0A0A9A
:1014D0000A0A0A0A0A0A0A0A0A0A0A0A0A0A002759
:1014E0002715270A0A0A00272727150A0A0A0027AC
:1014F0002715270A0A0A0A000027270A0A0A0A0AE1
:101500000A00270A0A0A0A0A0A0A000A0A0A0A0A32
:101510000A0A0A0A0A0A0A0A0A0A0A2715272700D3
:101520000A0A0A15272727000A0A0A27152727006B
:101530000A0A0A272700000A0A0A0A27000A0A0AD2
:101540000A0A0A000A0A0A0A0A0A0A0A0A0A0A0A05
:101550000A0A0A0A0A0A0A0A0A0A0A0A0A0037379B
:101560003737250A0A0A00373737370A0A0A0A00C6
:101570003737370A0A0A0A0A0037370A0A0A0A0AF4
:101580000A00370A0A0A0A0A0A0A000A0A0A0A0AA2
:101590000A0A0A0A0A0A0A0A0A0A0A252525252524
:1015A000000A0A25373737000A0A0A253737000AA2
:1015B0000A0A0A2537000A0A0A0A0A25000A0A0A3C
:1015C0000A0A0A000A0A0A0A0A0A0A0A0A0A0A0A85
:1015D0000A0A0A0A0A0A0A0A0A0A0A0A0A0A0A0075
:1015E000D040D00A0A0A0A00D0D0400A0A0A0A0AE1
:1015F00000D0400A0A0A0A0A00D0400A0A0A0A0A67
:101600000A00400A0A0A0A0A0A0A000A0A0A0A0A18
:101610000A0A0A0A0A0A0A0A0A0A0AD040D0000A72
:101620000A0A0A40D0D0000A0A0A0A40D0000A0A70
:101630000A0A0A40D0000A0A0A0A0A40000A0A0AEC
:101640000A0A0A000A0A0A0A0A0A0A0A0A0A0A0A04
:101650000A0A0A0A0A0A0A0A0A0A0A0A0A000707FA
:101660000007070A0A0007070007070A0A0007071A
:101670000000000A0A0007000707070A0A0000071F
:101680000707070A0A0A00000000000A0A0A0A0AF5
:101690000A0A0A0A0A0A0A0A0A0A0A0707000707C0
:1016A000000A0A0707000707000A0A0000000707E8
:1016B000000A0A0707070007000A0A0707070700CA
:1016C000000A0A00000000000A0A0A0A0A0A0A0AB6
:1016D0000A0A0A0A0A0A0A0A0A0A0A9191919191C7
:1016E00091919191FFFF9191FFFF9191FFFF919156
:1016F000FFFF9191FFFFFFFFFFFF9191FFFF91918E
:10170000FFFF9191FFFF9191FFFF9191FFFF919159
:10171000FFFF9191919191919191919191919191DD
:10172000919191919191FFFF9191919191919191CD
:101730009191919191FFFFFF919191919191FFFF73
:10174000919191919191FFFF9191919191FFFFFF63
:10175000FF9191919191919191919191919191910B
:1017600091919191919191919191919191FFFFFF1F
:10177000FFFF9191FFFF91919191919191FFFFFF57
:10178000FF91919191919191FFFF9191FFFFFFFF47
:10179000FF919191919191919191910A0A0A0A0A6E
:1017A0000A0A0A0A0A0A0A0A0A0A0A0A0A0A0A0A99
:1017B0000AFEFE0A0A0A0AFEFEFEFE0A0A0AFEFEE9
:1017C000FEFEFE0A0A0AFEFEFEFEFE0A0AFEFEFEFD
:1017D000FEFEFE0A0AFEFEFEFEFEFE0A0A0A0A0AD5
:1017E0000A0A0A0A0A0A0A0A0A0A0AFEFE0A0A0A71
:1017F0000A0A0AFEFEFEFE0A0A0A0AFEFEFEFEFEB5
:101800000A0A0AFEFEFEFEFE0A0A0AFEFEFEFEFEB0
:10181000FE0A0AFEFEFEFEFEFE0A0A0A0A0A0A0A7C
:101820000A0A0A0A0A0A0A0A0A0A0A0A0A0A0A0A18
:101830000A0AFE0A0A0A0A0A0AFEFE0A0A0A0A0A2C
:101840000AFEFE0A0A0A0A0AFEFEFE0A0A0A0A0A34
:10185000FEFEFE0A0A0A0AFEFEFEFE0A0A0A0A0A3C
:101860000A0A0A0A0A0A0A0A0A0A0AFE0A0A0A0AE4
:101870000A0A0AFEFE0A0A0A0A0A0AFEFE0A0A0AF8
:101880000A0A0AFEFEFE0A0A0A0A0AFEFEFE0A0A00
:101890000A0A0AFEFEFEFE0A0A0A0A0A0A0A0A0AD8
:1018A0000A0A0A0A0A0A0A0A0A0A0A0A0A0A0A0A98
:1018B000FEFEFE0A0A0A0AFEFEFEFE0A0A0AFEFEF4
:1018C000FEFEFE0A0AFEFEFEFEFEFE0A0AFEFEFE08
:1018D000FEFEFE0A0AFEFEFEFEFEFE0A0A0A0A0AD4
:1018E0000A0A0A0A0A0A0A0A0A0A0AFEFEFE0A0A7C
:1018F0000A0A0AFEFEFEFE0A0A0A0AFEFEFEFEFEB4
:101900000A0A0AFEFEFEFEFEFE0A0AFEFEFEFEFEBB
:10191000FE0A0AFEFEFEFEFEFE0A0A0A0A0A0A0A7B
:101920000A0A0A0A0A0A0A0A0A0A0A0A0A0A0A0A17
:101930000A0AFE0A0A0A0A0A0AFEFE0A0A0A0AFE37
:10194000FEFEFE0A0A0AFEFEFEFEFE0A0A0AFEFE6F
:10195000FEFEFE0A0A0AFEFEFEFEFE0A0A0A0A0A47
:101960000A0A0A0A0A0A0A0A0A0A0AFE0A0A0A0AE3
:101970000A0A0AFEFE0A0A0A0A0A0AFEFEFEFE0A0F
:101980000A0A0AFEFEFEFEFE0A0A0AFEFEFEFEFE2F
:101990000A0A0AFEFEFEFEFE0A0A0A0A0A0A0A0AE3
:1019A0000A0A0A0A0A0A0A0A0A0A0A0A0A0A0A0A97
:1019B0000A0AFE0A0A0A0A0A0AFEFE0A0A0A0A0AAB
:1019C000FEFEFE0A0A0A0AFEFEFEFE0A0A0AFEFEE3
:1019D000FEFEFE0A0AFEFEFEFEFEFE0A0A0A0A0AD3
:1019E0000A0A0A0A0A0A0A0A0A0A0AFE0A0A0A0A63
:1019F0000A0A0AFEFE0A0A0A0A0A0AFEFEFE0A0A83
:101A00000A0A0AFEFEFEFE0A0A0A0AFEFEFEFEFEA2
:101A10000A0A0AFEFEFEFEFEFE0A0A0A0A0A0A0A6E
:101A20000A0A0A0A0A0A0A0A0A0A0A0A0A0A0AFE22
:101A3000FEFEFE0A0A0AFEFEFEFEFE0A0AFEFEFE8A
:101A4000FEFEFE0A0AFEFEFEFEFEFE0A0A0AFEFE7A
:101A5000FEFEFE0A0A0AFEFEFEFEFE0A0A0A0A0A46
:101A60000A0A0A0A0A0A0A0A0A0A0AFEFEFEFE0A06
:101A70000A0A0AFEFEFEFEFE0A0A0AFEFEFEFEFE3E
:101A8000FE0A0AFEFEFEFEFEFE0A0AFEFEFEFEFE46
:101A90000A0A0AFEFEFEFEFE0A0A0A0A0A0A0A0AE2
:101AA0000A0A0A0A0A0A0A0A0A0A0A0A0A0AFEFEAE
:101AB000FEFEFE0A0AFEFEFEFEFEFE0A0AFEFEFE16
:101AC000FEFEFE0A0AFEFEFEFEFEFE0A0AFEFEFE06
:101AD000FEFEFE0A0AFEFEFEFEFEFE0A0A0A0A0AD2
:101AE0000A0A0A0A0A0A0A0A0A0A0AFEFEFEFEFE92
:101AF0000A0A0AFEFEFEFEFEFE0A0AFEFEFEFEFECA
:101B0000FE0A0AFEFEFEFEFEFE0A0AFEFEFEFEFEC5
:101B1000FE0A0AFEFEFEFEFEFE0A0A0A0AFEFEFE9D
:101B2000FEFEFE0A0AFEFEFEFEFEFE0A0A0AFEFE99
:101B3000FEFEFE0A0A0AFEFEFEFEFE0A0A0A0AFE71
:101B4000FEFEFE0A0A0A0A0A0AFEFE0A0A0A0A0A31
:101B50000A0A0A0A0A0A0A0A0A0A0AFEFEFEFEFE21
:101B6000FE0A0AFEFEFEFEFEFE0A0AFEFEFEFEFE65
:101B70000A0A0AFEFEFEFEFE0A0A0AFEFEFEFE0A31
:101B80000A0A0AFEFE0A0A0A0A0A0A0A0A0A0A0ACD
:101B90000A0A0A0A0A0A0A0A0A0A0A0A0A0A0AFEB1
:101BA000FEFEFE0A0A0AFEFEFEFEFE0A0A0AFEFE0D
:101BB000FEFEFE0A0AFEFEFEFEFEFE0A0AFEFEFE15
:101BC000FEFEFE0A0AFEFEFEFEFEFE0A0A0A0A0AE1
:101BD0000A0A0A0A0A0A0A0A0A0A0AFEFEFEFE0A95
:101BE0000A0A0AFEFEFEFEFE0A0A0AFEFEFEFEFECD
:101BF0000A0A0AFEFEFEFEFEFE0A0AFEFEFEFEFEC9
:101C0000FE0A0AFEFEFEFEFEFE0A0A0A0A0A0A0A88
:101C10000A0A0A0A0A0A0A0A0A0A0A0A0AFEFEFE48
:101C2000FEFEFE0A0AFEFEFEFEFEFE0A0AFEFEFEA4
:101C3000FEFEFE0A0A0AFEFEFEFEFE0A0A0A0AFE70
:101C4000FEFEFE0A0A0A0A0AFEFEFE0A0A0A0A0A3C
:101C50000A0A0A0A0A0A0A0A0A0A0AFEFEFEFEFE20
:101C6000FE0A0AFEFEFEFEFEFE0A0AFEFEFEFEFE64
:101C7000FE0A0AFEFEFEFEFE0A0A0AFEFEFEFE0A3C
:101C80000A0A0AFEFEFE0A0A0A0A0A0A0A0A0A0AD8
:101C90000A0A0A0A0A0A0A0A0A0A0A0A0A0AFEFEBC
:101CA000FEFEFE0A0A0AFEFEFEFEFE0A0A0AFEFE0C
:101CB000FEFEFE0A0A0A0AFEFEFEFE0A0A0A0A0AD8
:101CC0000AFEFE0A0A0A0A0A0A0AFE0A0A0A0A0A98
:101CD0000A0A0A0A0A0A0A0A0A0A0AFEFEFEFEFEA0
:101CE0000A0A0AFEFEFEFEFE0A0A0AFEFEFEFEFECC
:101CF0000A0A0AFEFEFEFE0A0A0A0AFEFE0A0A0A8C
:101D00000A0A0AFE0A0A0A0A0A0A0A0A0A0A0A0A3F
:101D10000A0A0A0A0A0A0A0A0A0A0A0A0AFEFEFE47
:101D2000FEFEFE0A0A0AFEFEFEFEFE0A0A0A0AFE7F
:101D3000FEFEFE0A0A0A0A0AFEFEFE0A0A0A0A0A4B
:101D40000AFEFE0A0A0A0A0A0A0AFE0A0A0A0A0A17
:101D50000A0A0A0A0A0A0A0A0A0A0AFEFEFEFEFE1F
:101D6000FE0A0AFEFEFEFEFE0A0A0AFEFEFEFE0A4B
:101D70000A0A0AFEFEFE0A0A0A0A0AFEFE0A0A0AFF
:101D80000A0A0AFE0A0A0A0A0A0A0A0A0A0A0A0ABF
:101D90000A0A0A0A0A0A0A0A0A0A0A0A0A0A0AFEAF
:101DA000FEFEFE0A0A0A0AFEFEFEFE0A0A0A0A0AE7
:101DB000FEFEFE0A0A0A0A0AFEFEFE0A0A0A0A0ACB
:101DC0000AFEFE0A0A0A0A0A0A0AFE0A0A0A0A0A97
:101DD0000A0A0A0A0A0A0A0A0A0A0AFEFEFEFE0A93
:101DE0000A0A0AFEFEFEFE0A0A0A0AFEFEFE0A0AA7
:101DF0000A0A0AFEFEFE0A0A0A0A0AFEFE0A0A0A7F
:101E00000A0A0AFE0A0A0A0A0A0A0A0A0A0A0A0A3E
:101E10000A0A0A0A0A0A0A0A0A0A0A0A0AFEFEFE46
:101E2000FEFEFE0A0AFEFEFEFEFEFE0A0AFEFEFEA2
:101E3000FEFEFE0A0AFEFEFEFEFEFE0A0AFEFEFE92
:101E4000FEFEFE0A0A0AFEFEFEFEFE0A0A0A0A0A52
:101E50000A0A0A0A0A0A0A0A0A0A0AFEFEFEFEFE1E
:101E6000FE0A0AFEFEFEFEFEFE0A0AFEFEFEFEFE62
:101E7000FE0A0AFEFEFEFEFEFE0A0AFEFEFEFEFE52
:101E8000FE0A0AFEFEFEFEFE0A0A0A0A0A0A0A0AFA
:101E90000A0A0A0A0A0A0A0A0A0A0A9191919191FF
:101EA00091919191FFFF919191919191FFFF91916A
:101EB00091919191FFFF919191919191FFFF91915A
:101EC00091919191FFFF919191919191FFFFFFFF6E
:101ED000FFFF919191919191919191919191919116
:101EE000919191919191919191919191FFFF919106
:101EF000FFFF9191FFFF9191FFFF9191FFFF919162
:101F0000FFFF919191FFFFFFFF9191919191FFFF51
:101F100091919191919191919191919191919191B1
:101F20009191919191FFFFFF919191919191FFFF7B
:101F3000919191919191FFFF919191919191FFFFD9
:101F4000919191919191FFFF9191919191FFFFFF5B
:101F5000FF91919191919191919191919191919103
:101F60009191919191FFFFFFFF919191FFFF9191CD
:101F7000FFFF9191FFFF91FFFFFF9191FFFFFF9105
:101F8000FFFF9191FFFF9191FFFF919191FFFFFF63
:101F9000FF919191919191919191919191919191C3
:101FA000919191919191FFFF9191919191FFFFFFFB
:101FB000919191919191FFFF919191919191FFFF59
:101FC000919191919191FFFF91919191FFFFFFFF6D
:101FD000FFFF919191919191919191919191919115
:101FE0009191919191FFFFFFFF919191FFFF91914D
:101FF000FFFF9191919191FFFF9191919191FFFF3D
:102000009191919191FFFF9191919191FFFFFFFF2C
:10201000FFFF9191919191919191919191919191D4
:1020200091919191FFFFFFFFFFFF9191919191FF9E
:10203000FF9191919191FFFF91919191919191FFD8
:10204000FF919191FFFF9191FFFF919191FFFFFF10
:10205000FF91919191919191919191919191919102
:1020600091919191919191FFFF9191919191FFFFA8
:10207000FF91919191FFFFFFFF919191FFFF91FFE0
:10208000FF919191FFFFFFFFFFFF9191919191FFD0
:10209000FF919191919191919191919191919191C2
:1020A00091919191FFFFFFFFFFFF9191FFFF9191B0
:1020B00091919191FFFFFFFFFF91919191919191EA
:1020C000FFFF9191FFFF9191FFFF919191FFFFFF22
:1020D000FF91919191919191919191919191919182
:1020E0009191919191FFFFFFFF919191FFFF91914C
:1020F00091919191FFFFFFFFFF919191FFFF9191CE
:10210000FFFF9191FFFF9191FFFF919191FFFFFFE1
:10211000FF91919191919191919191919191919141
:1021200091919191FFFFFFFFFFFF9191919191910B
:10213000FFFF9191919191FFFF9191919191FFFFFB
:102140009191919191FFFF919191919191FFFF91C7
:10215000919191919191919191919191919191916F
:102160009191919191FFFFFFFF919191FFFF9191CB
:10217000FFFF919191FFFFFFFF919191FFFF9191DF
:10218000FFFF9191FFFF9191FFFF919191FFFFFF61
:10219000FF919191919191919191919191919191C1
:1021A0009191919191FFFFFFFF919191FFFF91918B
:1021B000FFFF919191FFFFFFFFFF9191919191910D
:1021C000FFFF9191919191FFFF91919191FFFFFFFD
:1021D0009191919191919191919191848484848430
:1021E00084848484843131313184848431318484A1
:1021F00031318484313184313131848431313184DD
:102200003131848431318484313184848431313179
:1022100031848484848484848484848484848484D1
:10222000848484848484313184848484843131310D
:1022300084848484848431318484848484843131AA
:102240008484848484843131848484843131313140
:1022500031318484848484848484848484848484E4
:102260008484848484313131318484843131848420
:102270003131848484848431318484848484313110
:102280008484848484313184848484843131313100
:1022900031318484848484848484848484848484A4
:1022A0008484848431313131313184848484843133
:1022B000318484848484313184848484848484312A
:1022C0003184848431318484313184848431313166
:1022D0003184848484848484848484848484848411
:1022E00084848484848484313184848484843131FA
:1022F0003184848484313131318484843131843136
:102300003184848431313131313184848484843125
:1023100031848484848484848484848484848484D0
:102320008484848431313131313184843131848405
:1023300084848484313131313184848484848484FC
:102340003131848431318484313184848431313138
:102350003184848484848484848484848484848490
:10236000848484848431313131848484313184841F
:102370008484848431313131318484843131848462
:1023800031318484313184843131848484313131F8
:102390003184848484848484848484848484848450
:1023A00084848484313131313131848484848484DF
:1023B00031318484848484313184848484843131CF
:1023C0008484848484313184848484848431318419
:1023D00084848484848484848484848484848484BD
:1023E000848484848431313131848484313184849F
:1023F0003131848484313131318484843131848435
:102400003131848431318484313184848431313177
:1024100031848484848484848484848484848484CF
:10242000848484848431313131848484313184845E
:1024300031318484843131313131848484848484A1
:102440003131848484848431318484848431313191
:10245000848484848484848484848484848484843C
:102460008484848484843131848484848484313178
:1024700084848484313131313131848484843131B4
:1024800084848484848431318484848484848484B2
:1024900084848484848484848484849191919191BB
:1024A000919191919191919191919191FFFFFFFF64
:1024B000FF919191FFFF9191FFFF9191FFFF91910A
:1024C000FFFF9191FFFF9191FFFF9191FFFF91918C
:1024D000FFFF919191919191919191919191919110
:1024E000919191919191FFFF91919191FFFFFFFF48
:1024F000FFFF91919191FFFF919191919191FFFF38
:10250000919191919191FFFF91919191919191FF71
:10251000FFFF9191919191919191910A0A0A0A0A72
:102520000A0A0A0A0A0A0A0A0A0A0A0A0AFEFEFE2F
:10253000FEFEFE0A0AFEFEFEFEFEFE0A0AFEFEFE8B
:10254000FE83830A0AFEFEFE8383830A0AFEFE835D
:102550008383830A0AFEFE838383830A0A0A0A0AA4
:102560000A0A0A0A0A0A0A0A0A0A0AFEFEFEFEFE07
:10257000FEFEFEFEFEFEFEFEFEFEFE8383838383E2
:10258000838383838383838383838383838383831B
:1025900083838383838383838383830A0A0A0A0A68
:1025A0000A0A0A0A0A0A0A0A0A0A0AFEFEFEFEFEC7
:1025B000FE0A0AFEFEFEFEFEFE0A0A8383FEFEFE01
:1025C000FE0A0A838383FEFEFE0A0A83838383FE58
:1025D000FE0A0A83838383FEFE0A0A0A0AFEFE833A
:1025E0008383830A0AFEFE838383830A0AFEFE83B3
:1025F0008383830A0AFEFE838383830A0AFEFE83A3
:102600008383830A0AFEFE838383830A0AFEFE8392
:102610008383830A0AFEFE83838383838383838386
:10262000838383838383838383838383838383837A
:10263000838383838383838383838383838383836A
:10264000838383838383838383838383838383835A
:10265000838383838383838383838383838383834A
:1026600083838383FFFFFFFFFF838383FFFF8383D6
:10267000FFFF8383FFFF8383FFFF8383FFFFFFFF52
:10268000FF838383FFFF838383838383FFFF8383AE
:10269000838383838383838383838383838383830A
:1026A00083838383838383838383838383FFFFFF86
:1026B000FF83838383838383FFFF838383FFFFFF02
:1026C000FFFF8383FFFF8383FFFF838383FFFFFF7E
:1026D000FFFF8383838383838383838383838383D2
:1026E000838383838383838383838383FFFF8383C2
:1026F000FFFF8383FFFF8383FFFF8383FFFF8383CA
:10270000FFFF8383FFFF8383FFFF838383FFFFFF3D
:10271000FFFF838383838383838383838383838391
:1027200083838383838383838383838383FFFFFF05
:10273000FFFF8383FFFF83838383838383FFFFFF05
:10274000FF83838383838383FFFF8383FFFFFFFFF5
:10275000FF838383838383838383838383838383CD
:1027600083838383838383838383838383FFFFFFC5
:10277000FF838383FFFF8383FFFF8383FFFFFFFFCD
:10278000FFFF8383FFFF83838383838383FFFFFFB5
:10279000FF8383838383838383838383838383838D
:1027A0008383838383838383FFFF83838383838301
:1027B000FFFF838383FFFFFFFFFF8383FFFF83838D
:1027C000FFFF8383FFFF8383FFFF838383FFFFFF7D
:1027D000FFFF83838383838383838383838383FE56
:1027E000FE0A0A83838383FEFE0A0A83838383FEB1
:1027F000FE0A0A83838383FEFE0A0A83838383FEA1
:10280000FE0A0A83838383FEFE0A0A83838383FE90
:10281000FE0A0A83838383FEFE0A0A40404040E1A9
:10282000E1E1E140404040E1E1E1E1404040404041
:10283000E1E1E1404040404040E1E1404040404073
:102840004040404040404040404040404040404088
:102850004040404040404040404040E1E1E1E1E153
:10286000E1E1E1E1E1E1E1E1E1E1E1E1E1E1E1E158
:10287000E1E1E1E1E1E1E1E1E1E1E140404040406D
:102880004040404040404040404040404040404048
:102890004040404040404040404040E1E1E1E140B4
:1028A000404040E1E1E1E140404040E1E1E14040C1
:1028B000404040E1E14040404040404040404040D6
:1028C0004040404040404040404040404040404008
:1028D00040404040404040404040408383838383A9
:1028E00083838383838383838383838383838383B8
:1028F000838383FFFFFFFFFFFFFFFFFFFFFFFFFF5C
:10290000FFFFFF8383838383838383838383838323
:102910008383838383838383838383838383FF830B
:10292000838383838383FFFF838383838383FFFF87
:10293000FF8383838383FFFFFFFF83838383FFFF03
:10294000FF8383838383FFFF838383838383FF8367
:102950008383838383838383838383838383838347
:1029600083838383FFFFFFFFFF838383FFFF8383D3
:10297000FFFF8383FFFF8383FFFF8383FFFFFFFF4F
:10298000FF838383FFFF83FFFF838383FFFF8383B3
:10299000FFFF83838383838383838383838383830F
:1029A000838383838383838383838383FFFF8383FF
:1029B000FFFF8383FFFFFFFFFFFFFF83FFFFFFFF9B
:1029C000FFFFFF83FFFF83FF83FFFF83FFFF8383FF
:1029D00083FFFF83838383838383838383838383CF
:1029E0008383838383FFFFFFFF838383FFFF8383CF
:1029F000FFFF8383FFFF8383FFFF8383FFFF8383C7
:102A0000FFFF8383FFFF83FFFF83838383FFFF83B6
:102A1000FFFF83838383838383838383838383838E
:102A2000838383838383FFFF83838383838383837E
:102A30008383838383FFFFFF838383838383FFFFFA
:102A4000838383838383FFFF8383838383FFFFFFEA
:102A5000FF838383838383838383838383838383CA
:102A6000838383838383FFFF83838383FFFFFFFF4E
:102A7000FFFF83838383FFFF838383838383FFFF3E
:102A8000838383838383FFFF83838383838383FFA2
:102A9000FFFF83838383838383838383838383830E
:102AA00083838383FFFF838383FFFF83FFFFFF8392
:102AB000FFFFFF83FFFFFFFFFFFFFF83FFFF83FF9A
:102AC00083FFFF83FFFF838383FFFF83FFFF8383F6
:102AD00083FFFF83838383838383838383838383CE
:102AE00083838383838383838383838383FFFFFF42
:102AF000FF838383FFFF838383838383FFFF83833A
:102B000083838383FFFF83838383838383FFFFFF29
:102B1000FF83838383838383838383838383838309
:102B20008383838383FFFFFFFF838383FFFF83838D
:102B3000FFFF8383FFFF8383FFFF8383FFFF838385
:102B4000FFFF8383FFFF8383FFFF838383FFFFFFF9
:102B5000FF838383838383838383838383838383C9
:102B6000838383838383838383838383FFFFFFFF45
:102B7000FF838383FFFF8383FFFF8383FFFF8383C1
:102B8000FFFF8383FFFF8383FFFF8383FFFF838335
:102B9000FFFF83838383838383838383838383830D
:102BA00083838383838383FFFFFF83838383FFFF89
:102BB0008383838383FFFFFFFFFF83838383FFFF81
:102BC000838383838383FFFF838383838383FFFFE5
:102BD00083838383838383838383838484848484C0
:102BE00084848484848484848484848484848484A5
:102BF0008484848484848484848484848484848495
:102C00008484848484848484848484848484848484
:102C100084848484848484848484840A0AFEFE8375
:102C20008383830A0AFEFE838383830A0AFEFEFEF1
:102C30008383830A0AFEFEFEFE83830A0AFEFEFEEB
:102C4000FEFEFE0A0AFEFEFEFEFEFE0A0A0A0A0A50
:102C50000A0A0A0A0A0A0A0A0A0A0A838383838377
:102C60008383838383838383838383838383838334
:102C70008383838383838383838383FEFEFEFEFEBD
:102C8000FEFEFEFEFEFEFEFEFEFEFE0A0A0A0A0A28
:102C90000A0A0A0A0A0A0A0A0A0A0A83838383FEBC
:102CA000FE0A0A83838383FEFE0A0A838383FEFE71
:102CB000FE0A0A8383FEFEFEFE0A0AFEFEFEFEFEFA
:102CC000FE0A0AFEFEFEFEFEFE0A0A0A0A0A0A0AB8
:102CD0000A0A0A0A0A0A0A0A0A0A0A373737373773
:102CE00037373737373737373737371C1C1C1C1CFB
:102CF0001C1C1C1C1C1C1C1C1C1C1C1C1C1C1C1C14
:102D00001C1C1C1C1C1C1C1C1C1C1C37373737377C
:102D10003737373737373737373737373737373743
:102D200037373737373737373737372A1C1C1C1CAC
:102D30001C1C1C2A1C1C1C1C1C1C1C2A1C1C1C1CB7
:102D40001C1C1C2A1C1C1C1C1C1C1C37373737372E
:102D50003737373737373737373737373737373703
:102D600037373737373737373737372A2A1C1C1C5E
:102D70001C1C1C2A2A1C1C1C1C1C1C2A2A1C1C1C5B
:102D80001C1C1C2A2A1C1C1C1C1C1C3737373737E0
:102D900037373737373737373737373737373737C3
:102DA00037373737373737373737372A2A2A1C1C10
:102DB0001C1C1C2A2A2A1C1C1C1C1C2A2A2A1C1CFF
:102DC0001C1C1C2A2A2A1C1C1C1C1C373737373792
:102DD0003737373737373737373737373737373783
:102DE00037373737373737373737372A2A2A2A1CC2
:102DF0001C1C1C2A2A2A2A1C1C1C1C2A2A2A2A1CA3
:102E00001C1C1C2A2A2A2A1C1C1C1C373737373743
:102E10003737373737373737373737373737373742
:102E200037373737373737373737372A2A2A2A2A73
:102E30001C1C1C2A2A2A2A2A1C1C1C2A2A2A2A2A46
:102E40001C1C1C2A2A2A2A2A1C1C1C3737373737F5
:102E50003737373737373737373737373737373702
:102E600037373737373737373737372A2A2A2A2A33
:102E70002A1C1C2A2A2A2A2A2A1C1C2A2A2A2A2AEA
:102E80002A1C1C2A2A2A2A2A2A1C1C373737373799
:102E900037373737373737373737373737373737C2
:102EA00037373737373737373737372A2A2A2A2AF3
:102EB0002A2A1C2A2A2A2A2A2A2A1C2A2A2A2A2A8E
:102EC0002A2A1C2A2A2A2A2A2A2A1C37373737373D
:102ED0003737373737373737373737373737373782
:102EE00037373737373737373737372A2A2A2A2AB3
:102EF0002A2A2A2A2A2A2A2A2A2A2A2A2A2A2A2A32
:102F00002A2A2A2A2A2A2A2A2A2A2A3737373737E0
:102F1000373737373737373737373740404040371D
:102F200037373740404040373737374040404040E0
:102F300037373740404040404037374040404040BE
:102F40004040404040404040404040404040404081
:102F5000404040404040404040404037373737379E
:102F600037373737373737373737373737373737F1
:102F700037373737373737373737374040404040B4
:102F80004040404040404040404040404040404041
:102F90004040404040404040404040373737374055
:102FA0004040403737373740404040373737404060
:102FB0004040403737404040404040404040404023
:102FC0004040404040404040404040404040404001
:102FD00040404040404040404040404040404040F1
:102FE0004037374040404040373737404040403717
:102FF0003737374040404037373737404040403719
:1030000037373740404040373737374040404040FF
:1030100037373740404040404037373737404040EF
:1030200040404037373740404040403737373740DF
:1030300040404037373737404040403737373740D8
:1030400040404037373737404040403737374040BF
:103050004040403737404040404040838383838333
:1030600083838383FFFF838383838383FFFF838340
:1030700083838383FFFF838383838383FFFF838330
:1030800083838383FFFF838383838383FFFFFFFF28
:10309000FFFF838383838383838383838383838308
:1030A000838383838383838383838383FFFF8383F8
:1030B000FFFF8383FFFF8383FFFF8383FFFF838300
:1030C000FFFF838383FFFFFFFF8383838383FFFFF0
:1030D00083838383838383838383838383838383C0
:1030E0008383838383FFFFFF838383838383FFFF44
:1030F000838383838383FFFF838383838383FFFFB0
:10310000838383838383FFFF8383838383FFFFFF23
:10311000FF83838383838383838383838383838303
:1031200083838383FFFF8383FFFF8383FFFF838387
:10313000FFFF8383FFFF8383FFFF8383FFFF83837F
:10314000FFFF8383FFFF8383FFFF8383FFFFFFFF77
:10315000FFFF838383838383838383838383838347
:10316000838383838383838383838383FFFFFFFF3F
:10317000FF838383FFFF8383FFFF8383FFFF8383BB
:10318000FFFF8383FFFFFFFFFF838383FFFF8383B3
:1031900083838383FFFF8383838383838383838307
:1031A0008383838383FFFFFFFFFF8383FFFF83838B
:1031B00083838383FFFF838383838383FFFF83FF73
:1031C000FFFF8383FFFF8383FFFF838383FFFFFF73
:1031D000FFFF8383838383838383838383838383C7
:1031E000838383838383838383838383FFFFFFFFBF
:1031F000FF838383FFFF8383FFFF8383FFFF83833B
:1032000083838383FFFF838383838383FFFF83839E
:10321000838383838383838383838383838383837E
:10322000838383838383FFFF838383838383FFFF7E
:10323000838383838383FFFF838383838383FFFF6E
:103240008383838383838383838383838383FFFF56
:10325000838383838383838383838383838383833E
:10326000838383838383FF83838383838383FFFFBA
:10327000838383838383FFFFFF8383838383FFFFB2
:10328000FFFF83838383FFFFFF8383838383FFFFAA
:10329000838383838383FF83838383838383838382
:1032A00083838383838383FF838383838383FFFF7A
:1032B0008383838383FFFFFF83838383FFFFFFFF7A
:1032C0008383838383FFFFFF838383838383FFFF62
:1032D00083838383838383FF838383838383838342
:1032E00083838383FFFF8383FFFF8383FFFFFF834A
:1032F000FFFF8383FFFFFFFFFFFF8383FFFFFFFFCE
:10330000FFFF8383FFFF83FFFFFF8383FFFF838331
:10331000FFFF838383838383838383838383838385
:1033200083838383838383838383838383FFFFFFF9
:10333000FF838383FFFF8383FFFF8383FFFF8383F9
:10334000FFFF8383FFFF8383FFFF838383FFFFFFF1
:10335000FF8383838383838383838301010001014C
:10336000010101020101030101040101050101063E
:10337000010107010108FEFEFFFFFFFEFEFEFEFF4A
:10338000FFFFFFFEFEFEFFFFFFFEFEFEFEFEFFFF55
:10339000FEFEFEFEFEFEFFFFFEFEFEFEFEFEFEFE4B
:1033A000FEFEFEFEFEFEFEFEFEFEFEFEFEFEFEFE3D
:1033B000FEFEFEFEFEFEFEFEFEFFFFFFFEFEFEFE2A
:1033C000FEFFFFFFFFFEFEFEFEFEFEFFFFFFFEFE16
:1033D000FEFEFEFEFFFFFEFEFEFEFEFEFFFFFEFE09
:1033E000FEFEFEFEFEFEFEFEFEFEFEFEFEFEFEFEFD
:1033F000FEFEFEFEFEFEFEFEFEFEFEFEFEFEFEFEED
:10340000FEFEFEFEFEFEFEFEFEFEFEFEFEFEFFFFDA
:10341000FEFEFEFEFEFEFFFFFEFEFEFEFEFEFFFFC8
:10342000FFFEFEFEFEFEFEFFFFFFFFFEFEFEFEFEB7
:10343000FFFFFFFEFEFEFEFEFEFEFEFEFEFEFEFEA9
:10344000FEFEFEFEFEFEFEFEFEFEFEFEFEFEFEFE9C
:10345000FEFEFEFEFFFFFEFEFEFEFEFEFFFFFEFE88
:10346000FEFEFEFFFFFFFEFEFEFFFFFFFFFEFEFE75
:10347000FEFFFFFFFEFEFEFEE8E8E8FEFEFEFEE8C1
:10348000E8E8E8FEFEFEE8E8E8FEFEFEFEFEE8E80C
:10349000FEFEFEFEFEFEE8E8FEFEFEFEFEFEFEFE78
:1034A000FEFEFEFEFEFEFEFEFEFEFEFEFEFEFEFE3C
:1034B000FEFEFEFEFEFEFEFEFEE8E8E8FEFEFEFE6E
:1034C000FEE8E8E8E8FEFEFEFEFEFEE8E8E8FEFEB6
:1034D000FEFEFEFEE8E8FEFEFEFEFEFEE8E8FEFE64
:1034E000FEFEFEFEFEFEFEFEFEFEFEFEFEFEFEFEFC
:1034F000FEFEFEFEFEFEFEFEFEFEFEFEFEFEFEFEEC
:10350000FEFEFEFEFEFEFEFEFEFEFEFEFEFEE8E807
:10351000FEFEFEFEFEFEE8E8FEFEFEFEFEFEE8E823
:10352000E8FEFEFEFEFEFEE8E8E8E8FEFEFEFEFE29
:10353000E8E8E8FEFEFEFEFEFEFEFEFEFEFEFEFEED
:10354000FEFEFEFEFEFEFEFEFEFEFEFEFEFEFEFE9B
:10355000FEFEFEFEE8E8FEFEFEFEFEFEE8E8FEFEE3
:10356000FEFEFEE8E8E8FEFEFEE8E8E8E8FEFEFE15
:10357000FEE8E8E8FEFEFEFEFEFEFEFEFEFEFEFEAD
:10358000FEFEFDFEFEFEFEFEFDFEFDFEFDFEFEFE5F
:10359000FEFDFDFDFEFEFEFDFDFDFEFDFDFDFEFE54
:1035A000FEFDFDFDFEFEFEFEFDFEFDFEFDFEFEFE41
:1035B000FEFEFDFEFEFEFEFEFEFEFEFEFEFEFEFE2C
:1035C000FEFEFEFEFEFEFEFEFEFEFEFEFEFEFEFE1B
:1035D000FEFEFEFEFEFEFEFEFEFEFEFEFEFEFEFE0B
:1035E000FEFEFEFEFEFEFEFEFEFEFEFEFEFEFEFEFB
:1035F000FEFEFEFEFEFE0804208081828384858616
:103600008E8F9091929394959E9FA0A1A2A3A4A522
:10361000ABACAD8B8B8BAEAF08038788898A8B8B65
:103620008C8D969798999A9B9C9D2020A6A7A8A9D7
:10363000AA2000000000000000000000FFFF00FFC3
:10364000FF0000FFFFFFFFFFFFFF00FFFFFFFFFF87
:10365000FFFF0000FFFFFFFFFF00000000FFFFFF74
:10366000000000000000FF0000000000000000005B
:103670000000000000FFFF000000000000FFFF004E
:103680000000000000FFFF000000000000FFFFFF3F
:10369000FFFF000000FFFFFFFFFF000000FFFF0033
:1036A0000000000000FFFF000000000000FFFF001E
:1036B0000000000000000000FFFF0000000000000C
:1036C000FFFF000000000000FFFF000000000000FE
:1036D000FFFF000000000000FFFF000000000000EE
:1036E000FFFF000000000000FFFF000000000000DE
:1036F000FFFF000000FFFF000000000000FFFF00D0
:103700000000000000FFFF000000FFFFFFFFFF00C0
:103710000000FFFFFFFFFF000000000000000000AE
:103720000000000000000000000000000000000099
:103730000000000000FFFF000000000000FFFF008D
:103740000000000000FFFF000000FFFFFFFFFF0080
:103750000000FFFFFFFFFF000000000000FFFF0070
:103760000000000000FFFF000000000000FFFF005D
:103770000000000000000000000000000000000049
:1037800000000000000000000000FFFFFFFFFF003E
:103790000000FFFFFFFFFF000000000000FFFF0030
:1037A0000000000000FFFF000000000000FFFF001D
:1037B0000000000000000000FFFF0000000000FF0C
:1037C000FFFF00000000FFFFFF00000000FFFFFF01
:1037D00000000000FFFFFF00000000FFFFFF0000EF
:1037E0000000FFFFFF0000000000FFFF00000000DE
:1037F0000000FFFF000000000000FFFFFF000000CE
:10380000000000FFFFFF000000000000FFFFFF00BE
:103810000000000000FFFFFF000000000000FFFFAD
:10382000FF000000000000FFFFFF0000000000009C
:10383000FFFF00000000000000FF0000000000008B
:10384000FFFF0000000000FFFFFF00000000FFFF7F
:10385000FFFF000000FFFFFFFFFF0000FFFFFFFF73
:10386000FFFF00FFFFFFFFFFFFFFFFFFFFFFFFFF67
:10387000FFFF00000000000000000000000000004A
:103880000000000000000000000000000000000038
:10389000000000000000FFFFFFFF00000000FFFF2E
:1038A000FFFF00000000FFFFFFFF00000000FFFF20
:1038B000FFFFFF00000000000000FFFF000000000D
:1038C0000000FFFFFF0000000000FFFFFFFF0000FF
:1038D0000000FFFFFFFFFF000000FFFFFFFFFFFFF3
:1038E0000000FFFFFFFFFFFFFF00FFFFFFFFFFFFE5
:1038F000FFFF00000000FFFFFFFF00000000FFFFD0
:10390000FFFF00000000FFFFFFFF00000000FFFFBF
:10391000FFFF0000000000000000000000000000A9
:103920000000000000000000000000000000000097
:103930000000FFFFFFFF00000000FFFFFFFF00008F
:103940000000FFFFFFFF00000000FFFFFFFF00007F
:103950000000000000000000000000000000000067
:103960000000000000000000000000000000000057
:103970000000FFFFFFFFFFFFFFFFFFFFFFFFFFFF55
:10398000FFFF000000000000000000000000000039
:103990000000000000000000000000000000000027
:1039A0000000000000000000000000000000000017
:1039B0000000000000000000000000000000000007
:1039C00000000000000000000000000000000000F7
:1039D00000000000000000000000000000000000E7
:1039E0000000FFFFFFFFFFFFFFFFFFFFFFFFFFFFE5
:1039F000FFFF0000000000000000000000000000C9
:103A000000000000000000000000000000000000B6
:103A10000000FFFFFFFF00000000FFFFFFFF0000AE
:103A20000000FFFFFFFF00000000FFFFFFFF00009E
:103A300000000000000000000000000000FFFFFF89
:103A40000000000000FFFFFF000000FFFFFF00FF7D
:103A5000FFFF00FFFFFF00FFFFFF00000000FF006F
:103A60000000000000FFFFFF000000000000000059
:103A70000000000000000000000000000000000046
:103A800000000000000000000000000000FFFFFF39
:103A9000FFFF000000FFFFFFFFFF000000FFFF002F
:103AA0000000000000FFFF000000000000FFFF001A
:103AB0000000000000000000000000000000000006
:103AC00000000000000000000000FFFFFFFFFFFFFC
:103AD000FFFFFFFFFFFFFFFFFFFF000000000000F0
:103AE00000000000000000000000000000000000D6
:103AF0000000000000FFFF000000000000FFFF00CA
:103B00000000000000FFFF000000FFFFFFFFFFFFBD
:103B1000FFFFFFFFFFFFFFFFFFFF000000FFFF00B1
:103B20000000000000FFFF000000000000FFFF0099
:103B30000000000000000000000000000000000085
:103B400000000000FFFFFFFF000000FFFFFFFFFF7E
:103B5000FF0000FFFFFFFFFFFF0000FFFFFFFFFF71
:103B6000FF000000FFFFFFFF00000000000000005A
:103B70000000000000000000000000000000000045
:103B80000000000000000000000000000000000035
:103B90000000FFFFFFFFFFFFFFFFFFFFFFFFFFFF33
:103BA000FFFFFFFFFFFFFFFFFFFFFFFFFFFFFFFF25
:103BB000FFFFFFFF000000000000FFFF000000000B
:103BC0000000FFFF000000000000FFFF00000000F9
:103BD0000000FFFF000000000000FFFF00000000E9
:103BE0000000FFFF000000000000FFFF00000000D9
:103BF00000000000000000000000000000000000C5
:103C000000000000000000000000FFFFFFFFFFFFBA
:103C1000FFFFFFFFFFFFFFFFFFFF000000FFFF00B0
:103C20000000000000FFFF000000000000FFFF0098
:103C30000000000000FFFF000000000000FFFF0088
:103C40000000000000FFFF000000FFFFFFFFFFFF7C
:103C5000FFFFFFFFFFFFFFFFFFFF0000000000006E
:103C60000000000000000000000000000000000054
:103C70000000FFFFFFFF00000000FFFFFFFF00004C
:103C80000000FFFFFFFF00000000FFFFFFFF00003C
:103C90000000FFFFFFFF00000000FFFFFFFF00002C
:103CA0000000FFFFFFFF00000000FFFFFFFF00001C
:103CB0000000000000FFFF000000000000FFFF0008
:103CC0000000000000FFFF000000000000FFFFFFF9
:103CD000FFFF000000FFFFFFFFFF000000000000EB
:103CE00000000000000000000000000000000000D4
:103CF000000000FFFFFFFF00000000FFFF000000CA
:103D0000000000FFFFFFFF00000000FFFF000000B9
:103D1000000000FFFFFFFFFFFF00000000FFFF00AB
:103D20000000000000FFFFFFFF0000000000000097
:103D300000000000000000000000000000FFFF0085
:103D400000000000FFFFFFFF000000FFFFFFFFFF7C
:103D5000FF00000000FFFF000000000000FFFF0068
:103D60000000000000FFFF00000000000000000055
:103D700000000000000000000000000000FFFF0045
:103D80000000000000FFFF000000000000FFFF0037
:103D9000000000FFFFFFFFFFFF000000FFFFFFFF2D
:103DA0000000000000FFFF00000000000000000015
:103DB00000000000000000000000000000FFFF0005
:103DC00000000000FFFF0000000000FFFFFFFFFFFA
:103DD000FF000000FFFF00000000000000FFFF00E8
:103DE00000000000000000000000000000000000D3
:103DF00000000000000000000000000000FFFF00C5
:103E0000000000000000FFFF000000FFFFFFFFFFB9
:103E1000FF0000000000FFFF0000000000FFFF00A7
:103E20000000000000000000000000000000000092
:103E30000000000000000000000000000000000082
:103E40000000000000000000000000000000000072
:103E50000000000000000000000000000000000062
:103E60000000000000000000000000000000000052
:103E700000000000000000000000000000FFFF0044
:103E80000000000000FFFF000000000000FFFF0036
:103E90000000000000FFFF00000000000000000024
:103EA0000000000000FFFF00000000000000000014
:103EB0000000000000000000000000FFFF0000FF05
:103EC000FF0000FFFF0000FFFF0000FFFF0000FFFA
:103ED000FF000000000000000000000000000000E3
:103EE00000000000000000000000000000000000D2
:103EF0000000000000000000000000FFFF0000FFC5
:103F0000FF00FFFFFFFFFFFFFFFF00FFFF0000FFBD
:103F1000FF0000FFFF0000FFFF00FFFFFFFFFFFFAC
:103F2000FFFF00FFFF0000FFFF0000000000000097
:103F30000000000000FFFF0000000000FFFFFFFF87
:103F4000FF0000FFFF00000000000000FFFFFFFF78
:103F500000000000000000FFFF0000FFFFFFFFFF68
:103F60000000000000FFFF00000000000000000053
:103F70000000000000000000000000FFFF0000FF44
:103F8000FF0000FFFF00FFFF0000000000FFFF0038
:103F900000000000FFFF0000000000FFFF0000FF26
:103FA000FF0000FF000000FFFF0000000000000015
:103FB0000000000000FFFFFF00000000FFFF00FF07
:103FC000FF00000000FFFFFF00000000FFFFFF00F8
:103FD000000000FFFF00FFFFFFFF00FFFF0000FFEA
:103FE000FF000000FFFFFF00FFFF000000000000D7
:103FF00000000000000000000000000000FFFF00C3
:104000000000000000FFFF000000000000FFFF00B4
:1040100000000000000000000000000000000000A0
:104020000000000000000000000000000000000090
:104030000000000000000000000000000000FFFF82
:10404000FF00000000FFFFFF0000000000FFFF0076
:104050000000000000FFFF000000000000FFFFFF65
:10406000000000000000FFFFFF0000000000000053
:104070000000000000000000000000FFFFFF000043
:1040800000000000FFFFFF000000000000FFFF0035
:104090000000000000FFFF0000000000FFFFFF0025
:1040A000000000FFFFFF0000000000000000000013
:1040B0000000000000000000000000FFFF0000FF03
:1040C000FF000000FFFFFFFF0000FFFFFFFFFFFFFB
:1040D000FFFF0000FFFFFFFF000000FFFF0000FFE9
:1040E000FF000000000000000000000000000000D1
:1040F00000000000000000000000000000FFFF00C2
:104100000000000000FFFF00000000FFFFFFFFFFB6
:10411000FF00000000FFFF000000000000FFFF00A4
:10412000000000000000000000000000000000008F
:10413000000000000000000000000000000000007F
:10414000000000000000000000000000000000006F
:1041500000000000000000000000000000FFFF0061
:104160000000000000FFFF0000000000FFFF000053
:10417000000000000000000000000000000000003F
:104180000000000000000000000000FFFFFFFFFF34
:10419000FF00000000000000000000000000000020
:1041A000000000000000000000000000000000000F
:1041B00000000000000000000000000000000000FF
:1041C00000000000000000000000000000000000EF
:1041D00000000000000000000000000000FFFF00E1
:1041E0000000000000FFFF000000000000000000D1
:1041F000000000000000000000000000000000FFC0
:10420000FF0000000000FFFF0000000000FFFF00B3
:1042100000000000FFFF0000000000FFFF000000A2
:10422000000000FF0000000000000000000000008F
:10423000000000000000000000000000FFFFFFFF82
:10424000000000FFFF0000FFFF0000FFFF00FFFF76
:10425000FF0000FFFFFF00FFFF0000FFFF0000FF67
:10426000FF000000FFFFFFFF000000000000000053
:1042700000000000000000000000000000FFFF0040
:1042800000000000FFFFFF000000000000FFFF0033
:104290000000000000FFFF000000000000FFFF0022
:1042A000000000FFFFFFFFFFFF0000000000000014
:1042B000000000000000000000000000FFFFFFFF02
:1042C000000000FFFF0000FFFF0000000000FFFFF4
:1042D0000000000000FFFF0000000000FFFF0000E2
:1042E000000000FFFFFFFFFFFF00000000000000D4
:1042F0000000000000000000000000FFFFFFFFFFC3
:10430000FF0000000000FFFF0000000000FFFF00B2
:10431000000000000000FFFF000000FFFF0000FFA2
:10432000FF000000FFFFFFFF000000000000000092
:104330000000000000000000000000000000FFFF7F
:104340000000000000FFFFFF00000000FFFFFFFF74
:10435000000000FFFF00FFFF000000FFFFFFFFFF66
:10436000FF0000000000FFFF000000000000000050
:104370000000000000000000000000FFFFFFFFFF42
:10438000FF0000FFFF000000000000FFFFFFFFFF35
:1043900000000000000000FFFF0000FFFF0000FF22
:1043A000FF000000FFFFFFFF000000000000000012
:1043B000000000000000000000000000FFFFFFFF01
:1043C000000000FFFF000000000000FFFFFFFFFFF4
:1043D000000000FFFF0000FFFF0000FFFF0000FFE4
:1043E000FF000000FFFFFFFF0000000000000000D2
:1043F0000000000000000000000000FFFFFFFFFFC2
:10440000FF000000000000FFFF0000000000FFFFB1
:104410000000000000FFFF0000000000FFFF0000A0
:1044200000000000FFFF000000000000000000008E
:10443000000000000000000000000000FFFFFFFF80
:10444000000000FFFF0000FFFF000000FFFFFFFF74
:10445000000000FFFF0000FFFF0000FFFF0000FF63
:10446000FF000000FFFFFFFF000000000000000051
:10447000000000000000000000000000FFFFFFFF40
:10448000000000FFFF0000FFFF000000FFFFFFFF34
:10449000FF000000000000FFFF0000000000FFFF21
:1044A00000000000FFFFFF0000000000000000000F
:1044B00000000000000000000000000000000000FC
:1044C0000000000000FFFF000000000000FFFF00F0
:1044D00000000000000000000000000000FFFF00DE
:1044E0000000000000FFFF000000000000000000CE
:1044F00000000000000000000000000000000000BC
:104500000000000000FFFF000000000000FFFF00AF
:1045100000000000000000000000000000FFFF009D
:104520000000000000FFFF0000000000FFFF00008F
:1045300000000000000000FFFF0000000000FFFF7F
:104540000000000000FFFF0000000000FFFF00006F
:104550000000000000FFFF00000000000000FFFF5F
:1045600000000000000000FFFF000000000000004D
:10457000000000000000000000000000000000003B
:10458000000000FFFFFFFFFFFF0000000000000031
:104590000000000000000000000000FFFFFFFFFF20
:1045A000FF0000000000000000000000000000000C
:1045B000000000FFFF00000000000000FFFF0000FF
:1045C0000000000000FFFF00000000000000FFFFEF
:1045D0000000000000FFFF0000000000FFFF0000DF
:1045E000000000FFFF0000000000000000000000CD
:1045F000000000000000000000000000FFFFFFFFBF
:10460000000000FFFF0000FFFF0000000000FFFFB0
:104610000000000000FFFF0000000000000000009C
:104620000000000000FFFF0000000000000000008C
:10463000000000000000000000000000FFFFFFFF7E
:10464000000000FFFF0000FFFF0000FFFF00FFFF72
:10465000FF0000FFFF00FFFFFF0000FFFF00000062
:1046600000000000FFFFFFFFFF000000000000004F
:1046700000000000000000000000000000FFFF003C
:1046800000000000FFFFFFFF000000FFFF0000FF31
:10469000FF0000FFFF0000FFFF0000FFFFFFFFFF24
:1046A000FF0000FFFF0000FFFF000000000000000F
:1046B0000000000000000000000000FFFFFFFFFFFF
:1046C000000000FFFF0000FFFF0000FFFFFFFFFFF3
:1046D000000000FFFF0000FFFF0000FFFF0000FFE1
:1046E000FF0000FFFFFFFFFF0000000000000000D0
:1046F000000000000000000000000000FFFFFFFFBE
:10470000000000FFFF0000FFFF0000FFFF000000AF
:10471000000000FFFF000000000000FFFF0000FF9E
:10472000FF000000FFFFFFFF00000000000000008E
:104730000000000000000000000000FFFFFFFF007D
:10474000000000FFFF00FFFF000000FFFF0000FF70
:10475000FF0000FFFF0000FFFF0000FFFF00FFFF62
:10476000000000FFFFFFFF0000000000000000004D
:104770000000000000000000000000FFFFFFFFFF3E
:10478000FF0000FFFF000000000000FFFFFFFFFF31
:10479000000000FFFF000000000000FFFF0000001D
:1047A000000000FFFFFFFFFFFF000000000000000F
:1047B0000000000000000000000000FFFFFFFFFFFE
:1047C000FF0000FFFF000000000000FFFFFFFFFFF1
:1047D000000000FFFF000000000000FFFF000000DD
:1047E000000000FFFF0000000000000000000000CB
:1047F000000000000000000000000000FFFFFFFFBD
:10480000FF0000FFFF000000000000FFFF000000AD
:10481000000000FFFF00FFFFFF0000FFFF0000FFA0
:10482000FF000000FFFFFFFFFF000000000000008E
:104830000000000000000000000000FFFF0000FF7B
:10484000FF0000FFFF0000FFFF0000FFFFFFFFFF72
:10485000FF0000FFFF0000FFFF0000FFFF0000FF60
:10486000FF0000FFFF0000FFFF000000000000004D
:104870000000000000000000000000FFFFFFFFFF3D
:10488000FF00000000FFFF000000000000FFFF002D
:104890000000000000FFFF000000000000FFFF001C
:1048A000000000FFFFFFFFFFFF000000000000000E
:1048B0000000000000000000000000000000FFFFFA
:1048C000FF000000000000FFFF000000000000FFEC
:1048D000FF000000000000FFFF0000FFFF0000FFDE
:1048E000FF000000FFFFFFFF0000000000000000CD
:1048F0000000000000000000000000FFFF0000FFBB
:10490000FF0000FFFF00FFFF000000FFFFFFFF00B0
:10491000000000FFFFFFFF00000000FFFF00FFFF9F
:10492000000000FFFF0000FFFF000000000000008B
:104930000000000000000000000000FFFF00000079
:10494000000000FFFF000000000000FFFF0000006B
:10495000000000FFFF000000000000FFFF0000005B
:10496000000000FFFFFFFFFFFF000000000000004D
:104970000000000000000000000000FFFF00000039
:10498000FFFF00FFFFFF00FFFFFF00FFFFFFFFFF34
:10499000FFFF00FFFF00FF00FFFF00FFFF00000020
:1049A000FFFF00FFFF000000FFFF0000000000000D
:1049B0000000000000000000000000FFFF0000FFFA
:1049C000FF0000FFFFFF00FFFF0000FFFFFFFFFFF2
:1049D000FF0000FFFFFFFFFFFF0000FFFF00FFFFE2
:1049E000FF0000FFFF0000FFFF00000000000000CC
:1049F000000000000000000000000000FFFFFFFFBB
:104A0000000000FFFF0000FFFF0000FFFF0000FFAD
:104A1000FF0000FFFF0000FFFF0000FFFF0000FF9E
:104A2000FF000000FFFFFFFF00000000000000008B
:104A30000000000000000000000000FFFFFFFFFF7B
:104A4000000000FFFF0000FFFF0000FFFF0000FF6D
:104A5000FF0000FFFFFFFFFF000000FFFF0000005E
:104A6000000000FFFF000000000000000000000048
:104A7000000000000000000000000000FFFFFFFF3A
:104A8000000000FFFF0000FFFF0000FFFF0000FF2D
:104A9000FF0000FFFF0000FFFF0000FFFF00FFFF1F
:104AA00000000000FFFF00FFFF000000000000000A
:104AB0000000000000000000000000FFFFFFFFFFFB
:104AC000000000FFFF0000FFFF0000FFFF0000FFED
:104AD000FF0000FFFFFFFFFF000000FFFF00FFFFE0
:104AE000000000FFFF0000FFFF00000000000000CA
:104AF000000000000000000000000000FFFFFFFFBA
:104B0000000000FFFF00000000000000FFFFFFFFAB
:104B100000000000000000FFFF000000000000FF98
:104B2000FF000000FFFFFFFF00000000000000008A
:104B30000000000000000000000000FFFFFFFFFF7A
:104B4000FF00000000FFFF000000000000FFFF006A
:104B50000000000000FFFF000000000000FFFF0059
:104B60000000000000FFFF00000000000000000047
:104B70000000000000000000000000FFFF0000FF38
:104B8000FF0000FFFF0000FFFF0000FFFF0000FF2D
:104B9000FF0000FFFF0000FFFF0000FFFF0000FF1D
:104BA000FF0000FFFFFFFFFFFF000000000000000C
:104BB0000000000000000000000000FFFF0000FFF8
:104BC000FF0000FFFF0000FFFF0000FFFF0000FFED
:104BD000FF0000FFFF0000FFFF000000FFFFFFFFDE
:104BE0000000000000FFFF000000000000000000C7
:104BF0000000000000000000000000FFFF000000B7
:104C0000FFFF00FFFF000000FFFF00FFFF00FF00AD
:104C1000FFFF00FFFFFFFFFFFFFF00FFFFFF00FFA1
:104C2000FFFF00FFFF000000FFFF0000000000008A
:104C30000000000000000000000000FFFF0000FF77
:104C4000FF0000FFFF0000FFFF000000FFFFFFFF6D
:104C500000000000FFFFFFFF000000FFFF0000FF5B
:104C6000FF0000FFFF0000FFFF0000000000000049
:104C70000000000000000000000000FFFF0000FF37
:104C8000FF0000FFFF0000FFFF000000FFFFFFFF2D
:104C90000000000000FFFF000000000000FFFF0018
:104CA0000000000000FFFF00000000000000000006
:104CB0000000000000000000000000FFFFFFFFFFF9
:104CC000FF0000000000FFFF0000000000FFFF00E9
:104CD00000000000FFFF0000000000FFFF000000D8
:104CE000000000FFFFFFFFFFFF00000000000000CA
:104CF00000000000000000000000000000FFFFFFB7
:104D0000FF00000000FFFF000000000000FFFF00A8
:104D10000000000000FFFF000000000000FFFF0097
:104D20000000000000FFFFFFFF0000000000000087
:104D30000000000000000000000000FF0000000074
:104D4000000000FFFF00000000000000FFFF000067
:104D50000000000000FFFF00000000000000FFFF57
:104D600000000000000000FFFF0000000000000045
:104D70000000000000000000000000FFFFFFFF0037
:104D80000000000000FFFF000000000000FFFF0027
:104D90000000000000FFFF000000000000FFFF0017
:104DA000000000FFFFFFFF00000000000000000007
:104DB0000000000000000000000000000000FF00F4
:104DC0000000000000FFFFFF00000000FFFF00FFE9
:104DD000FF0000FFFF000000FFFF000000000000D8
:104DE00000000000000000000000000000000000C3
:104DF00000000000000000000000000000000000B3
:104E000000000000000000000000000000000000A2
:104E10000000000000000000000000000000000092
:104E20000000FFFFFFFFFFFFFFFF0000000000008A
:104E300000000000000000000000000000FFFF0074
:104E400000000000FFFFFFFF000000FFFFFFFFFF6B
:104E5000FF0000FFFFFFFFFFFF000000FFFFFFFF5D
:104E60000000000000FFFF00000000000000000044
:104E70000000000000000000000000000000000032
:104E800000000000FFFFFFFF00000000000000FF27
:104E9000FF000000FFFFFFFFFF0000FFFF0000FF1B
:104EA000FF000000FFFFFFFFFF0000000000000008
:104EB0000000000000000000000000FFFF000000F4
:104EC000000000FFFF000000000000FFFFFFFFFFE9
:104ED000000000FFFF0000FFFF0000FFFF0000FFD9
:104EE000FF0000FFFFFFFFFF0000000000000000C8
:104EF00000000000000000000000000000000000B2
:104F000000000000FFFFFFFF000000FFFF000000A7
:104F1000000000FFFF000000000000FFFF00000095
:104F200000000000FFFFFFFF000000000000000085
:104F3000000000000000000000000000000000FF72
:104F4000FF000000000000FFFF000000FFFFFFFF68
:104F5000FF0000FFFF0000FFFF0000FFFF0000FF59
:104F6000FF000000FFFFFFFFFF0000000000000047
:104F70000000000000000000000000000000000031
:104F800000000000FFFFFFFF000000FFFF0000FF28
:104F9000FF0000FFFFFFFFFFFF0000FFFF0000001A
:104FA00000000000FFFFFFFF000000000000000005
:104FB0000000000000000000000000000000FFFFF3
:104FC000FF00000000FFFF0000000000FFFFFFFFE8
:104FD000FF00000000FFFF000000000000FFFF00D6
:104FE0000000000000FFFF000000000000000000C3
:104FF00000000000000000000000000000000000B1
:1050000000000000FFFFFFFFFF0000FFFF0000FFA8
:10501000FF0000FFFF0000FFFF000000FFFFFFFF99
:10502000FF000000000000FFFF0000FFFFFFFFFF88
:105030000000000000000000000000FFFF00000072
:10504000000000FFFF000000000000FFFFFFFFFF67
:10505000000000FFFF0000FFFF0000FFFF0000FF57
:10506000FF0000FFFF0000FFFF0000000000000045
:1050700000000000000000000000000000FFFF0032
:10508000000000000000000000000000FFFFFF0023
:105090000000000000FFFF000000000000FFFF0014
:1050A00000000000FFFFFFFF000000000000000004
:1050B000000000000000000000000000000000FFF1
:1050C000FF0000000000000000000000000000FFE2
:1050D000FF000000000000FFFF000000000000FFD4
:1050E000FF000000000000FFFF000000FFFFFFFFC7
:1050F0000000000000000000000000FFFF000000B2
:10510000000000FFFF000000000000FFFF00FFFFA5
:10511000000000FFFFFFFF00000000FFFF00FFFF97
:10512000000000FFFF0000FFFF0000000000000083
:10513000000000000000000000000000FFFFFF0072
:105140000000000000FFFF000000000000FFFF0063
:105150000000000000FFFF000000000000FFFF0053
:1051600000000000FFFFFFFF000000000000000043
:10517000000000000000000000000000000000002F
:10518000000000FFFF0000FFFF0000FFFFFFFFFF28
:10519000FFFF00FFFFFFFFFFFFFF00FFFF00FF001B
:1051A000FFFF00FFFF000000FFFF00000000000005
:1051B00000000000000000000000000000000000EF
:1051C000000000FFFFFFFFFF000000FFFF0000FFE7
:1051D000FF0000FFFF0000FFFF0000FFFF0000FFD7
:1051E000FF0000FFFF0000FFFF00000000000000C4
:1051F00000000000000000000000000000000000AF
:1052000000000000FFFFFFFF000000FFFF0000FFA5
:10521000FF0000FFFF0000FFFF0000FFFF0000FF96
:10522000FF000000FFFFFFFF000000000000000083
:10523000000000000000000000000000000000006E
:10524000000000FFFFFFFFFF000000FFFF0000FF66
:10525000FF0000FFFF0000FFFF0000FFFFFFFFFF58
:10526000000000FFFF000000000000FFFF00000042
:10527000000000000000000000000000000000002E
:1052800000000000FFFFFFFFFF0000FFFF0000FF26
:10529000FF0000FFFF0000FFFF000000FFFFFFFF17
:1052A000FF000000000000FFFF000000000000FF02
:1052B000FF000000000000000000000000000000EF
:1052C000000000FFFFFFFFFF000000FFFF0000FFE6
:1052D000FF0000FFFF000000000000FFFF000000D3
:1052E000000000FFFF0000000000000000000000C0
:1052F00000000000000000000000000000000000AE
:1053000000000000FFFFFFFFFF0000FFFF000000A4
:1053100000000000FFFFFFFF00000000000000FF92
:10532000FF0000FFFFFFFFFF000000000000000083
:1053300000000000000000000000000000FFFF006F
:10534000000000FFFFFFFFFFFF00000000FFFF0065
:105350000000000000FFFF000000000000FFFF0051
:10536000000000000000FFFFFF0000000000000040
:10537000000000000000000000000000000000002D
:10538000000000FFFF0000FFFF0000FFFF0000FF24
:10539000FF0000FFFF0000FFFF0000FFFF0000FF15
:1053A000FF000000FFFFFFFFFF0000000000000003
:1053B00000000000000000000000000000000000ED
:1053C000000000FFFF0000FFFF0000FFFF0000FFE4
:1053D000FF0000FFFF0000FFFF000000FFFFFFFFD6
:1053E0000000000000FFFF000000000000000000BF
:1053F00000000000000000000000000000000000AD
:10540000000000FFFF000000FFFF00FFFF00FF00A3
:10541000FFFF00FFFFFFFFFFFFFF0000FFFFFFFF99
:10542000FF000000FFFF00FFFF0000000000000081
:10543000000000000000000000000000000000006C
:10544000000000FFFF0000FFFF000000FFFFFFFF64
:105450000000000000FFFF0000000000FFFFFFFF52
:10546000000000FFFF0000FFFF0000000000000040
:10547000000000000000000000000000000000002C
:10548000000000FFFF0000FFFF0000FFFF0000FF23
:10549000FF0000FFFF0000FFFF000000FFFFFFFF15
:1054A000FF0000000000FFFF000000FFFFFFFF0003
:1054B00000000000000000000000000000000000EC
:1054C000000000FFFFFFFFFFFF0000000000FFFFE4
:1054D0000000000000FFFF0000000000FFFF0000D0
:1054E000000000FFFFFFFFFFFF00000000000000C2
:1054F00000000000000000000000000000FFFF00AE
:1055000000000000FFFFFFFF000000FFFFFFFFFFA4
:10551000FF0000FFFFFFFFFFFF00000000FFFF0094
:1055200000000000FFFFFFFF00000000000000007F
:105530000000000000FFFF000000000000FFFF006F
:105540000000000000FFFF000000000000FFFF005F
:105550000000000000FFFF000000000000FFFF004F
:105560000000000000FFFF000000000000FFFF003F
:105570000000000000000000000000FFFFFFFFFF30
:10558000FF0000FFFFFFFF00000000FFFFFFFFFF25
:10559000000000FFFF00FFFFFF0000FFFF0000FF13
:1055A000FF000000000000FFFF00000000000000FE
:1055B000000000000000FF000000000000FFFF00EE
:1055C00000000000FFFFFF00000000FFFFFFFF00E2
:1055D00000000000FFFFFF000000000000FFFF00D0
:1055E000000000000000FF000000000000000000BC
:1055F0000000000000FF00000000000000FFFF00AE
:105600000000000000FFFFFF0000000000FFFFFFA0
:10561000FF00000000FFFFFF0000000000FFFF0090
:105620000000000000FF000000000000000000007B
:10563000000000000000000000000000000000006A
:105640000000000000000000000100000000000158
:10565000010100000000000103020000000001023F
:105660000404000000000102040400000000010323
:10567000040400000000000000000000000101011F
:105680000000010001020201000001000203030109
:1056900000000101030303010000020103040301F0
:1056A00001010202040C0402010103030C0D040BAE
:1056B00002020000000000000001000000000000E5
:1056C00000010000000000000102000101000000D4
:1056D0000102010A010000000203020B01010000A7
:1056E0000304030C01010000030503140A0B01016C
:1056F000020500000101000000000101010000009E
:10570000000001020200000000000203010100008D
:105710000001030401000000000204030101010173
:1057200001030403020102020204050C0B0B0B032C
:10573000040D000000000000000000000000000058
:105740000000010100000001000002010001010150
:105750000000020100010202000003020001020138
:10576000000004030002030100010D030203030211
:105770000101000000000000000000000000000027
:105780000000000000000100000000010001020014
:1057900000000101010302000000010303040100F5
:1057A00000000204040401000000030405040100D9
:1057B00000000000000000000000000000000000E9
:1057C00000000000000000000000000000000000D9
:1057D00000000000000000000000000000000000C9
:1057E00000000000000001010000010000010101B3
:1057F000000000000112FFFF362E00010009AEFF7D
:10580000FF360000000112FFFF76000000000AF7DB
:10581000FFFF000000000113FFFF00000000000A6E
:1058200065FF0000000000091CFF000000000000F0
:10583000091C2E25262536FF7676362E2E3636FF87
:10584000FF7E3E362E3636BFFFB63E362E36363615
:10585000FFFFFF773636363EBFFFFFFF3636363660
:105860003EBFFFFFBF3E3E373636B7FFFFFFFFFFAD
:10587000FFFFFFFFFFFFFFFFFFFFFFFFFFFFFFFF38
:10588000FFFFFFFFFFFFFFFFFFFFFFFFFFFFFFFF28
:10589000FFFFFFFFFFFFFFFFFFFFFFFFFFFFFFFF18
:1058A00036FFFFFFFFFFFFB62D76FFFFFFFFFF1C58
:1058B0001313FFFFFFFFFFFFFFFFFFFFFFFFFFFFD0
:1058C000FFFFFFFFFFFFFFFFFFFFFFFFFFFFFFFFE8
:1058D000FFFFFFFFFFFFFFFFFFFF252D36FFFFFF4D
:1058E000FFFF24252EBFFFFFFFFF12131D6EFFFFDA
:1058F000FFFFFFFFFFFFFFFFFFFFFFFFFFFFFFFFB8
:10590000FFFFFFFFFFFFFFFFFFFFFFFFFFFFFFFFA7
:10591000FFFFFFFFFFFFFFFFFFFFFFFFFFFFFFFF97
:10592000FFFFFFFFFFFFFFFFFFFFFFFFFFFFFFFF87
:10593000FFFFFFFFFFFFFFFFBF25FFFFFFFFFFFF91
:10594000FF2EFFFFFFFFFFFFFF36FFFFFFFFFFFF01
:10595000FF7EFFFFFFFFFFFFFFFFFFFFFFFFFFFFD8
:10596000BFFFFFFFFFFFFFFF77FFFFFFFFFFFFFF0F
:1059700036FF1D150D040302000026150403020165
:10598000000025150C020000000026150B01000088
:1059900000002E140A0100000000761C0B09000014
:1059A0000000FF1D0B0A00000000FFFF140A0000AA
:1059B00000000000000000000000000000000000E7
:1059C00000000000000000000000000000000000D7
:1059D00000000000000000000000000000000000C7
:1059E00000000000000000000000000000000000B7
:1059F000010000000001020304040000000203048F
:105A0000040C000000020C04040C00000001030C54
:105A10000C0C00000101030C050D00010103030C37
:105A20000C0D0102010C14151515020201031514C9
:105A30001515030315150C0C03020C03151D0D0C95
:105A40000B0B0D041D1D0D150C0C1D1515251D1D15
:105A50000C14252515252525151D252E1D252E253E
:105A60001D25252E25262D2E2E2E2636362E2E367B
:105A7000FFFF0B1C0B14020B03040C1C14150B046E
:105A80000D0D0C251D1D0C0D0D150C25251D0C14C3
:105A900015150C25252514151D1D152E2E2E1D1D25
:105AA0001D1D152E362E252E2525FF763636362E33
:105AB0002E2D0D0C0C0C0C0C0C150D0C140C140DC7
:105AC00015151515151515151D151D151D1D1D155E
:105AD00025151D1D2525251D251D1D252E25251DAD
:105AE000251D25252E2E25252E252E2E363625251F
:105AF0002D250D040203030B02010D0404040C14F4
:105B00000C020D040C0C151D0D030D0D0D0C1C1DB0
:105B10000D03151D150D1D1D0D041D1D2515251D20
:105B20000D041D262E1D251D0D05252E362525258A
:105B30001515040505040101000104050503020112
:105B4000020205050404020203030405050404041B
:105B5000040305040404040D0D04050D0D05040DD6
:105B60000D040D1D150D0D150D041D1D150D0D1527
:105B70000D0501000101000000000101020100000B
:105B80000000020202010101000002030202010002
:105B900000000303030100000000040402010000F0
:105BA00000000404020101000000040402010100DD
:105BB00000000000000000000009000000000000DC
:105BC00000000000000000000000000000000000D5
:105BD00000000000000000000000000000000000C5
:105BE00000000000000000000000000000000000B5
:105BF0000000131CFFFFFFFFFFFF00091C242565A9
:105C0000252500000100090A0A0A00000000000022
:105C10000000000000000000000000000000000084
:105C20000000000000000000000000000000000074
:105C30000000FFFFFFFFFF1C090025FFFFFFFF1D06
:105C40000A0013AEFFFFFF251200000A6EFFFFB629
:105C50001B0000091C6DFFFF1B0100091C1DFFFF3D
:105C60001C090000131CFFFF6E0900000A1BFFFF48
:105C7000B60900091325FFFFFFFF00001225FFFFF3
:105C8000FFFF00000A25FFFFFFFF00000A65FFFF7E
:105C9000FFFF0001126EFFFFFFFF000913FFFFFF70
:105CA000FFFF000813FFFFFFFFFF00081BFFFFFFC0
:105CB000FFFFFFFFFFFFFFFFFFFFFFFFFFFFFFFFF4
:105CC000FFFFFFFFB6BFFFFFB665FFFF130901002F
:105CD0000101FFFF0A0000000000FFAE0A00000003
:105CE0000000FFF7130100000000FFFF1C09000087
:105CF0000000FFFFFFFFFFFFFFFFFFFFFFFFFFFFB2
:105D0000FFFF25252525FFFFFFFF0809131DFFFFC6
:105D1000FFFF0000091C6EFFFFFF0000091B25FFAD
:105D2000FFFF0000091B6DFFFFFF0000091CFFFFC4
:105D3000FFFFFFFFFFFFFFFF2D2EFFFFFFFFFFFF16
:105D40002525FFFFFFFFFFBF1C12FFFFFFFFFF2501
:105D50000900FFFFFFFFBF1B0900FFFFFFFF7613D6
:105D60000100FFFFFFFF6E130000FFFFFFFFB613F0
:105D70000800FFFF1C0A00000000B61D1309000008
:105D800000001312090000000000000000000000E5
:105D90000000000000000000000000000000000003
:105DA00000000000000000000000000000000000F3
:105DB00000000000000001010101000000000001DE
:105DC00002010000000102020302000000020202C0
:105DD000030300010203040303030103040D04038E
:105DE0000B040001040D0D0C04AE0000020D0D0C9F
:105DF000B6FF030302030C151515020302030C156D
:105E00001D1D030302040C15151D030B03550C1473
:105E1000151D03045D040C15151D5DF7030C141509
:105E2000151DFF5D040C151D1D1D0C040C031D2DFF
:105E30002E2E262E363676FFFFFF262E3636FFFF15
:105E4000FFFF2E2E36BFFFFFFFFF252EFFFFFFFFB8
:105E5000FFFF1D2DFFFFFFFFFFFF1D25FFFFFFFFC2
:105E6000FFFF1D2EFFFFFFFFFFFF2636FFFFFFFF97
:105E7000FFFFFFFFFF3636363636FFFFFFFF367671
:105E80007676FFFFFFFFFFFFFFFFFFFFFFFFFFFF34
:105E9000FFFFFFFFFFFFFFFFFFFFFFFFFFFFFFFF12
:105EA000FFFFFFFFFFFFFFFFFFFFFFFFFFFFFFFF02
:105EB000FFFF2E2E36362D2E362E762E36362E2EF1
:105EC0002E2DFFFF7F3636363636FFFFFFFF763644
:105ED0003637FFFFFFFFFFFFFF7FFFFFFFFFFFFFE3
:105EE000FFFFFFFFFFFFFFFFFFFFFFFFFFFFFFFFC2
:105EF000FFFF2E36362D2625251D3636362E2D252E
:105F0000252536363E362E2E2D2D3E363E362E3665
:105F10002E2D7F3E36362E362E36FFFFFFFF3636CD
:105F20002E36FFFFFFFFFFFF3636FFFFFFFFFFFFAD
:105F3000FF36251D1D0D15150C04251D15151515F0
:105F40000D052E261D151D150D0D2E2E26251D1594
:105F5000150D2E362D251D1D1D0D363636251D25FC
:105F60001D0D363636252525150D363636252625C2
:105F70001D150404010101000000050402020100D6
:105F800000000504030202000000040403030100F2
:105F900000000404040301000100050504030202DB
:105FA0000100050404040302000005040D040201BD
:105FB00000000000091265FFB609000000010A1286
:105FC00009000000000000000000000000000000C8
:105FD00000000000000000000000000000000000C1
:105FE00000000000000000000000000000000000B1
:105FF0000000000113FFFFFFFFFF00011BFFFFFF79
:10600000FFFF000965FFFFFFFFFF0009246EFFFF90
:10601000FFFF00091CFFFFFFFFFF000913FFFFFF49
:10602000FFFF000112131313131C000000000108EE
:106030000001FFFF1C0900000000FFFF2512000007
:106040000000FFFF6E1B09000000FFFFF71C0900A6
:106050000000FFFFFF1C09000000FFFFFF1301000D
:1060600000001B13120900000000090000000000DE
:10607000000000000A65FFFFFFFF000012FFFFFFA6
:10608000FFFF00001265FFFFFFFF0000091C25FF56
:10609000FFFF0000000913F6FFFF000000000109E8
:1060A000131C0000000000000809000000000000B0
:1060B0000000FFFFFFFFB71B0900FFFFFFFFFF1CF2
:1060C0000900FFFFFFFFFF250A00FFFFFFFFFFB6EC
:1060D0001200FFFFFFFFFF6E0A0025252D251C1370
:1060E0000900090A0A0A0901000000000000000076
:1060F00000000000020D156EFF5D00090A1DB6FFCD
:106100001D0C0001131DFFFF1D150008131DFFFFCF
:1061100025150000131DFFB6251D00001265FFB6F2
:10612000251D00000A1CFFB72E1D0000091BFFFFE4
:1061300036250C0C14041D2D36360C0D1D251D7630
:1061400076360C1515261DFF2E360D0C152D25FF48
:106150002E36150D152D25FF3636150D152576FF16
:10616000363615151D1D76FF36361D1D252536FFC5
:106170003E362E36FFFFFFFFFFFF36FFFFFFFFFF1C
:10618000FFFF36FFFFFFFFFFFFFF7EFFFFFFFFFF69
:10619000FFFFBFFFFFFFFFFFFFFFFFFFFFFFFFFF4F
:1061A000FFFFFFFFFFFFFFFFFFFFFFFFFFFFFFFFFF
:1061B000FFFF7F36362E2E251D15FFFFFF362D2EB5
:1061C0001D0DFFFFFFFF3625151DFFFFFFFF361DCD
:1061D0001D25FFFFFFFFFF252E2EFFFFFFFFFFBF47
:1061E000362DFFFFFFFFFFFF361DFFFFFFFFFFFF05
:1061F000761D0D0D0C0300000000151502010102B3
:106200000201250C0202030300001D0C020303021D
:1062100000001D0C0304030100000D040404010030
:1062200000000C0D0D03010100000D0D0D04030213
:1062300001000002020000FB00FF0002020000FB60
:1062400000FF0002020000FB00FF0002020000FB52
:1062500000FF0001010007A00000E70100F10001BC
:106260000100FF0002000008260000E200FF00021B
:10627000000008400000D800FF0002040000F80001
:10628000085003084E03085402084C02085802083C
:106290004A01085C0000FC03086003085A03086018
:1062A00003085A03086003085A01050000FF0002B2
:1062B000040000FB0008340003020A040A0A040A6E
:1062C0001E050000FF000000326200000000000018
:1062D000003A62000000000000004262000000007E
:1062E0000000004A6200000000010000526200004D
:1062F00000000000006362000000000000006E6209
:1063000000000000000000796200000000000000B2
:10631000AE620000000000C10000C00000904564B3
:1063200000FF0601530790476407486400912D64FD
:106330001E9045640F456400912D640E9044640FD7
:1063400045640F406400912D641D9045640F4564C1
:1063500000912D640F9044640F45640F47640091D1
:106360002B641D9043640F436400912B640F90478E
:10637000640E48640F4A6400912B640F9047640FC9
:1063800043640E436400912B640F9045640F47648F
:106390000F486400912D641D9045640F4564009181
:1063A0002D640F9043640F45640E406400912D648A
:1063B0001E9045640F456400912D641D904C640F40
:1063C0004C64009124640F904A640F48640E476443
:1063D00000912B640F9045640F43640F406400915B
:1063E0002D641D9045640F456400912D641E9045F9
:1063F0006407476407486400912D641E9045640F4C
:10640000456400912D640E9044640F45640F406410
:1064100000912D641D9045640F456400912D640F1B
:106420009044640F45640F476400912B641D9043B2
:10643000640F436400912B640F9047640E48640F0F
:106440004A6400912B640F9047640F43640F4364C8
:1064500000912B640E9045640F47640F48640091CF
:106460002D641D9045640F456400912D640F904389
:10647000640F45640E406400912D641E9045640FC6
:10648000456400912D641D904C640F4C6400912470
:10649000640F904A640F48640E476400912B640FA8
:1064A0009045640F40640F912D640F9045640E4534
:1064B000640F912D640F9040640F45640E912D641C
:1064C0000F9047640F48640F912D640E904A640F3B
:1064D0004C640F9128640F904E640F4F640E912806
:1064E000640F904C640F4E640F5364009126640E49
:1064F000904E640F4F640F9124640F904C640E4AC9
:10650000640F476400912B640F9043640F43640F42
:10651000456400912B640E9047640F45640F912DE4
:10652000640F9047640E48640F912D640F904A6485
:106530000F4C640F4E6400912D640E904C640F5309
:10654000640F912D640F904E640E4C640F4A6400EA
:106550009124640F9048640F47640E456400912BAA
:10656000640F9047640F48640F912D640F90456449
:106570000E45640F912D640F9040640F45640E9199
:106580002D640F9047640F48640F912D640E904A5C
:10659000640F4C640F9128640F904E640F4F640E8B
:1065A0009128640F904C640F4E640F536400912641
:1065B000640E904E640F4F640F9124640F904C64EE
:1065C0000F4A640E476400912B640F9043640F439D
:1065D000640F456400912B640E9047640F45640F6F
:1065E000912D640F9047640E48640F912D640F90B5
:1065F0004A640F4C640F4E6400912D640E904C64FD
:106600000F53640F912D640F904E640E4C640F4A2B
:1066100064009124640F9048640F47640F45640040
:10662000912B640E9047640F48640F912D640F9076
:1066300045640E45640F912D640FFF06014500FF70
:106640002F0011241FBECFEFD0E1DEBFCDBF14BE9F
:1066500088E10FB6F89480936000109260000FBE3E
:1066600011E0A0E0B1E0E4E5FCEC02C005900D9281
:10667000AC3AB107D9F71BE0A0ECB1E001C01D9224
:10668000A239B107E1F70E94543E882311F40E9419
:10669000313FF894EDEEF7E080E090E020E802C0B2
:1066A0002193019632E08C309307D4F38DEE97E07E
:1066B0009093FA098093F9091092FB09EEEFF9E043
:1066C00080E090E003C0108201963A9684309105F4
:1066D000D4F39093400A80933F0A91E090931E0A6E
:1066E00090931F0A90931D0A1092810015BC8FEFA2
:1066F00087B984B988E98AB95C9A8CE081B98BEF53
:1067000082B91092B00786E08093B107109285009D
:106710001092840083E0809389008DE88093880044
:1067200089E08093810082E080936F0082E484BDE1
:1067300017BC95BD83E88093B0001092B30090938E
:10674000B10081E185B91092C5071092B40710928B
:10675000B5071092C0071092BF071092C40710929D
:10676000C3071092E0070E94034080E00E94223E8F
:1067700080FF03C084E00E941F3E0E94C7457894BA
:106780000E94C6450E94B6610C9428660C940000D5
:1067900007E00A95F1F7E5E7F7E0C0ECD1E02091DA
:1067A000B00A0027A081B181AC0FBD1F1C911283DC
:1067B000021708F4102F1C9333960395093090F3B9
:1067C00000E416E01A95F1F70A95D9F7C0ECD1E08C
:1067D00000EEA02E662778E04ED237E23A95F1F728
:1067E0000E9425343BE03A95F1F700C0AA9489F065
:1067F0006395C895683029F0C895C895C89500007C
:10680000EBCF662700243EE1C30FD01DC8950000E2
:10681000E3CF35E03A95F1F700C02DD20E947245E2
:1068200011E00091B30701270093B3072091B4074B
:10683000002309F021272093B407E1E0E093B20799
:10684000E2E0E093360011240895DE01679F000026
:106850000091BA071091BB0700541240000D111DA2
:10686000180105E315E0000D111D280130E41EE1BB
:106870002D9129306FB660FA239FA1010EF4A20179
:10688000040E151EF001F6F0059108B92D91059141
:1068900008B9239F059108B929306FB6059108B949
:1068A00008F4A201059108B960FA040E059108B92F
:1068B000151E1A95059108B9059139F1F00108B92D
:1068C0001EF700C0019108B92D910191000008B98F
:1068D000239F0191000008B929306FB660FA019139
:1068E00008B90EF0A1010191040E08B9151E00C0EF
:1068F000019108B9000000C0019108B901911A95F1
:1069000021F0F00108B906F6DDCF08B90027C895D7
:10691000000008B905E00A95F1F7089520E4E09138
:10692000BA07F091BB078950829FE00DF11DA5E3E6
:10693000B5E0629FA00DB11D002405900D92059059
:106940000D9205900D9205900D9205900D92059077
:106950000D9205900D9205900D9205900D92059067
:106960000D9205900D9205900D9205900D92059057
:106970000D9205900D9205900D9205900D92059047
:106980000D9205900D9205900D9205900D92059037
:106990000D9205900D9205900D9205900D92059027
:1069A0000D9205900D9205900D9205900D92059017
:1069B0000D9205900D9205900D9205900D92059007
:1069C0000D9205900D9205900D9205900D920590F7
:1069D0000D9205900D9205900D9205900D920590E7
:1069E0000D9205900D9205900D9205900D920590D7
:1069F0000D9205900D9205900D9205900D920590C7
:106A00000D9205900D9205900D9205900D920590B6
:106A10000D9205900D9205900D9205900D920590A6
:106A20000D9205900D9205900D9205900D92059096
:106A30000D9205900D9205900D92112408950F93DB
:106A40001F9395E0899FE8E0F5E0E00DF11D0481DA
:106A500082819381E0E48E9FD0019E9FB00DE091F2
:106A60009007F0919107EA0FFB1FA5E3B5E090E4D2
:106A7000699FA00DB11D1124403051F4A20FB11D2A
:106A8000822F122F00FF11C0379610E1121B0DC08C
:106A900088E0821B00FD04C0182FE80FF11D05C01F
:106AA00018E0120FE20FF11D3197503031F498E0E9
:106AB000939FA00DB11D932F06C098E0931B58E043
:106AC000599FE00DF11D11243EEFE89400FD6894FC
:106AD00058E0591B48E0481B3EF0259123132C93A6
:106AE00011964A95D1F707C02491319723132C931F
:106AF00011964A95C9F7E10FF11DA80FB11D5A95DE
:106B000049F711241F910F91089549365336613684
:106B1000893528980E941A38E7E1EA95F1F7289A12
:106B20000FD1E0E0F6E0F2D0E0FF32D0E0FF2FC07E
:106B30002F933F934F935F936F937F938F939F9385
:106B4000AF93BF9378941124E091B607F091B70703
:106B5000E115F10509F009950E9476470E9464400D
:106B60000E94543F0E9447371124E091B807F091EA
:106B7000B907E115F10509F00995BF91AF919F9112
:106B80008F917F916F915F914F913F912F910895D8
:106B9000EF93E091B107E93EE0F5E930D0F12F92B3
:106BA0003F924F925F926F927F928F929F92AF929D
:106BB000BF92CF92DF92EF92FF920F931F932F938A
:106BC0003F934F935F936F937F938F939F93AF9375
:106BD000BF93CF93DF930E94C833DF91CF91BF91D2
:106BE000AF919F918F917F916F915F914F913F9165
:106BF0002F911F910F91FF90EF90DF90CF90BF905A
:106C0000AF909F908F907F906F905F904F903F904C
:106C10002F90EF910895FF93EF93EFB7EF93E091EB
:106C20008400EE50E13000F0E23000F0E33000F09C
:106C3000E43000F0E53000F0E63000F0E73000F03E
:106C4000E83000F0E93000F005D0EF91EFBFEF91B0
:106C5000FF9118950F921F92EAE0FBE60090B007B3
:106C6000000C1124E00DF11D05901490F001099520
:106C70001F900F90089528980E941A38E5E1EA9530
:106C8000F1F7E091B107EA95E093B107289A00C0C7
:106C9000089528980E944138289A0000E1E0F6E023
:106CA00035D047D0089528980E944138E0EB000085
:106CB000EA95E9F700000000289AF6E0E2E026D025
:106CC000089528980E944138289A0000E3E0FDEFDB
:106CD0001DD0E091B107E53091F4E091B307E130C8
:106CE0000000F091C50719F4F091C507F195E3E0B4
:106CF000E0938900EDE8EF0FE09388000895E3E06A
:106D0000E0938900EDE8E093880008950090B107D2
:106D10000A9410905F0011FC0F2E0092B1070090B2
:106D2000B00711FC0E2E0092B007E0E011FCE1E08C
:106D30000895E3E0E0938900EDE8E093880008958A
:106D4000E7E0E0938900EBE1E0938800089500001C
:106D50000000000000000000000000000000000033
:106D60000000000000000000000000000000000023
:106D70000000000000000000000000000000000013
:106D80000000000000000000000000000000000003
:106D900000000000000000000000000000000000F3
:106DA00000000000000000000000000000000000E3
:106DB00000000000000000000000000000000000D3
:106DC00000000000000000000000000000000000C3
:106DD00000000000000000000000000000000000B3
:106DE00000000000000000000000000000000000A3
:106DF0000000000000000000000000000000000093
:106E000099277727833008F00895E0E0FBE7660FC5
:106E1000771FE60FF71FA591B491EEEFF9E02AE096
:106E2000289FE00DF11DA183B28311240895909154
:106E30001D0A9170880F892B80931D0A0895992748
:106E40007727EEEFF9E02AE0289FE00DF11D6E3F75
:106E500031F460911D0A6E7F60931D0A0BC06F3F75
:106E600031F460911D0A6E6F60931D0A03C071E7D3
:106E7000760F75831124089599277727EEEFF9E0AF
:106E80002AE0289FE00DF11D6083112408950E94DF
:106E900056420090FB09002019F4ADEEB7E002C0A5
:106EA000A3EFB8E021E002260092FB0922E0209344
:106EB000FC092F923F924F925F926F927F928F9236
:106EC0009F92AF92BF92CF92DF92EF92FF920F9379
:106ED0001F93CF93DF9350911C0A60911E0A70910B
:106EE0001F0A8091200A2090FF093090000A4090EC
:106EF000020A5090030A6090010A1091FE097090F6
:106F0000090A80900A0A90900B0AA0900C0AB0908F
:106F10000D0A2091080AC090130AD090140AE0903C
:106F2000160AF090170A0091150A3091120A9FEF85
:106F3000620C431CF2014491410300240008C12D5E
:106F4000D02D970CA81CF5014491420300240008A1
:106F5000C10DD01D0C0DED1CF7014491430300241D
:106F60000008C10DD01D8A956AF440911D0A842F36
:106F70008695062E0694062600FA7695679576F98C
:106F800040FF66F940E860FD4FE745030024000834
:106F9000C10DD01D0024C038D0050CF0CFE70A94F5
:106FA000C038D0050CF4C0E8C058CD939A9509F0CC
:106FB000BFCF4091FC094A954093FC0997E009F046
:106FC000B7CF6092010A4092020A90920B0AA092F7
:106FD0000C0A0093150AE092160A60931E0A709339
:106FE0001F0A8093200ADF91CF911F910F91FF908C
:106FF000EF90DF90CF90BF90AF909F908F907F9059
:107000006F905F904F903F902F900895E091F90915
:10701000F091FA09019100000093B30009E0E93F03
:10702000F0070DEE17E008F0F801E093F909F0938E
:10703000FA0908950C941C380C941E380F931F9372
:107040002F93E091F909F091FA0901910093B300AF
:1070500009E0E93FF00710F40000000010F0EDEE49
:10706000F7E0E093F909F093FA09C895C895C89537
:10707000C895C895C895000000002F911F910F91E9
:1070800008950000E091B107E0FFD8CFE1E1EA9573
:10709000F1F700000000089500000000000000006B
:1070A00000000000000000000000000000000000E0
:1070B00000000000000000000000000000000000D0
:1070C00000000000000000000000000000000000C0
:1070D00000000000000000000000000000000000B0
:1070E00000000000000000000000000000000000A0
:1070F0000000000000000000000000000000000090
:10710000000306090C101316191C1F2225282B2E0C
:10711000313336393C3F414447494C4E5153555821
:107120005A5C5E60626466686A6B6D6F70717374DE
:10713000757678797A7A7B7C7D7D7E7E7E7F7F7F97
:107140007F7F7F7F7E7E7E7D7D7C7B7A7A7978767D
:1071500075747371706F6D6B6A68666462605E5C93
:107160005A585553514E4C494744413F3C393633A8
:10717000312E2B2825221F1C191613100C0906036B
:1071800000FDFAF7F4F0EDEAE7E4E1DEDBD8D5D272
:10719000CFCDCAC7C4C1BFBCB9B7B4B2AFADABA83D
:1071A000A6A4A2A09E9C9A9896959391908F8D8C60
:1071B0008B8A888786868584838382828281818187
:1071C0008181818182828283838485868687888A81
:1071D0008B8C8D8F9091939596989A9C9EA0A2A44B
:1071E000A6A8ABADAFB2B4B7B9BCBFC1C4C7CACD16
:1071F000CFD2D5D8DBDEE1E4E7EAEDF0F4F7FAFD33
:10720000808182838485868788898A8B8C8D8E8F06
:10721000909192939495969798999A9B9C9D9E9FF6
:10722000A0A1A2A3A4A5A6A7A8A9AAABACADAEAFE6
:10723000B0B1B2B3B4B5B6B7B8B9BABBBCBDBEBFD6
:10724000C0C1C2C3C4C5C6C7C8C9CACBCCCDCECFC6
:10725000D0D1D2D3D4D5D6D7D8D9DADBDCDDDEDFB6
:10726000E0E1E2E3E4E5E6E7E8E9EAEBECEDEEEFA6
:10727000F0F1F2F3F4F5F6F7F8F9FAFBFCFDFEFF96
:10728000000102030405060708090A0B0C0D0E0F86
:10729000101112131415161718191A1B1C1D1E1F76
:1072A000202122232425262728292A2B2C2D2E2F66
:1072B000303132333435363738393A3B3C3D3E3F56
:1072C000404142434445464748494A4B4C4D4E4F46
:1072D000505152535455565758595A5B5C5D5E5F36
:1072E000606162636465666768696A6B6C6D6E6F26
:1072F000707172737475767778797A7B7C7D7E7F16
:1073000000020406080A0C0E10121416181A1C1E8D
:1073100020222426282A2C2E30323436383A3C3E7D
:1073200040424446484A4C4E50525456585A5C5E6D
:1073300060626466686A6C6E70727476787A7C7E5D
:107340007F7D7B79777573716F6D6B69676563613D
:107350005F5D5B59575553514F4D4B49474543412D
:107360003F3D3B39373533312F2D2B29272523211D
:107370001F1D1B19171513110F0D0B09070503010D
:10738000FFFDFBF9F7F5F3F1EFEDEBE9E7E5E3E1FD
:10739000DFDDDBD9D7D5D3D1CFCDCBC9C7C5C3C1ED
:1073A000BFBDBBB9B7B5B3B1AFADABA9A7A5A3A1DD
:1073B0009F9D9B99979593918F8D8B8987858381CD
:1073C00080828486888A8C8E90929496989A9C9ECD
:1073D000A0A2A4A6A8AAACAEB0B2B4B6B8BABCBEBD
:1073E000C0C2C4C6C8CACCCED0D2D4D6D8DADCDEAD
:1073F000E0E2E4E6E8EAECEEF0F2F4F6F8FAFCFE9D
:107400007F7F7F7F7F7F7F7F7F7F7F7F7F7F7F7F8C
:107410007F7F7F7F7F7F7F7F7F7F7F7F7F7F7F7F7C
:107420007F7F7F7F7F7F7F7F7F7F7F7F7F7F7F7F6C
:107430007F7F7F7F7F7F7F7F7F7F7F7F7F7F7F7F5C
:107700000309131E28313A40464C5054585B5E61C1
:10771000636567696B6C6E6F707172737475767781
:10772000777879797A7A7B7B7C7C7C7D7D7D7E7EA7
:107730007E7E7F7F7F7F7F7F7F7F7F7F7F7F7F7F5B
:107740007F7F7F7F7F7F7F7F7F7F7F7F7F7E7E7E4C
:107750007E7D7D7D7C7C7C7B7B7A7A79797877777E
:10776000767574737271706F6E6C6B696765636147
:107770005E5B5854504C46403A31281E13090300B2
:10778000C6CCD5DBDFE3E5E7E9EAEBECEDEEEFEFC6
:10779000F0F0F0F1F1F1F1F2F2F2F2F2F2F2F2F3D2
:1077A000F3F3F3F3F3F3F3F3F3F3F3F3F3F3F3F3A9
:1077B000F3F3F3F3F3F3F3F3F3F3F3F3F3F3F3F399
:1077C000F3F3F3F3F3F3F3F3F3F3F3F3F3F3F3F389
:1077D000F3F3F3F3F3F3F3F3F3F3F3F3F3F3F3F379
:1077E000F2F2F2F2F2F2F2F2F1F1F1F1F0F0F0EF86
:1077F000EFEEEDECEBEAE9E7E5E3DFDBD5CCC60045
:1078000000283D42302D2C2B2C2D2E2F303233359D
:1078100037393B3D3F414345484A4C4E50535557FD
:10782000595B5D5F61636567696B6C6E70717374E2
:10783000757778797A7B7C7D7D7E7E7F7F7F7F7F89
:107840007F7F7F7F7F7F7E7E7D7D7C7B7A7978776F
:1078500075747371706E6C6B69676563615F5D5B96
:1078600059575553504E4C4A484543413F3D3B398B
:1078700037353332302F2E2D2C2B2C2D30423D28F6
:1078800000E9E5FED4D7D7D7D6D4D2D0CECCCAC85B
:10789000C6C3C1BFBDBAB8B6B4B1AFADABA9A7A599
:1078A000A3A19F9E9C9A999795949391908F8D8C6C
:1078B0008B8A89888887868585848484838383836B
:1078C0008383838383848484858586878888898A63
:1078D0008B8C8D8F909193949597999A9C9E9FA154
:1078E000A3A5A7A9ABADAFB1B4B6B8BABDBFC1C36C
:1078F000C6C8CACCCED0D2D4D6D7D7D7D4FEE5E925
:10790000F9F8F9F5EBE1DDDEE0E2E4E5E6E5E4E2F5
:10791000DED9D2CAC1B7ACA299918A868381808010
:107920008182838586888A8C8D8F90929395969795
:1079300098999A9B9B9C9D9D9D9E9E9E9F9F9F9F7D
:107940009F9F9F9E9E9E9D9D9D9C9B9B9A99989775
:1079500096959392908F8D8C8A888685838281807C
:10796000808183868A9199A2ACB7C1CAD2D9DEE25E
:10797000E4E5E6E5E4E2E0DEDDE1EBF5F9F8F90067
:107980000708070B151F2322201E1C1B1A1B1C1E79
:1079900022272E363F49545E676F767A7E7F7F7F3F
:1079A0007F7E7D7B7A7876747371706E6D6B6A6999
:1079B0006867666565646463636262626161616190
:1079C0006161616262626363636465656667686979
:1079D0006A6B6D6E7071737476787A7B7D7E7F7F53
:1079E0007F7F7E7A766F675E54493F362E27221E50
:1079F0001C1B1A1B1C1E2022231F150B0708070027
:107A00001F313D444E5354565A5F64696E74767903
:107A10007C7F7F7F7F7F7F7F7F7F7F7F7F7F7F7F79
:107A20007F7F7F7F7F7F7F7F7F7F7F7F7F7F7F7F66
:107A30007F7F7F7F7F7F7F7F7F7F7F7F7F7F7F7F56
:107A40007F7F7F7F7F7F7F7F7F7F7F7F7F7F7F7F46
:107A50007F7F7F7F7F7F7F7F7F7F7F7F7F7F7F7F36
:107A60007F7F7F7F7F7F7F7F7F7F7F7F7F7F7F7F26
:107A70007F7F7F7F7F7F7F7F7F7F7F7C7871684C78
:107A80002C1C120C0A0B0A05FDF3E9DFD4CAC0B79F
:107A9000AEA69E97918B8685828080808080808034
:107AA00080808080808080808080808080808080D6
:107AB00080808080808080808080808080808080C6
:107AC00080808080808080808080808080808080B6
:107AD00080808080808080808080808080808080A6
:107AE0008080808080808080808080808080808096
:107AF000808080808087919DACC4CBD4DDF2FAFA7F
:107B000022002400260028002B002D003000330026
:107B1000360039003D004000440048004C00510050
:107B200056005B00600066006C0073007900810005
:107B3000880090009900A200AC00B600C100CC0003
:107B4000D800E500F30001011001210132014401D8
:107B500057016C0181019801B001CA01E5010202DF
:107B60002102410264028802AE02D70203033003FD
:107B700061039403CB03050442048304C704100586
:107B80005D05AF0505066106C206290796070908C7
:107B9000830805098E09200ABA0A5D0B0A0CC10C7C
:107BA000840D510E2B0F121007110A121D134014D1
:107BB0007415BA1614188319071BA31C571E24200A
:107BC0000E22142439267F28E82A752D2930063301
:107BD0000F364539AD3C49401B442848734CFE5094
:107BE000CF55EA5A51600C661D6C8B725A7992809F
:107BF00037885090E598FDA19FABD3B5A3C0000096
:107C000080939007909391070895992777272EE105
:107C1000629F080E191EA0ECB1E0A00DB11D475FD8
:107C20004C93112408958093BA079093BB0708954D
:107C30008091B207089511241092B207089580939D
:107C4000C5070895882329F48091BD079091BE0748
:107C500008958091C1079091C2070895882329F45F
:107C60008091BF079091C00708958091C3079091BC
:107C7000C407089578E07A95F1F700000197D1F7ED
:107C80000895F999FECF92BD81BD60BDF894FA9A2E
:107C9000F99A78940895F999FECF92BD81BDF89430
:107CA000F89A80B5789408951F9380E090E00E9440
:107CB0004B3E182F81E090E00E944B3E90E0382F21
:107CC00020E0210F311D2A55354509F491E0892F17
:107CD0001F910895BF92CF92DF92EF92FF920F9380
:107CE0001F93CF93DF936C01062FB72E0E94543E53
:107CF0008823F1F18FEFC8168FEFD80611F481E0D9
:107D00003AC0EE24FF24C7010E944B3E182FC70142
:107D100001960E944B3ED82FC0E0CE01810F911DED
:107D20008C159D0521F4E114F10459F423C080E27F
:107D300090E0E80EF91E90E0E91694E0F90619F7D4
:107D400019C0802F9B2D9C01E90180E2C82ED12C07
:107D5000C20ED31E87010F5F1F4FC7010E944B3E0B
:107D60008993CC15DD0511F480E005C07801F2CFD0
:107D700084E001C083E0DF91CF911F910F91FF90CC
:107D8000EF90DF90CF90BF900895BF92CF92DF9297
:107D9000EF92FF920F931F93CF93DF936C010E949A
:107DA000543E882311F484E04EC0F6018081918115
:107DB000FFEF8F3F9F0709F445C08A55954509F4A9
:107DC00041C002E010E020E4E22EF12CC7010E9445
:107DD0004B3EB82EC70101960E944B3ED82FC0E003
:107DE0009E012B0D311DF6018081918128173907E5
:107DF00019F41123B1F00EC02F5F3F4F19F4112376
:107E000009F4102F0F5F80E290E0E80EF91E0034B5
:107E1000E9F623C0E12EFF2495E0EE0CFF1C9A95B5
:107E2000E1F7C0E0D0E0F601EC0FFD1FCE018E0DB2
:107E30009F1D60810E94413E2196C032D10599F775
:107E400080E001C081E0DF91CF911F910F91FF9001
:107E5000EF90DF90CF90BF9008951123D9F682E084
:107E6000F2CFCF93DF93C0E0D0E0FE01E059FF4FA7
:107E7000E491CE016E2F0E94413E2196C531D1057D
:107E8000A1F7C0E4D0E0CE016FEF0E94413ECE01E9
:107E900001966FEF0E94413EA09688E0C030D8075F
:107EA00091F7DF91CF9108950F938091E007882398
:107EB00009F4A7C08091E107882309F043C08091AD
:107EC000E2070E94223E282F86FF0FC08091E30721
:107ED0009091E40702979093E4078093E30797FF5C
:107EE00004C01092E4071092E30727FF12C08091AC
:107EF000E3079091E40702969093E4078093E307E9
:107F0000883E910534F087EE90E09093E4078093EB
:107F1000E30724FF0FC08091E5079091E6070297E1
:107F20009093E6078093E50797FF04C01092E60759
:107F30001092E50725FF59C08091E5079091E6076B
:107F4000029646C08091E2070E942E3E9C0140911D
:107F5000E3075091E4078F77907027FF0EC0BA01B6
:107F6000681B790B7093E4076093E30777FF14C0F5
:107F70001092E4071092E3070FC0840F951F9093AF
:107F8000E4078093E307883E910534F087EE90E0A4
:107F90009093E4078093E3074091E5075091E6074B
:107FA000832F992737FF10C08F7790709A01281B75
:107FB000390B3093E6072093E50737FF16C0109280
:107FC000E6071092E50711C08F779070840F951F18
:107FD0009093E6078093E507883D910534F087ED9F
:107FE00090E09093E6078093E50780913D0A6091C9
:107FF000E3074091E50720913E0A0091430A0E9461
:1080000089450F910895FF920F931F93CF93DF93AC
:10801000129A8091E007882329F081E090E00E9485
:108020003A3E02C0C895C895129800E010E0FF24BF
:10803000C0E0D0E0D695C795169507951398809126
:10804000E007882329F085E090E00E943A3E02C0D4
:10805000C895C895009BD068019B1068139A8091C1
:10806000E007882329F085E090E00E943A3E02C0B4
:10807000C895C895F39480E1F816E1F6D093BE0751
:10808000C093BD071093C2070093C1078091BD073D
:108090009091BE070F9731F08091C1079091C20770
:1080A0000F9761F428E088E190E00FB6F894A89566
:1080B000809360000FBE20936000FFCFDF91CF91CF
:1080C0001F910F91FF900895FF920F931F93CF93ED
:1080D000DF930E9403408091BD079091BE0797FDFA
:1080E00006C08091C1079091C20797FF27C081E029
:1080F00090E00E943A3EFF2400E010E0C0E0D0E0B3
:10810000000F111FCC0FDD1F1398C895C895C89597
:10811000C895009B0160019BC160139A88E090E0C4
:108120000E943A3EF39480E1F81651F71093C0078D
:108130000093BF07D093C407C093C307DF91CF91CB
:108140001F910F91FF90089590E026E130E0829F0B
:10815000F001839FF00D929FF00D1124EA5BF54F23
:108160006287089560931D0A089590E026E130E04B
:10817000829FF001839FF00D929FF00D1124EA5B26
:10818000F54F13861182089590E026E130E0829F3A
:10819000F001839FF00D929FF00D1124EA5BF54FE3
:1081A00081E0838B089590E026E130E0829FF0012A
:1081B000839FF00D929FF00D1124EA5BF54F6187CC
:1081C000089590E026E130E0829FF001839FF00D5A
:1081D000929FF00D1124EA5BF54F6483089590E0BF
:1081E00026E130E0829FF001839FF00D929FF00D19
:1081F0001124EA5BF54F658308959093A10A80935B
:10820000A00A8FE68093A60A1092EC07E6E4FAE053
:1082100021E08FEF98E12083108686838783148680
:108220001182958376963AE0EE39F307A1F7089527
:108230001092470A10925D0A1092730A1092890AEE
:1082400001969093AA0A8093A90A9093450A809375
:10825000440A9093AD0A8093AC0A1092A80A109237
:10826000A70A10929F0A10929E0A1092A20A81E019
:108270008093EC071092A50A1092A40A08958091A9
:10828000500A87FD03C08AEF8093500A8091660AE6
:1082900087FD03C08AEF8093660A80917C0A87FD80
:1082A00003C08AEF80937C0A8091920A87FD03C005
:1082B0008AEF8093920A1092EC070895DC01ED9109
:1082C000FC911197AF014F5F5F4F11965C934E93F6
:1082D000E4912E2F30E0E7FF13C02F7730703695F2
:1082E000322F222737952795FA014F5F5F4FE49190
:1082F0008E2F8F77280F311DE7FDF1CF4D935C93C3
:10830000C90108950E941F370895EF92FF920F93BD
:108310001F93CF93DF93182F062FF42EE22EC82F32
:10832000D0E086E190E0C89FF001C99FF00DD89F92
:10833000F00D1124EA5BF54F8385882321F08181BC
:10834000882309F0ACC0EE2091F486E190E0C89F4C
:10835000F001C99FF00DD89FF00D1124EA5BF54F95
:10836000138A8285882309F09AC0108698C013303A
:1083700059F481E091E090931F0A80931E0A81E0F6
:1083800080931D0A0F2D08C0812F60E00E941F37C7
:10839000812F6F2D0E9400370F3799F486E190E00E
:1083A000C89FF001C99FF00DD89FF00D1124EA5B22
:1083B000F54F8091A30A878784EA9AE0958B848B96
:1083C00030C089E0089FC0011124E091A00AF0911B
:1083D000A10AE80FF91F33964591549141155105B3
:1083E00071F486E190E0C89FF001C99FF00DD89F1D
:1083F000F00D1124EA5BF54F158A148A12C0FA01B8
:10840000249186E190E0C89FF001C99FF00DD89FAC
:10841000F00D1124EA5BF54F27874F5F5F4F558BB7
:10842000448B86E190E0C89FD001C99FB00DD89FD2
:10843000B00D1124AA5BB54F50961C9250971A9616
:108440001C921A971C960C931C9711961C921197CC
:108450002FEF19962C9319971896EC9218978BE09A
:1084600090E0C89FF001C99FF00DD89FF00D112436
:10847000EE0FFF1FE85BF54FF08251961C9251976B
:1084800081E01B968C931B9753961C9253975296A0
:108490001C92529714961C92149716962C93DF9167
:1084A000CF911F910F91FF90EF900895CF92DF929F
:1084B000FF920F931F93CF93DF93EFE4FAE0818154
:1084C000282F332727FD30958081280F311D2F3F1E
:1084D000310519F014F02FEF30E0C90137FF02C069
:1084E00080E090E0808376964AE0E73AF40739F737
:1084F0008091EC07882309F028C144C1E091A90AC2
:10850000F091AA0A9F012F5F3F4F3093AA0A209350
:10851000A90A44914F3F69F5A9014F5F5F4F5093FE
:10852000AA0A4093A90AF90184918F3219F4109292
:10853000EC0719C1863009F0FBC0FA013196CF0172
:1085400001969093AA0A8093A90AE491E33529F44D
:108550009093AD0A8093AC0AEBC0E53409F0E8C013
:108560008091AC0A9091AD0A9093AA0A8093A90ACF
:10857000DFC047FF02C04093A20A542F5F70842FD0
:1085800090E0807F9070803B910531F1803C9105B7
:1085900081F18039910509F043C0C9010196F901C3
:1085A000449101969093AA0A8093A90A0197FC012D
:1085B0002491852F90E08C9FF0018D9FF00D9C9F62
:1085C000F00D1124EA5BF54F8081882309F4B0C0D7
:1085D000220F852F648553C0C9010196F90144918A
:1085E00001969093AA0A8093A90A0197FC0124910D
:1085F00053C02F5F3F4F3093AA0A2093A90A2150FE
:108600003040F9012491852F90E08C9FF0018D9FDF
:10861000F00D9C9FF00D1124EA5BF54F248788C074
:108620008091A20A582F5F7090E0807F9070803B0D
:10863000910541F1803C910509F46EC080399105A6
:1086400009F076C02F5F3F4F3093AA0A2093A90A02
:1086500021503040F9012491852F90E08C9FD0016A
:108660008D9FB00D9C9FB00D1124AA5BB54F8C91CE
:10867000882309F45DC0220F852F1C966C910E94FF
:10868000854156C02F5F3F4F3093AA0A2093A90A15
:1086900021503040F9012491473071F4852F90E04A
:1086A0008C9FF0018D9FF00D9C9FF00D1124EA5BD3
:1086B000F54F220F27833CC04B3071F4852F90E09B
:1086C0008C9FF0018D9FF00D9C9FF00D1124EA5BB3
:1086D000F54F220F26832CC04C3571F4852F90E086
:1086E0008C9FF0018D9FF00D9C9FF00D1124EA5B93
:1086F000F54F220F24831CC04436D1F4852F90E01F
:108700008C9FF0018D9FF00D9C9FF00D1124EA5B72
:10871000F54F220F25830CC0852F90E08C9FF00130
:108720008D9FF00D9C9FF00D1124EA5BF54F44875F
:1087300089EA9AE00E945E419093A80A8093A70A72
:1087400010929F0A10929E0A02C0C6E1D0E060918A
:108750009E0A70919F0A8091A70A9091A80A6817B3
:10876000790709F4CBCE6F5F7F4F70939F0A6093B8
:108770009E0A8091A40A9091A50A01969093A50A59
:108780008093A40A0EEF19E0C7E4DAE0FF24BFEFFC
:10879000CB2ED12C8A89882309F05EC08B899C89D5
:1087A000892B09F456C09F858E85981708F04CC018
:1087B00050C08B852B893C898F37E9F4D9018D9185
:1087C000BC8BAB8B8F3F01F1F90161811196BC8BA2
:1087D000AB8BE82FF0E0EE0FFF1FEB57FF4F019040
:1087E000F081E02D8F2D0995EB89FC8981918E8791
:1087F000FC8BEB8B28C0A9014F5F5F4F5C8B4B8BD1
:10880000F90184918F3F21F418821C8A1B8A21C0B0
:108810004F5F5F4F5C8B4B8B41505040FA0164912E
:1088200090E0880F991F8B579F4FFC012591349141
:108830008F2DF9010995EB89FC893196FC8BEB8B27
:108840003197E491EE871F869F858E85981709F4EE
:10885000B0CF8F858F5F8F878A85882319F420E0BA
:1088600030E06BC088898F3F11F08F5F888B9F81CC
:10887000992309F45CC02885222309F458C08E810D
:10888000882309F454C04091A60A442309F44FC038
:10889000899FC001112480509F4F892F992730E074
:1088A000B901869F9001879F300D969F300D11244E
:1088B00020503F4F232F33278D8190E0FC012E9FC6
:1088C000C0012F9F900D3E9F900D112480509F4F0F
:1088D000892F9927242F30E0AC01429FC001439F8C
:1088E000900D529F900D112480509F4F292F3327B8
:1088F0008B818823F1F0EA81F0E0E050FF48E491B9
:10890000E058E89FC001112480509F4F892F99277C
:10891000B601681B790B629FC001639F900D729F27
:10892000900D112480509F4F292F332702C020E043
:1089300030E08A819C81890F8A83F8012083F39437
:10894000065F1F4F6696F4E0FF1609F023CFDF9114
:10895000CF911F910F91FF90DF90CF9008951F93BB
:10896000CF93DF93582F89E0589FC00111242091A5
:10897000A00A3091A10A280F391FC9010396FC01F2
:10898000A591B491F90184918150823010F413E0E3
:108990001DC080915D0A8823B1F08091690A851716
:1089A00011F4442381F48091730A882371F080913B
:1089B0007F0A851711F4442341F490916D0A809148
:1089C000830A891710F411E001C012E0212F30E072
:1089D000FD01449186E190E0289FE001299FD00DA0
:1089E000389FD00D1124CA5BD54F4F871196BD8B90
:1089F000AC8B188A8BE090E0289FF001299FF00D46
:108A0000389FF00D1124EE0FFF1FE85BF54F80E556
:108A1000808368878FEF89871A861B8A198A21E0ED
:108A20002B871A8A5D8729831C828E83133049F431
:108A300081E091E090931F0A80931E0A20931D0A03
:108A400008C0812F60E50E940037812F6A890E944B
:108A50001F37DF91CF911F910895FF920F931F93BE
:108A6000082FF62E0E94003710E08BE090E0089F60
:108A7000F001099FF00D189FF00D1124EE0FFF1F5C
:108A8000E85BF54FF0821F910F91FF900895962FAC
:108A9000482F50E02BE030E0429FF001439FF00D63
:108AA000529FF00D1124EE0FFF1FE85BF54F608120
:108AB000691B60830E9400370895482F50E02BE027
:108AC00030E0429FF001439FF00D529FF00D1124C2
:108AD000EE0FFF1FE85BF54F9081690F60830E94E6
:108AE000003708953091B00A20E010C0822F90E046
:108AF000FC01EE0FFF1FE80FF91FEB58F84FA081A4
:108B0000B181A054BE4F82818C932F5F231770F3E5
:108B10000895DF92EF92FF920F931F93CF93DF930D
:108B2000182FD62E622F70E0A0E0B0E0E42EFF24D4
:108B30001BC090E0FC01EE0FFF1FEE0FFF1FE80FC0
:108B4000F91FE85FFA4F5083C13ED10514F021832D
:108B500001C041833F5F585F832F810F361748F371
:108B6000160F7F5F485F1896701740F4242F205E21
:108B70005D2D30E0ED01CE0DDF1DEECFDF91CF9109
:108B80001F910F91FF90EF90DF9008950895E8E016
:108B9000F5E080EF8083359695E0E533F907D1F76E
:108BA00008951F93CF93DF93FA0174913196149136
:108BB000C72FD0E0AF014F5F5F4F9EE1699F9001EB
:108BC0001124280F311D60E00CC08491875F8D93C4
:108BD0009F5F31969717C8F36F5F4C0F5D1F225E42
:108BE0003F4F611730F4D901A054BE4FFA0190E015
:108BF000F1CFDF91CF911F910895982F882319F419
:108C00008FEF87B9089581E08093B30A8093AF0A0C
:108C10009093AE0A1092B20A8093B10A662321F0B3
:108C20008091B10A8823E1F70895982F882311F4E1
:108C300017B808958CE08093B30A8FEF8093AF0A42
:108C40009093AE0A1092B20A81E08093B10A662333
:108C500021F08091B10A8823E1F708958091B10A4B
:108C60008823F9F08091B20A8823C1F48091AE0A7A
:108C70008093B20A9091B30AE92FF0E0E050FF4FE1
:108C8000808187B98091AF0A890F8093B30A8823C6
:108C900011F08D3031F41092B10A08958150809313
:108CA000B20A08950F931F93CF93DF938C01C0E016
:108CB000D0E007C00E94183E8823E1F30E941B3ECB
:108CC0002196C017D107B4F3DF91CF911F910F9177
:108CD00008957F928F929F92AF92BF92CF92DF9230
:108CE000EF92FF920F931F93CF93DF93782E862EF0
:108CF0005A016901780100E010E00CC0872D8C0F4B
:108D0000692DA7010E94053E2196CA15DB05B4F323
:108D10000F5F1F4F0C151D052CF4C0E0D0E0902E06
:108D2000980CF3CFDF91CF911F910F91FF90EF90AF
:108D3000DF90CF90BF90AF909F908F907F900895DD
:108D40002F923F924F925F926F927F928F929F925B
:108D5000AF92BF92CF92DF92EF92FF920F931F9349
:108D6000DF93CF9300D00F92CDB7DEB71092B00A49
:108D700080910001882309F4A3C0A8E08A2EA5E011
:108D80009A2E7724F4018081803F09F47AC0918182
:108D9000F82FF695F695F695F983282F277019F098
:108DA000F2E02F2E02C022242394392F36953695D7
:108DB0003695892F877019F0E2E06E2E02C0662486
:108DC0006394B82EAA242501420E511CC32EEE2412
:108DD000FF244DC02BE12C1510F09C2D01C0932DCC
:108DE0004DE14D1510F08D2D02C08D2D8E51EEE10F
:108DF0009E9F90011124280F311D890100541E4FA0
:108E0000F80160816930F0F04091B00A493000F516
:108E1000842F90E0FC01EE0FFF1FE80FF91FEB58C5
:108E2000F84F318320836283862F642F0E948E3413
:108E30006091B00AF80160836F5F6093B00A61507F
:108E4000693030F4872D4A815B8192010E941F3581
:108E50008A819B8101969B838A83D394821508F42F
:108E6000B9CF0894E11CF11CC394E61450F480E0DF
:108E70009E2D9C013B832A83D98064EE362E3C0CC8
:108E8000A9CF7394E5E0F0E08E0E9F1EF9E07F1607
:108E900009F078CF3091B00A20E010C0822F90E026
:108EA000FC01EE0FFF1FE80FF91FEB58F84FA081F0
:108EB000B181A054BE4F82818C932F5F231770F332
:108EC0000F900F900F90CF91DF911F910F91FF9016
:108ED000EF90DF90CF90BF90AF909F908F907F905A
:108EE0006F905F904F903F902F9008950E942E4674
:108EF0000E94A0460895EF92FF920F931F9395E072
:108F0000899F802D112450E0EFEFFAE0E80FF11D6A
:108F1000CA018C7190709595879595958795660F88
:108F2000660F660F682B628330E02F713070220F5E
:108F3000331F86E0440F551F8A95E1F7242B2383C6
:108F40000483F582E6821F910F91FF90EF900895C0
:108F5000EF92FF920F931F93CF93DF93DB01790181
:108F600095E0899FE02D1124F0E02FEF3AE0B90160
:108F70006E0F7F1FEB018A818695869586958C936F
:108F800031968A8190E087709070880F991F880FC2
:108F9000991FE20FF31F22812295269526952370B3
:108FA000282BDA012C93828190E08E739070959536
:108FB0008795E7018883FB01248130E040E050E0A1
:108FC000A90133272227858190E0A0E0B0E0BA2FE5
:108FD000A92F982F8827282B392B4A2B5B2B86818A
:108FE00090E0A0E0B0E0282B392B4A2B5B2BD80176
:108FF0002D933D934D935C931397DF91CF911F91E8
:109000000F91FF90EF9008958F929F92AF92BF9231
:10901000DF92EF92FF920F931F93DF93CF93CDB721
:10902000DEB72D970FB6F894DEBF0FBECDBF4B0154
:109030005C0123E0429FC0011124D82E7E010894D8
:10904000E11CF11CB701A70197018E010E5F1F4FB4
:109050000E94A8478D2D8F5FB701A70197018E0150
:109060000A5F1F4F0E94A8478D2D8E5FB701A70191
:1090700097018E01065F1F4F0E94A8478A859B8536
:10908000AC85BD8588159905AA05BB0510F084E05F
:1090900017C08E819F81A885B98588159905AA0575
:1090A000BB0510F083E00CC08A819B81AC81BD813F
:1090B00088159905AA05BB0510F481E001C082E07E
:1090C0002D960FB6F894DEBF0FBECDBFCF91DF91C6
:1090D0001F910F91FF90EF90DF90BF90AF909F9006
:1090E0008F90089590E09C01F4E0220F331FFA95D1
:1090F000E1F7285A2093080570E06D5F7F4FAB01C0
:10910000E4E0440F551FEA95E1F763507040409347
:109110000905069634E0880F991F3A95E1F7809388
:109120000D0540930E0520931205B4E0660F771FDE
:10913000BA95E1F7685C6093130580931705609317
:109140001805089590E09C0144E0220F331F4A95D2
:10915000E1F7285A20931C0570E06D5F7F4FAB014B
:1091600034E0440F551F3A95E1F763507040409347
:109170001D050696B4E0880F991FBA95E1F7809314
:1091800021054093220520932605A4E0660F771F52
:10919000AA95E1F7685C6093270580932B0560939F
:1091A0002C05089530E020E01BC0E22FF0E063E0E2
:1091B000EE0FFF1F6A95E1F7E90FF11DE45CF44F34
:1091C0008081873039F4222321F030E028E098E0D4
:1091D00001C031E09F5F983040F32F5F283010F4DA
:1091E00090E0E3CF832F0895582F722F623058F10B
:1091F000A62FB0E0282F30E0FD01329793E0EE0F6C
:10920000FF1F9A95E1F7E20FF31FE45CF44F9081A2
:10921000FD01319783E0EE0FFF1F8A95E1F7E20F22
:10922000F31FE45CF44F8081981769F4E3E0AA0F20
:10923000BB1FEA95E1F7A20FB31FA45CB44F8C915A
:10924000981709F497C1862F8150863058F5A62FBC
:10925000B0E0252F30E0FD01319793E0EE0FFF1FC6
:109260009A95E1F7E20FF31FE45CF44F9081FD0162
:1092700083E0EE0FFF1F8A95E1F7E20FF31FE45C36
:10928000F44F8081981771F41196E3E0AA0FBB1F89
:10929000EA95E1F7A20FB31FA45CB44F8C91981725
:1092A00009F468C1663058F5A62FB0E0252F30E0EC
:1092B000FD0193E0EE0FFF1F9A95E1F7E20FF31F18
:1092C000E45CF44F9081FD01319683E0EE0FFF1FC7
:1092D0008A95E1F7E20FF31FE45CF44F8081981761
:1092E00071F41296E3E0AA0FBB1FEA95E1F7A20F13
:1092F000B31FA45CB44F8C91981709F43BC1523052
:10930000D8F0A62FB0E0252F30E083E0AA0FBB1FD6
:109310008A95E1F7FD01E45CF44FE20FF31F329709
:1093200091918081981741F4A20FB31FA45CB44FB0
:109330008C91981709F41EC1852F81508630E0F476
:10934000E62FF0E0852F90E0A3E0EE0FFF1FAA9537
:10935000E1F7DF01A45CB44FA80FB91F2E9111965D
:10936000E80FF91FE45CF44F8081281729F4119667
:109370008C91281709F4FEC05630D8F4862F90E05F
:10938000252F30E053E0880F991F5A95E1F7FC0133
:10939000E20FF31FE45CF44F5081FC01E45CF44FF6
:1093A000E20FF31F8181581721F48281581709F4C5
:1093B000E1C0723058F1A72FB0E0242F30E0FD015A
:1093C000329783E0EE0FFF1F8A95E1F7E20FF31F5C
:1093D000E45CF44F9081FD01319763E0EE0FFF1FD5
:1093E0006A95E1F7E20FF31FE45CF44F8081981770
:1093F00069F453E0AA0FBB1F5A95E1F7A20FB31F00
:10940000A45CB44F8C91981709F4B4C0872F815095
:10941000863058F5A72FB0E0242F30E0FD013197BA
:1094200083E0EE0FFF1F8A95E1F7E20FF31FE45C84
:10943000F44F9081FD0163E0EE0FFF1F6A95E1F7A5
:10944000E20FF31FE45CF44F8081981771F41196DA
:1094500053E0AA0FBB1F5A95E1F7A20FB31FA45CFC
:10946000B44F8C91981709F485C0763058F5A72F22
:10947000B0E0242F30E0FD0183E0EE0FFF1F8A955E
:10948000E1F7E20FF31FE45CF44F9081FD013196A8
:1094900063E0EE0FFF1F6A95E1F7E20FF31FE45C54
:1094A000F44F8081981771F4129653E0AA0FBB1FF6
:1094B0005A95E1F7A20FB31FA45CB44F8C91981793
:1094C00009F458C04230D0F0A72FB0E0242F30E08C
:1094D00083E0AA0FBB1F8A95E1F7FD01E45CF44F1E
:1094E000E20FF31F329791918081981739F4A20F00
:1094F000B31FA45CB44F8C919817E1F1842F815075
:109500008630D8F4E72FF0E0842F90E0A3E0EE0F50
:10951000FF1FAA95E1F7DF01A45CB44FA80FB91FA4
:109520002E911196E80FF91FE45CF44F8081281703
:1095300021F411968C912817E9F04630E8F4872F32
:1095400090E0242F30E073E0880F991F7A95E1F7BF
:10955000FC01E20FF31FE45CF44F4081FC01E45C8A
:10956000F44FE20FF31F8181481731F430E082811C
:10957000481719F431E001C030E0832F0895582FC7
:10958000722F623058F1A62FB0E0282F30E0FD0195
:10959000329793E0EE0FFF1F9A95E1F7E20FF31F6A
:1095A000E154F54F9081FD01319783E0EE0FFF1FED
:1095B0008A95E1F7E20FF31FE154F54F8081981788
:1095C00069F4E3E0AA0FBB1FEA95E1F7A20FB31F0E
:1095D000A154B54F8C91981709F497C1862F8150EB
:1095E000863058F5A62FB0E0252F30E0FD013197E9
:1095F00093E0EE0FFF1F9A95E1F7E20FF31FE1549E
:10960000F54F9081FD0183E0EE0FFF1F8A95E1F792
:10961000E20FF31FE154F54F8081981771F4119612
:10962000E3E0AA0FBB1FEA95E1F7A20FB31FA15415
:10963000B54F8C91981709F468C1663058F5A62F7C
:10964000B0E0252F30E0FD0193E0EE0FFF1F9A956B
:10965000E1F7E20FF31FE154F54F9081FD013196E0
:1096600083E0EE0FFF1F8A95E1F7E20FF31FE1544D
:10967000F54F8081981771F41296E3E0AA0FBB1F93
:10968000EA95E1F7A20FB31FA154B54F8C9198173B
:1096900009F43BC15230D8F0A62FB0E0252F30E0BE
:1096A00083E0AA0FBB1F8A95E1F7FD01E154F54F56
:1096B000E20FF31F329791918081981741F4A20F26
:1096C000B31FA154B54F8C91981709F41EC1852F73
:1096D00081508630E0F4E62FF0E0852F90E0A3E0A3
:1096E000EE0FFF1FAA95E1F7DF01A154B54FA80FB8
:1096F000B91F2E911196E80FF91FE154F54F8081A3
:10970000281729F411968C91281709F4FEC05630B9
:10971000D8F4862F90E0252F30E053E0880F991F72
:109720005A95E1F7FC01E20FF31FE154F54F508128
:10973000FC01E154F54FE20FF31F8181581721F42A
:109740008281581709F4E1C0723058F1A72FB0E0B8
:10975000242F30E0FD01329783E0EE0FFF1F8A9542
:10976000E1F7E20FF31FE154F54F9081FD013197CE
:1097700063E0EE0FFF1F6A95E1F7E20FF31FE1547C
:10978000F54F8081981769F453E0AA0FBB1F5A95D3
:10979000E1F7A20FB31FA154B54F8C91981709F4AC
:1097A000B4C0872F8150863058F5A72FB0E0242F02
:1097B00030E0FD01319783E0EE0FFF1F8A95E1F75E
:1097C000E20FF31FE154F54F9081FD0163E0EE0FCE
:1097D000FF1F6A95E1F7E20FF31FE154F54F808117
:1097E000981771F4119653E0AA0FBB1F5A95E1F731
:1097F000A20FB31FA154B54F8C91981709F485C0DF
:10980000763058F5A72FB0E0242F30E0FD0193E02B
:10981000EE0FFF1F9A95E1F7E20FF31FE154F54FAA
:109820009081FD01319683E0EE0FFF1F8A95E1F7ED
:10983000E20FF31FE154F54F8081981771F41296EF
:10984000E3E0AA0FBB1FEA95E1F7A20FB31FA154F3
:10985000B54F8C91981709F458C04230D0F0A72F1B
:10986000B0E0242F30E063E0AA0FBB1F6A95E1F758
:10987000FD01E154F54FE20FF31F32979191808182
:10988000981739F4A20FB31FA154B54F8C919817B4
:10989000E1F1842F81508630D8F4E72FF0E0842F57
:1098A00090E053E0EE0FFF1F5A95E1F7DF01A1545E
:1098B000B54FA80FB91F2E911196E80FF91FE1546B
:1098C000F54F8081281721F411968C912817E9F023
:1098D0004630E8F4872F90E0242F30E043E0880FF3
:1098E000991F4A95E1F7FC01E20FF31FE154F54F90
:1098F0004081FC01E154F54FE20FF31F81814817CD
:1099000031F430E08281481719F431E001C030E0D1
:10991000832F08954CE45BE021E030E011C08081AA
:109920008730B9F03196E417F507C9F72F5F3F4F3D
:10993000AF01485F5F4F2830310511F480E0089592
:10994000F901A3E0EE0FFF1FAA95E1F7E45CF44FE5
:10995000E6CF81E0089560E040E035C0A92FB0E097
:10996000242F30E0FD01329753E0EE0FFF1F5A9590
:10997000E1F7E20FF31FE45CF44F5081FD013197F2
:1099800083E0EE0FFF1F8A95E1F7E20FF31FE45C1F
:10999000F44F8081581779F473E0AA0FBB1F7A95B2
:1099A000E1F7A20FB31FA45CB44F8C91581719F4C0
:1099B00061E048E098E09F5F983080F24F5F483068
:1099C00010F040E025C092E0C9CFA42FB0E0292FCD
:1099D00030E083E0AA0FBB1F8A95E1F7FD01E45C4C
:1099E000F44FE20FF31F329751918081581751F4D1
:1099F000A20FB31FA45CB44F8C91581719F498E0D0
:109A000061E048E09F5F983000F34F5F483010F40A
:109A100092E0DBCF862F08958F929F92BF92CF92D4
:109A2000DF92EF92FF920F931F93DF93CF930F92EA
:109A3000CDB7DEB744E45BE020E030E010C08191B8
:109A40008D93E417F507D9F72F5F3F4FAF01485FBC
:109A50005F4F2830310519F4EE24FF2439C0C901C5
:109A6000A3E0880F991FAA95E1F7FC01E45CF44F8D
:109A7000DC01A154B54FE3CFF401C080B084B082C3
:109A8000C086202F2F5F8D2D602F4D2D0E94BF4A45
:109A9000882341F08D2D8F5FF3E0000F111FFA95A1
:109AA000E1F737C0F401C082B0860F5F1F4F88E036
:109AB00090E0880E991E07301105F1F60894E11C1C
:109AC000F11C98E0E916F10419F400E010E030C050
:109AD000DE2CEFEB8E2EEAE09E2E8E0C9F1C00E01B
:109AE00010E0CACF892F982F9F5FF401F080E180AA
:109AF000E082F1826D2D492F2D2D99830E94BF4A5E
:109B00009981882341F073E0000F111F7A95E1F7E6
:109B1000892F800F1BC0F401F082E1820894811C20
:109B2000911C9730F9F60F5F1F4F0830110569F04F
:109B3000D02E480163E0880C991C6A95E1F78FEB01
:109B40009AE0880E991E80E0CECF80E00F90CF91F2
:109B5000DF911F910F91FF90EF90DF90CF90BF901A
:109B60009F908F9008950F931F9382E396E30E9436
:109B7000133E80E090E060E070E04EE150E02CE1C8
:109B800030E000E210E00E9469461F910F910895B5
:109B900070E090E0FB01A3E0EE0FFF1FAA95E1F754
:109BA000E80FF91FE45CF44FE081EE2351F4880FD5
:109BB000991F6D5F7F4F660F771F855F41EF54E000
:109BC0003BC0E13051F4880F991F6D5F7F4F660FE6
:109BD000771F855F47EF54E02FC0E23051F4880FC4
:109BE000991F6D5F7F4F660F771F855F4DEF54E0C4
:109BF00023C0E33051F4880F991F6D5F7F4F660FCC
:109C0000771F855F43E055E017C0E43051F4880FBB
:109C1000991F6D5F7F4F660F771F855F49E055E0A5
:109C20000BC0E53061F4880F991F6D5F7F4F660FA1
:109C3000771F855F4FE055E00E94D1450895E630DB
:109C400059F4880F991F6D5F7F4F660F771F855FEF
:109C500045E155E00E94D145089570E090E0FB0198
:109C600023E0EE0FFF1F2A95E1F7E80FF91FE45CF0
:109C7000F44FE081EE2361F4880F991F6D5F7F4FF1
:109C8000660F771F460F855F642F41EC54E053C089
:109C9000E13061F4880F991F6D5F7F4F660F771F6A
:109CA000460F855F642F47EC54E045C0E23061F415
:109CB000880F991F6D5F7F4F660F771F460F855F77
:109CC000642F4DEC54E037C0E33061F4880F991FE6
:109CD0006D5F7F4F660F771F460F855F642F43EDE3
:109CE00054E029C0E43061F4880F991F6D5F7F4F05
:109CF000660F771F460F855F642F49ED54E01BC048
:109D0000E53061F4880F991F6D5F7F4F660F771FF5
:109D1000460F855F642F4FED54E00DC0E63071F4BF
:109D2000880F991F6D5F7F4F660F771F460F855F06
:109D3000642F45EE54E00E94D1450895E73069F460
:109D4000880F991F6D5F7F4F660F771F460F855FE6
:109D5000642F4BEE54E00E94D14508950F931F935A
:109D6000142F022FA62FB0E02CE33BE073E0AA0FE4
:109D7000BB1F7A95E1F7A80FB11DA20FB31F4C913D
:109D8000E02FF0E053E0EE0FFF1F5A95E1F7E10FEF
:109D9000F11DE20FF31F90819C93408340E00E94ED
:109DA0002D4E812F602F40E00E942D4E1F910F916C
:109DB0000895880F70E06D5F7F4F660F771F855F96
:109DC0004BEE54E00E94D145089588E06FEF41E0EA
:109DD0000E94AF448DE06CE04FE854E00E94D14512
:109DE00080EF8093080580930D0580931205809382
:109DF000170580931C058093210580932605809389
:109E00002B051092B50A6091380B7091390B809137
:109E10003A0B90913B0B4091B40A0E940448843065
:109E200018F482E08093B50A81E080932B0B81E0E7
:109E300090E00E94524680E00E94223E83FFF7CFCE
:109E400008952F923F924F925F926F927F928F92DE
:109E50009F92AF92BF92CF92DF92EF92FF920F93B9
:109E60001F93DF93CF93CDB7DEB767970FB6F89404
:109E7000DEBF0FBECDBF81E090E00E94524680EF72
:109E8000809330051092880B84E06FEF41E00E94D0
:109E9000AF4427EC3AE080E090E00BC01192E2176B
:109EA000F307E1F701969F01285F3F4F8830910546
:109EB00049F0FC01A3E0EE0FFF1FAA95E1F7E15482
:109EC000F54FECCFFE01319686E0DF011D928A95B9
:109ED000E9F710E001E07F01A4C08C91811711F433
:109EE0002F5F17C02330A0F0832F821B07C0FA0119
:109EF000E80FF11DE154F54F00838F5F8317B8F32E
:109F0000E22FF0E03397EE0DFF1D80818F5F80839D
:109F100020E03F5F1196383001F72330D0F0832FD7
:109F2000821BAB01F3E0440F551FFA95E1F707C020
:109F3000FA01E80FF11DE154F54F00838F5F88307F
:109F4000B8F3E22FF0E03397EE0DFF1D80818F5FB5
:109F500080836F5F7F4F6830710519F420E030E037
:109F600054C0CB01E3E0880F991FEA95E1F7DC01CB
:109F7000A45CB44F20E030E0AC01AFCF8C918117EE
:109F800011F49F5F1DC09330D0F0842F891B0DC04A
:109F9000E82FF0E073E0EE0FFF1F7A95E1F7E20F94
:109FA000F31FE154F54F00838F5F841788F3E92F87
:109FB000F0E03397EE0DFF1D80818F5F808390E08E
:109FC0004F5F18964830D1F69330D0F0842F891B1C
:109FD0000DC0E82FF0E063E0EE0FFF1F6A95E1F798
:109FE000E20FF31FE154F54F00838F5F883088F351
:109FF000E92FF0E03397EE0DFF1D80818F5F8083A6
:10A000002F5F3F4F2830310531F0D901A45CB44FA8
:10A0100090E040E0B3CF1F5F173019F4EE24FF2427
:10A0200019C060E070E09DCFF8018081813031F48B
:10A03000892F6D2D9D870E94C84D9D859F5F0F5F65
:10A040001F4F983089F70894E11CF11CF8E0EF16D7
:10A05000F10459F0DE2C870153E0000F111F5A95CF
:10A06000E1F70154154F90E0DFCF85E090E00E94CA
:10A070005246EE24FF2447E0A42E41C0D6018C9125
:10A08000813049F4F801A082892F6B2D40E09D8733
:10A090000E942D4E9D859F5F0894C11CD11C0F5FAF
:10A0A0001F4F983059F70894E11CF11CF8E0EF16A7
:10A0B000F10429F5C090380ACF824090BB0A509035
:10A0C000BC0A6090BD0A7090BE0A1E010894211C53
:10A0D000311C188619861A861B863AE0832E912C2D
:10A0E000A12CB12C81E090E0A0E0B0E08C8B9D8BA6
:10A0F000AE8BBF8BDE011796BF87AE87A0C0BE2C8C
:10A10000C70123E0880F991F2A95E1F70FEBC02EB6
:10A110000AE0D02EC80ED91E8C01045C144F90E0CA
:10A12000ADCF1F5F113029F420E030E040E050E077
:10A1300035C0123029F42AE030E040E050E02EC073
:10A14000133029F424E130E040E050E027C014301F
:10A1500029F42EE130E040E050E020C0153029F431
:10A1600028E230E040E050E019C0163029F426E43F
:10A1700030E040E050E012C0173029F424E630E02F
:10A1800040E050E00BC0183029F028EC30E040E00F
:10A1900050E004C026E930E040E050E069017A0177
:10A1A000C80CD91CEA1CFB1C88859985AA85BB852F
:10A1B0008C0D9D1DAE1DBF1D88879987AA87BB8703
:10A1C000CA01B9012AE030E040E050E00E94B262EA
:10A1D000CC88DD88EE88FF882C0D3D1D4E1D5F1D4F
:10A1E000CA01B90120EA3CE840E050E00E946C62FC
:10A1F000460E571E681E791E0F5FDC840D1508F48D
:10A2000090CFEF80ED0CEF820894211C311C8AE086
:10A2100090E0A0E0B0E0880E991EAA1EBB1E8C89BB
:10A220009D89AE89BF890196A11DB11D8C8B9D8B27
:10A23000AE8BBF8BAE85BF852A163B0631F0F10190
:10A24000F081FC871F8100E0D8CFCF80C092380A10
:10A250004092BB0A5092BC0A6092BD0A7092BE0A3C
:10A260002091340B3091350B4091360B5091370BC8
:10A27000688579858A859B850E946C623B014C01CB
:10A2800085E090E00E94524667C0D6018C918730ED
:10A2900001F58F2D6E2D0E94D94E8F2D642D0E94B9
:10A2A000D94E8F2D6E2D41E00E942D4EF8019081E8
:10A2B000D5018C9180839C9381E090E00E9452466E
:10A2C0008F2D6E2D0E94D94E8F2D642D40E00E945F
:10A2D0002D4EF3940894C11CD11C0F5F1F4F08949E
:10A2E000A11CB11CB8E0FB1681F6EA940894410861
:10A2F0005108EFEFEE16B1F0620113E0CC0CDD1C5B
:10A300001A95E1F78CE39BE0C80ED91E0E2D10E0E4
:10A31000B3E0000F111FBA95E1F7080F191F56019E
:10A32000FF24B3CF0CE31BE0FF24D8018C918730CE
:10A3300069F40E94256367E070E00E949F62F80163
:10A3400080838F2D60E040E00E942D4EF3940F5FDC
:10A350001F4FF8E0FF1649F70E948A4C882331F01E
:10A36000A6E0EA2EF7E04F2E512CC6CF0E94AB4C50
:10A37000882361F185E090E00E9452460E94D24815
:10A380008823D1F00CE31BE0FF24D8018C918730A7
:10A3900069F40E94256367E070E00E949F62F80103
:10A3A00080838F2D60E040E00E942D4EF3940F5F7C
:10A3B0001F4FF8E0FF1649F785E090E00E945246F3
:10A3C0000E94214F660E771E881E991E1092380A31
:10A3D000B301C40167960FB6F894DEBF0FBECDBFC0
:10A3E000CF91DF911F910F91FF90EF90DF90CF9071
:10A3F000BF90AF909F908F907F906F905F904F90A5
:10A400003F902F900895EF92FF920F931F93CF9359
:10A41000DF9310E020E02EC098818885981729F5F9
:10A420008889981711F50E94256363E070E00E9407
:10A430009F62882341F40E94256367E070E00E94D8
:10A440009F62888311C0813041F40E94256367E0D8
:10A4500070E00E949F62888707C00E94256367E0C2
:10A4600070E00E949F62888B21E02896CE15DF0560
:10A4700099F61F5F183038F042E4E42E4BE0F42EDA
:10A4800000E010E043C0812F90E0EC01C45CD44FA9
:10A490003CE6E32E3BE0F32EE80EF91EBDCF98819B
:10A4A0008981981729F58A81981711F50E942563EB
:10A4B00063E070E00E949F62882341F40E9425635C
:10A4C00067E070E00E949F62888311C0813041F490
:10A4D0000E94256367E070E00E949F62898307C045
:10A4E0000E94256367E070E00E949F628A8321E0FA
:10A4F0002196CE15DF0599F60F5F1F4F88E0E82EF5
:10A50000F12CEC0EFD1E0830110549F0E801B3E016
:10A51000CC0FDD1FBA95E1F7C45CD44FC0CF21301A
:10A5200019F410E020E0AFCFDF91CF911F910F9190
:10A53000FF90EF900895EF92FF920F931F93CF93A8
:10A54000DF9374E4E72E7BE0F72E00E010E014C008
:10A550000E94256367E070E00E949F628993CE1598
:10A56000DF05B1F70F5F1F4F68E0E62EF12CEC0E10
:10A57000FD1E0830110549F0E80153E0CC0FDD1F46
:10A580005A95E1F7C45CD44FE3CF0E9403520E9476
:10A590000C4D882311F40E949B5200E00BC0812FC8
:10A5A000602F40E00E942D4E1F5F1830C1F70F5FF3
:10A5B000083011F010E0F3CFDF91CF911F910F9190
:10A5C000FF90EF900895FF920F931F938DE06AE044
:10A5D0004DE054E00E94D14580EF809308058093C0
:10A5E0000D05809312058093170580931C058093B9
:10A5F00021058093260580932B05FF2481E090E0C0
:10A600000E94524680E00E94223E9C019093280ABC
:10A610008093270A4091330A5091340ACA018095E9
:10A6200090958223932390932C0A80932B0AC9013F
:10A6300080959095842395239093300A80932F0AD8
:10A640003093340A2093330A81E00E94223E9C0119
:10A6500090932A0A8093290A4091350A5091360A2C
:10A66000CA01809590958223932390932E0A80931C
:10A670002D0AC90180959095842395239093320AE1
:10A680008093310A3093360A2093350A90912B0A31
:10A6900095FF05C081E08F1510F0F39405C094FF7D
:10A6A00003C0FF20E1F0FA9482E0F816C1F497FFAE
:10A6B00009C08091370A813029F41092370A0E942C
:10A6C0003F410DC096FF0BC08091370A882339F4B3
:10A6D00081E08093370A86E193E60E9418418091D9
:10A6E0002B0A807F91F18EE06DE044E850E00E94FB
:10A6F000053E8FE06EE044E850E00E94053E8FE0AA
:10A7000060E144E850E00E94053E82E160E144E8F7
:10A7100050E00E94053EFF2019F48EE06DE011C06C
:10A7200081E0F81619F48FE06EE00BC082E0F816B5
:10A7300061F48091370A813011F48FE001C082E129
:10A7400060E140E950E00E94053E80912B0A909123
:10A750002C0A90FF53CF81E08F1508F44FCF00E013
:10A760000BC0812F602F40E00E942D4E1F5F1830DC
:10A77000C1F70F5F083011F010E0F3CF81E0F81659
:10A7800011F40E94E54E80911F0B60917C0B0E949A
:10A7900072488091330B813031F48091250B6091A8
:10A7A000310B0E94A2481F910F91FF900895DF92F4
:10A7B000EF92FF920F931F93DF93CF930F92CDB73A
:10A7C000DEB7F7E0660F771F881F991FFA95D1F75C
:10A7D0000E94B26279018A01D801C701E3E0B6950F
:10A7E000A79597958795EA95D1F7D82E9BE0892F65
:10A7F00067E14FE950E099830E94053E99819F5F90
:10A800009B31A9F790E00AC0892F855F67E147EA8D
:10A8100050E099830E94053E99819F5F9D15A0F3AA
:10A820008FE08D1550F04E2D477050E041565F4F30
:10A830008D2D855F67E10E94053E0F90CF91DF91DE
:10A840001F910F91FF90EF90DF9008952F923F920C
:10A850004F925F926F927F928F929F92AF92BF9230
:10A86000CF92DF92EF92FF920F931F93DF93CF93DC
:10A8700000D00F92CDB7DEB78091270B9091280BB7
:10A88000A091290BB0912A0B803422E492072FE08B
:10A89000A20720E0B20710F0FF2432C0803A46E859
:10A8A000940741E0A40740E0B40718F0FF24F394B4
:10A8B00027C0803157E2950750E0A50750E0B50763
:10A8C00018F022E0F22E1CC0883EE3E09E07E0E094
:10A8D000AE07E0E0BE0718F093E0F92E11C0843611
:10A8E0009105A105B10518F084E0F82E09C00A977A
:10A8F000A105B10518F406E0F02E02C015E0F12E16
:10A9000082E090E06DE070E047E050E021E030E070
:10A9100008E310E00E94694646E050E05B834A830A
:10A9200088242F2C33244CC04090270B5090280BA8
:10A930006090290B70902A0B582D5F5F598310E0AF
:10A94000B1E0AB2EB12CC12CD12C0BC0C601B5018E
:10A950002AE030E040E050E00E946C625B016C0154
:10A960001F5F8981181794F39924A1E0EA2EF12C36
:10A97000012D112D0BC0C801B7012AE030E040E0E5
:10A9800050E00E946C627B018C01939498149CF3BC
:10A99000C301B201A60195010E94B262A80197010C
:10A9A0000E94B26227593F4F8A818E5F6DE0A901F4
:10A9B0000E94053EEA81FB813197FB83EA8389800F
:10A9C0004A815B81421553050CF0AECF0F900F907A
:10A9D0000F90CF91DF911F910F91FF90EF90DF903B
:10A9E000CF90BF90AF909F908F907F906F905F902F
:10A9F0004F903F902F9008958DE06CE045E654E035
:10AA00000E94D14580EF8093080580930D058093C7
:10AA100012058093170580931C0580932105809370
:10AA2000260580932B058091270B9091280BA091F0
:10AA3000290BB0912A0B0196A11DB11D8093270B04
:10AA40009093280BA093290BB0932A0B0E942654B5
:10AA500081E090E00E94524680E00E94223E83FF07
:10AA6000F7CF80911F0B60917C0B0E947248809100
:10AA7000330B813031F48091250B6091310B0E94B2
:10AA8000A24808952F923F924F925F926F927F92C9
:10AA90008F929F92AF92BF92CF92DF92EF92FF92EE
:10AAA0000F931F93DF93CF9300D00F92CDB7DEB7F4
:10AAB0008091340B9091350BA091360BB091370BF0
:10AAC000803422E492072FE0A20720E0B20710F0C2
:10AAD000FF2432C0803A46E8940741E0A40740E0F2
:10AAE000B40718F0FF24F39427C0803157E295078C
:10AAF00050E0A50750E0B50718F0F2E0FF2E1CC0AB
:10AB0000883EE3E09E07E0E0AE07E0E0BE0718F015
:10AB1000E3E0FE2E11C084369105A105B10518F0C1
:10AB200074E0F72E09C00A97A105B10518F466E094
:10AB3000F62E02C055E0F52E82E090E06BE070E06A
:10AB400047E050E021E030E008E310E00E94694671
:10AB500046E050E05B834A8388242F2C33244CC08A
:10AB60004090340B5090350B6090360B7090370B43
:10AB7000582D5F5F598310E041E0A42EB12CC12C09
:10AB8000D12C0BC0C601B5012AE030E040E050E016
:10AB90000E946C625B016C011F5F8981181794F33E
:10ABA000992431E0E32EF12C012D112D0BC0C801A9
:10ABB000B7012AE030E040E050E00E946C627B0187
:10ABC0008C01939498149CF3C301B201A6019501E2
:10ABD0000E94B262A80197010E94B26227593F4FBA
:10ABE0008A818E5F6BE0A9010E94053EEA81FB81AC
:10ABF0003197FB83EA8389804A815B814215530543
:10AC00000CF0AECF0F900F900F90CF91DF911F916E
:10AC10000F91FF90EF90DF90CF90BF90AF909F90FB
:10AC20008F907F906F905F904F903F902F900895FE
:10AC3000CF92DF92EF92FF920F931F93DF93CF9308
:10AC40000F92CDB7DEB787E06FEF41E00E94AF44CF
:10AC50008091340B9091350BA091360BB091370B4E
:10AC60000196A11DB11D8093340B9093350BA093D9
:10AC7000360BB093370B0E9442558091B40A88235B
:10AC800059F58091B70A9091B80AA091B90AB0918C
:10AC9000BA0A8093800B9093810BA093820BB093A0
:10ACA000830B2091340B3091350B4091360B509132
:10ACB000370BCA01B9010E946C6224EF31E040E019
:10ACC00050E00E946C626093B70A7093B80A809358
:10ACD000B90A9093BA0A54C0813009F051C080E497
:10ACE00092E4AFE0B0E08093BB0A9093BC0AA093DB
:10ACF000BD0AB093BE0A8091340B9091350BA091A0
:10AD0000360BB091370B81309105A105B10529F4BF
:10AD100089EB90E0A0E0B0E02BC082309105A10566
:10AD2000B10529F48EED90E0A0E0B0E021C08330C1
:10AD30009105A105B10529F485E191E0A0E0B0E01D
:10AD400017C084309105A105B10529F482E791E08F
:10AD5000A0E0B0E00DC00597A105B10529F48BE294
:10AD600092E0A0E0B0E004C087E594E0A0E0B0E0AD
:10AD700080938E0B90938F0BA093900BB093910BBD
:10AD80000E94FC5400E00AC0812F602F0E94C84D31
:10AD90001F5F1830C9F70F5F083011F010E0F4CFD3
:10ADA00085E090E00E94524600E010E0B7E0EB2E14
:10ADB00012C0F601E1926F01892F6F2D40E0998357
:10ADC0000E942D4E99819F5F983099F70F5F1F4F1A
:10ADD0000830110569F0F02E6801A3E0CC0CDD1CF1
:10ADE000AA95E1F78CE39BE0C80ED91E90E0E1CF75
:10ADF00084E190E00E9452460E949B5280EF809333
:10AE00001C05809321058093260580932B050F90C8
:10AE1000CF91DF911F910F91FF90EF90DF90CF9036
:10AE200008952F923F924F925F926F927F928F92EE
:10AE30009F92AF92BF92CF92DF92EF92FF920F93C9
:10AE40001F93DF93CF9300D00F92CDB7DEB78091E1
:10AE5000B40A882349F46090890B70908A0B809023
:10AE60008B0B90908C0B08C060902D0B70902E0B6C
:10AE700080902F0B9090300B40E4641642E47406EF
:10AE80004FE0840640E0940610F0FF2438C050EAFA
:10AE9000651656E8750651E0850650E0950618F0EF
:10AEA000FF24F3942CC080E1681687E2780680E0E6
:10AEB000880680E0980618F062E0F62E20C098EE32
:10AEC000691693E0790690E0890690E0990618F0FB
:10AED00053E0F52E14C0E4E66E167104810491046B
:10AEE00018F044E0F42E0BC0FAE06F1671048104F0
:10AEF000910418F436E0F32E02C025E0F22E82E031
:10AF000090E069E070E047E050E021E030E008E3E5
:10AF100010E00E94694646E050E05B834A83442487
:10AF20002F2C332444C0542D5F5F598310E091E0EF
:10AF3000A92EB12CC12CD12C0BC0C601B5012AE021
:10AF400030E040E050E00E946C625B016C011F5FEA
:10AF50008981181794F3552481E0E82EF12C012DF6
:10AF6000112D0BC0C801B7012AE030E040E050E0ED
:10AF70000E946C627B018C01539454149CF3C401B5
:10AF8000B301A60195010E94B262A80197010E9437
:10AF9000B26227593F4F8A818E5F69E0A9010E9402
:10AFA000053EEA81FB813197FB83EA8349804A8130
:10AFB0005B81421553050CF0B6CF0F900F900F90A8
:10AFC000CF91DF911F910F91FF90EF90DF90CF9085
:10AFD000BF90AF909F908F907F906F905F904F90B9
:10AFE0003F902F9008952F923F924F925F926F92D1
:10AFF0007F928F929F92AF92BF92CF92DF92EF9209
:10B00000FF920F931F93DF93CF9300D00F92CDB792
:10B01000DEB78091380B9091390BA0913A0BB0912B
:10B020003B0B803422E492072FE0A20720E0B20716
:10B0300010F0FF2432C0803A46E8940741E0A407AC
:10B0400040E0B40718F0FF24F39427C0803157E2A2
:10B05000950750E0A50750E0B50718F002E0F02E84
:10B060001CC0883EE3E09E07E0E0AE07E0E0BE07DC
:10B0700018F013E0F12E11C084369105A105B10539
:10B0800018F0B4E0FB2E09C00A97A105B10518F429
:10B09000A6E0FA2E02C0F5E0FF2E82E090E067E025
:10B0A00070E047E050E021E030E008E310E00E946B
:10B0B000694646E050E05B834A8388242F2C332482
:10B0C0004CC04090380B5090390B60903A0B709008
:10B0D0003B0B582D5F5F598310E0E1E0AE2EB12CA1
:10B0E000C12CD12C0BC0C601B5012AE030E040E0F4
:10B0F00050E00E946C625B016C011F5F8981181730
:10B1000094F3992471E0E72EF12C012D112D0BC041
:10B11000C801B7012AE030E040E050E00E946C62D4
:10B120007B018C01939498149CF3C301B201A60196
:10B1300095010E94B262A80197010E94B26227594C
:10B140003F4F8A818E5F67E0A9010E94053EEA8138
:10B15000FB813197FB83EA8389804A815B814215B9
:10B1600053050CF0AECF0F900F900F90CF91DF9161
:10B170001F910F91FF90EF90DF90CF90BF90AF9015
:10B180009F908F907F906F905F904F903F902F9007
:10B1900008950F931F938BE195E00E94133E86E77D
:10B1A00093E30E94003E80E060E04BE950E00E94A3
:10B1B000D14580E090E068E170E046E150E024E0B5
:10B1C00030E000E010E00E9469460E949B5210921D
:10B1D0000B0510920A0581E090E090931005809392
:10B1E0000F0582E090E0909315058093140583E0AD
:10B1F00090E090931A058093190584E090E0909375
:10B200001F0580931E0585E090E0909324058093B0
:10B21000230586E090E0909329058093280587E038
:10B2200090E090932E0580932D0588E090E0909318
:10B230003305809332051092380B1092390B10921F
:10B240003A0B10923B0B81E090E0A0E0B0E08093DD
:10B25000340B9093350BA093360BB093370B1092B1
:10B26000800B1092810B1092820B1092830B84EF53
:10B2700091E0A0E0B0E08093B70A9093B80AA09361
:10B28000B90AB093BA0A1092840B1092850B1092EF
:10B29000860B1092870B1092200B1092210B1092AC
:10B2A000220B1092230B10921F0B10927C0B80E448
:10B2B00092E4AFE0B0E08093BB0A9093BC0AA09305
:10B2C000BD0AB093BE0A89EB90E0A0E0B0E08093A5
:10B2D0008E0B90938F0BA093900BB093910B80915A
:10B2E000B40A882369F483E090E0A0E0B0E08093A2
:10B2F000270B9093280BA093290BB0932A0B08C01F
:10B300001092270B1092280B1092290B10922A0BE7
:10B3100080E060E00E94724880EF80931C0580937B
:10B3200021058093260580932B058093300510928C
:10B33000880B0E94F3570E9411570E9442550E94A9
:10B34000265481E061E00E94FD451F910F91089510
:10B350002F923F924F925F926F927F928F929F9225
:10B36000AF92BF92CF92DF92EF92FF920F931F9313
:10B37000DF93CF9300D00F92CDB7DEB73B014C01E6
:10B3800080EA681686E8780681E0880680E09806FC
:10B3900018F076E0472E2CC090E1691697E2790606
:10B3A00090E0890690E0990618F065E0462E20C0EE
:10B3B000E8EE6E16E3E07E06E0E08E06E0E09E0634
:10B3C00018F054E0452E14C0F4E66F1671048104A1
:10B3D000910418F043E0442E0BC08AE06816710413
:10B3E0008104910418F44424439402C032E0432EB3
:10B3F00007E010E00419110915950795802F8E5F5D
:10B4000064E14DE750E00E94053E342C1B821A8215
:10B41000902F9D5F998310E091E0A92EB12CC12C53
:10B42000D12C0BC0C601B5012AE030E040E050E06D
:10B430000E946C625B016C011F5F13159CF3232C4F
:10B440002A94552481E0E82EF12C012D112D0BC0FA
:10B45000C801B7012AE030E040E050E00E946C6291
:10B460007B018C01539452149CF3C401B301A601D7
:10B4700095010E94B262A80197010E94B2622D5804
:10B480003F4F8981EA818E0F64E1A9010E94053E48
:10B490008A819B8101969B838A833A94841508F460
:10B4A000BACF0F900F900F90CF91DF911F910F9116
:10B4B000FF90EF90DF90CF90BF90AF909F908F90D4
:10B4C0007F906F905F904F903F902F900895EF92F4
:10B4D000FF920F931F9380912B0B8130D1F4109228
:10B4E0002C0B10922B0B80EF8093080580930D0599
:10B4F000809312058093170580931C058093210586
:10B500008093260580932B05809330051092880B3D
:10B51000F5C280912B0A83FF02C00E94E352809102
:10B520002B0A82FF8EC01091B40A112391F58091ED
:10B53000270B9091280BA091290BB0912A0B009713
:10B54000A105B10509F47DC00E940C4D8150282F42
:10B5500027702295207F285A20933005869586955E
:10B56000869590E00396F4E0880F991FFA95E1F72D
:10B570008093310581E08093880B8091270B909117
:10B58000280BA091290BB0912A0B0197A109B109B1
:10B590004EC0113009F055C00E940C4D8150282F2B
:10B5A00027702295207F285A20933005869586950E
:10B5B000869590E00396E4E0880F991FEA95E1F7FD
:10B5C000809331051093880B60918E0B70918F0BD7
:10B5D0008091900B9091910B28EA3DEF4FEF5FEF38
:10B5E0000E946C622091BB0A3091BC0A4091BD0A56
:10B5F0005091BE0A620F731F841F951F6093BB0A90
:10B600007093BC0A8093BD0A9093BE0A20E834E888
:10B610004EE150E00E94D7538091270B9091280B68
:10B62000A091290BB0912A0B0196A11DB11D809309
:10B63000270B9093280BA093290BB0932A0B0E9401
:10B6400026548091B40A813011F56091BB0A709143
:10B65000BC0A8091BD0A9091BE0A20918E0B309158
:10B660008F0B4091900B5091910B621B730B840BCD
:10B67000950B6093BB0A7093BC0A8093BD0A9093AC
:10B68000BE0A20E834E84EE150E00E94D753809192
:10B69000260B882309F46CC08091840B9091850B54
:10B6A000A091860BB091870B2091200B3091210B3C
:10B6B0004091220B5091230B821B930BA40BB50BD3
:10B6C0000A97A105B10508F4A5C08091270A86FF55
:10B6D00007C090911F0B992319F0915090931F0B65
:10B6E00087FF07C090911F0B973018F49F5F9093CE
:10B6F0001F0B84FF07C090917C0B992319F0915088
:10B7000090937C0B85FF07C090917C0B973018F4C9
:10B710009F5F90937C0B807FC1F080911F0B6091A5
:10B720007C0B0E94724886E06FEF41E00E94AF44BC
:10B7300082E090E064E170E047E050E021E030E03A
:10B740000BE910E00E94694602C01092260B80911E
:10B75000840B9091850BA091860BB091870B809301
:10B76000200B9093210BA093220BB093230B52C07C
:10B770008091270A86FF07C090911F0B992319F02B
:10B78000915090931F0B87FF07C090911F0B97302C
:10B7900018F49F5F90931F0B84FF07C090917C0B60
:10B7A000992319F0915090937C0B85FF07C09091DD
:10B7B0007C0B973018F49F5F90937C0B807F51F146
:10B7C00080911F0B60917C0B0E94724881E08093F6
:10B7D000260B8091840B9091850BA091860BB091E4
:10B7E000870B8093200B9093210BA093220BB09397
:10B7F000230B86E06FEF41E00E94AF4482E090E0CF
:10B8000064E170E047E050E021E030E00BE910E057
:10B810000E9469468091330B813009F018C1209154
:10B820001F0B4091250B241739F490917C0B8091CC
:10B83000310B981709F40BC1822F60917C0B20917A
:10B84000310B0E94AE4E80911F0B60917C0B40919A
:10B85000250B2091310B0E94F4488823F1F485E0F8
:10B860006FEF41E00E94AF448AE090E00E945246B0
:10B8700080911F0B60917C0B4091250B2091310B27
:10B880000E94AE4E8091250B80931F0B6091310B6F
:10B8900060937C0B0E947248CFC00E94214F7B01B5
:10B8A0008C010E94A8598091380B9091390BA0917E
:10B8B0003A0BB0913B0B8E0D9F1DA01FB11F8093C3
:10B8C000380B9093390BA0933A0BB0933B0B0E942B
:10B8D000F3578091B40A2091380B3091390B409185
:10B8E0003A0B50913B0B8823B1F48091890B9091D6
:10B8F0008A0BA0918B0BB0918C0B82179307A40736
:10B90000B50700F52093890B30938A0B40938B0B7E
:10B9100050938C0B15C080912D0B90912E0BA09104
:10B920002F0BB091300B82179307A407B50750F483
:10B9300020932D0B30932E0B40932F0B5093300BF5
:10B940000E9411570E940C4D8823D9F48091B40AAB
:10B95000882311F000E00DC00E94E54E12C0812F37
:10B96000602F0E94C84D1F5F1830C9F70F5F083065
:10B9700011F010E0F4CF85E090E00E9452460E9462
:10B980009B528091B40A8823C1F52091380B3091E5
:10B99000390B40913A0B50913B0B8091B70A909133
:10B9A000B80AA091B90AB091BA0A281739074A070C
:10B9B0005B0710F00E941856E090800BF090810B0E
:10B9C0000091820B1091830B6091380B7091390BB1
:10B9D00080913A0B90913B0B6E197F09800B910B74
:10B9E0002091B70A3091B80A4091B90A5091BA0A29
:10B9F0002E193F09400B510B1DC08130E9F4809195
:10BA0000BB0A9091BC0AA091BD0AB091BE0A8058B1
:10BA10009448AE41B04014F00E9418566091BB0AA1
:10BA20007091BC0A8091BD0A9091BE0A20E834E86A
:10BA30004EE150E00E94D75380EF80931C05809325
:10BA400021058093260580932B051092330B80915E
:10BA5000330B8823C1F480912B0A90912C0A90FF1C
:10BA600027C080911F0B60917C0B0E94A24880919F
:10BA70001F0B8093250B80917C0B8093310B81E011
:10BA80008093330B15C0813099F480912B0A9091EB
:10BA90002C0A81709170892B59F01092330B80EF32
:10BAA00080931C05809321058093260580932B05A8
:10BAB0008091B40A813079F48091BB0A9091BC0ADC
:10BAC000A091BD0AB091BE0A181619061A061B06E7
:10BAD00014F00E94E54E8091840B9091850BA0910B
:10BAE000860BB091870B0196A11DB11D8093840B2D
:10BAF0009093850BA093860BB093870B1F910F91AA
:10BB0000FF90EF90089585E190E09093000B809373
:10BB1000FF0A8FEF9AE00E94C53E08952F923F9250
:10BB20004F925F926F927F928F929F92AF92BF924D
:10BB3000CF92DF92EF92FF920F931F93DF93CF93F9
:10BB4000CDB7DEB729970FB6F894DEBF0FBECDBFD5
:10BB5000A82E6887498738014901C901B8014E2DCF
:10BB60000E94044893E0E99E70011124CE2CCA94EF
:10BB7000C80EB82EDC2CA4E02A2E312C2C0E3D1E33
:10BB80002E010894411C511C17C08D2D8150B2010B
:10BB9000AE014E5F5F4F9E012D5F3F4F81010E94BE
:10BBA000A847EC80FD800E811F818D2D69814A811F
:10BBB0002B810E947B47B394D39482E08B1528F7A6
:10BBC0008C2D6A2D48852985840173010E947B474D
:10BBD0000E94835D29960FB6F894DEBF0FBECDBFDD
:10BBE000CF91DF911F910F91FF90EF90DF90CF9059
:10BBF000BF90AF909F908F907F906F905F904F908D
:10BC00003F902F900895EF920F931F932091320B46
:10BC1000223060F480912B0A90912C0A80789170E8
:10BC2000892B11F02F5F07C0222339F080912B0A56
:10BC300086FF03C021502093320B90912B0A94FF72
:10BC40000DC08091320BE82FF0E0E358F44F808173
:10BC5000882311F0815001C089E1808395FF0DC0D8
:10BC60008091320BE82FF0E0E358F44F8081893166
:10BC700018F48F5F808301C01082892F807F79F153
:10BC80008DE090E06DE070E043E050E022E030E0D5
:10BC900000E210E00E94694640917D0B50E04F5B4E
:10BCA0005F4F8DE06DE00E94053E40917E0B50E0BD
:10BCB0004F5B5F4F8EE06DE00E94053E40917F0B31
:10BCC00050E04F5B5F4F8FE06DE00E94053E80913A
:10BCD000320B835F6EE04DE050E00E94053E8091A4
:10BCE0002B0A83FF15C00091380B1091390B20915E
:10BCF0003A0B30913B0B80917D0B60917E0B409114
:10BD00007F0BE090B40A0E948E5D81E08093B50ABB
:10BD10001F910F91EF90089585E190E09093000BB3
:10BD20008093FF0A6FEF7AE00E946A3E0895DF92E7
:10BD3000EF92FF920F931F93CF93DF93D82EE62EAF
:10BD40008A01F82EC0E0D0E012C0F801EC0FFD1F10
:10BD500040814A3019F4E394FD2C08C0552747FD73
:10BD600050958F2D6E2D0E94053EF3942196F8017B
:10BD700001900020E9F73197E01BF10BCE17DF07A8
:10BD800020F3DF91CF911F910F91FF90EF90DF9003
:10BD900008952F923F924F925F926F927F928F926F
:10BDA0009F92AF92BF92CF92DF92FF920F931F9319
:10BDB000DF93CF93CDB7DEB72F970FB6F894DEBFE2
:10BDC0000FBECDBF80E090E060E070E04EE150E05B
:10BDD0002CE130E000E210E00E9469468AE06AE06F
:10BDE0004DE051E00E94975E84E06CE049E151E053
:10BDF0000E94975E83E16CE041E251E00E94975E11
:10BE0000FF2443E0242E312C2C0E3D1E34E0432E23
:10BE1000512C4C0E5D1E3E010894611C711C28E0E3
:10BE2000C22ED12CCC0EDD1E97E2A92E91E0B92EA8
:10BE30008EE2882E81E0982E8F2DB301AE014E5FE9
:10BE40005F4F910182010E94A8478DB79EB70A9764
:10BE50000FB6F8949EBF0FBE8DBFEDB7FEB73196FB
:10BE6000ADB7BEB71296DC92CE921197B382A28282
:10BE70008981992787FD90958F5B9F4F9583848358
:10BE80008A81992787FD90958F5B9F4F9783868343
:10BE90008B81992787FD90958F5B9F4F9187808736
:10BEA0000E9435631F2D135F8DB79EB70A960FB69C
:10BEB000F8949EBF0FBE8DBF82E0612FA6010E9445
:10BEC000975EADB7BEB718970FB6F894BEBF0FBE5A
:10BED000ADBFEDB7FEB731961296DC92CE921197B8
:10BEE000938282828C819D81AE81BF818483958380
:10BEF000A683B7830E9435638DB79EB708960FB6A9
:10BF0000F8949EBF0FBE8DBF86E0612FA6010E94F0
:10BF1000975EF39493E0F91609F08ECF03E0F02ECC
:10BF200014E0212E312C2C0E3D1E2E010894411CB4
:10BF3000511CB8E0CB2ED12CCC0EDD1E35015401A6
:10BF40008F2DB201AE014E5F5F4F9E012D5F3F4FBF
:10BF500081010E94A847ADB7BEB71A970FB6F894F3
:10BF6000BEBF0FBEADBFEDB7FEB731961296DC92E5
:10BF7000CE921197628273828981992787FD90956D
:10BF80008F5B9F4F958384838A81992787FD909546
:10BF90008F5B9F4F978386838B81992787FD909531
:10BFA0008F5B9F4F918780870E9435631F2D165F9F
:10BFB0008DB79EB70A960FB6F8949EBF0FBE8DBF81
:10BFC00081E1612FA6010E94975EADB7BEB71897B9
:10BFD0000FB6F894BEBF0FBEADBFEDB7FEB731963A
:10BFE0001296DC92CE921197A282B3828C819D81AF
:10BFF000AE81BF8184839583A683B7830E94356316
:10C000008DB79EB708960FB6F8949EBF0FBE8DBF32
:10C0100085E1612FA6010E94975EF39496E0F916E0
:10C0200009F08ECF81E061E00E94FD452F960FB6AA
:10C03000F894DEBF0FBECDBFCF91DF911F910F915E
:10C04000FF90DF90CF90BF90AF909F908F907F90A8
:10C050006F905F904F903F902F90089580912D0AA0
:10C0600090912E0A20912B0A30912C0A822B932B2F
:10C0700085FF15C06091260A63308CF4645F88E008
:10C0800040E250E00E94053E6091260A6F5F609397
:10C09000260A645F88E04FE750E00E94053E8091E9
:10C0A0002D0A90912E0A20912B0A30912C0A822B76
:10C0B000932B84FF15C06091260A16168CF4645FDA
:10C0C00088E040E250E00E94053E6091260A6150FF
:10C0D0006093260A645F88E04FE750E00E94053EC7
:10C0E00080912D0A90912E0A20912B0A30912C0AD2
:10C0F000822B932B90FF30C08091260A882321F455
:10C100001092B40A81E004C0813029F48093B40A0B
:10C1100080932C0B08958230D1F481E09091370AFE
:10C12000891B8093370A882339F40E943F4180E1BC
:10C130006EE043E351E008C086E193E60E941841B7
:10C1400080E16EE049E351E00E94975E08958330FC
:10C1500019F481E08093B50A0895982FAB01FB0193
:10C16000DB010D900020E9F7EA1BFB0B7F96F695AB
:10C17000E7958E2F692F0E94975E08950F931F9366
:10C1800081E061E00E94154682E396E30E94133E3F
:10C1900080E090E060E070E04EE150E02CE130E0C3
:10C1A00000E210E00E9469468BE069E046EF55E34B
:10C1B0000E94D1458BE06DE048E156E30E94D145F5
:10C1C00081E16FE371E00E94AD6081E061E00E9477
:10C1D000FD4500E010E081E090E00E945246095FDA
:10C1E0001F4F80E00E94223E83FFF5CFC8010E94CE
:10C1F0002A631F910F9108950F931F9380E090E0A1
:10C2000060E070E04EE150E02CE130E000E210E050
:10C210000E9469468AE065E571E00E94AD608BE0AE
:10C2200065E671E00E94AD608DE06DE04AE751E0A7
:10C230000E94975E8DE06EE04DE050E00E94053E6A
:10C240001092320B10927D0B10927E0B10927F0B8E
:10C2500081E061E00E94FD451F910F9108950F93C9
:10C260001F9380E090E060E070E04EE150E02CE150
:10C2700030E000E210E00E9469468AE06EE771E07B
:10C280000E94AD606091260A645F88E04FE750E04D
:10C290000E94053E8AE06CE04AE851E00E94975E09
:10C2A0008AE06DE047E951E00E94975E8AE06EE027
:10C2B00042EA51E00E94975E8091370A882329F470
:10C2C00080E16EE043E351E004C080E16EE049E3C9
:10C2D00051E00E94975E8AE06FE04DE051E00E94DD
:10C2E000975E81E061E00E94FD451F910F910895E6
:10C2F0008091B50A87FD1BC081E061E00E94154670
:10C300008091B50A882319F40E942F6109C08130F9
:10C3100019F40E94C95E04C0823011F40E94FC60CE
:10C320008091B50A8093240B8FEF8093B50A80919A
:10C33000240B882319F40E942E600895813089F41B
:10C3400080912D0A90912E0A20912B0A30912C0A6F
:10C35000822B932B89709070892B39F01092B50A3B
:10C360000895823011F40E94035E0895CF92DF9207
:10C37000EF92FF920F931F93DF93CF9300D000D0E3
:10C380000F92CDB7DEB785EC92E60E94FD400E9489
:10C390008C5E72E0C72ED12CCC0EDD1E80E07E01BB
:10C3A0000894E11CF11CB701A701970186010E94C6
:10C3B000A8478A819B81AC81BD818093890B909332
:10C3C0008A0BA0938B0BB0938C0B83E0B701A70172
:10C3D00097010E94A8478A819B81AC81BD8180938F
:10C3E0002D0B90932E0BA0932F0BB093300B0E942C
:10C3F000BE6010922C0B1092B50A1FEF81E090E006
:10C400000E94524680E00E94223E9C019093280A9E
:10C410008093270A4091330A5091340ACA018095CB
:10C4200090958223932390932C0A80932B0AC90121
:10C4300080959095842395239093300A80932F0ABA
:10C440003093340A2093330A81E00E94223E9C01FB
:10C4500090932A0A8093290A4091350A5091360A0E
:10C46000CA01809590958223932390932E0A8093FE
:10C470002D0AC90180959095842395239093320AC3
:10C480008093310A3093360A2093350A80912C0B21
:10C4900087FD15C081E061E00E94154680912C0B5C
:10C4A000882319F40E94B34D04C0813011F40E9416
:10C4B000C95880912C0B8093B60A10932C0B809155
:10C4C000B60A882319F40E94786198CF813009F068
:10C4D00095CF0E94675A92CF629FD001739FF0015F
:10C4E000829FE00DF11D649FE00DF11D929FF00D04
:10C4F000839FF00D749FF00D659FF00D9927729F3B
:10C50000B00DE11DF91F639FB00DE11DF91FBD01C5
:10C51000CF0111240895AA1BBB1B51E107C0AA1F1C
:10C52000BB1FA617B70710F0A61BB70B881F991FD4
:10C530005A95A9F780959095BC01CD01089597FB78
:10C54000092E07260AD077FD04D0E5DF06D00020AB
:10C550001AF4709561957F4F0895F6F7909581953F
:10C560009F4F0895A1E21A2EAA1BBB1BFD010DC00F
:10C57000AA1FBB1FEE1FFF1FA217B307E407F50793
:10C5800020F0A21BB30BE40BF50B661F771F881F6F
:10C59000991F1A9469F760957095809590959B0105
:10C5A000AC01BD01CF010895A0E0B0E0EAEDF2E6F4
:10C5B0000C94F965EC01A880B980CA80DB80A114D5
:10C5C000B104C104D10441F484E2A82E89EDB82E4F
:10C5D0008BE5C82E87E0D82EC601B5012DE133EFDB
:10C5E00041E050E00E94D66527EA31E440E050E0A7
:10C5F0000E946C627B018C01C601B5012DE133EF15
:10C6000041E050E00E94D665CA01B9012CEE34EF3A
:10C610004FEF5FEF0E946C626E0D7F1D801F911FB8
:10C6200097FF04C0615070408040904868837983D0
:10C630008A839B839B013F77C901CDB7DEB7EAE0D0
:10C640000C9415660E94D462089588EA91E00E94D5
:10C65000D4620895A0E0B0E08093A8019093A9016E
:10C66000A093AA01B093AB010895AEE0B0E0EBE374
:10C67000F3E60C94FF650D891E8986E08C831A838E
:10C6800009838FEF9FE79E838D839E01275E3F4F37
:10C69000CE0101966F89788DA9010E9459632F817F
:10C6A0003885020F131FF80110822E96E4E00C94D7
:10C6B0001B66ABE0B0E0EFE5F3E60C94F1653C01FE
:10C6C0002B015A01FC0117821682838181FD03C070
:10C6D0006FEF7FEFC6C19AE0892E1E010894211CDE
:10C6E000311CF3012381F20123FD859123FF819108
:10C6F0002F01882309F4B2C1853239F423FD8591D5
:10C7000023FF81912F01853229F490E0B3010E942B
:10C710004C65E7CF982FFF24EE249924FFE1FF1505
:10C72000D0F09B3269F09C3228F4903259F0933269
:10C7300091F40EC09D3249F0903369F441E024C079
:10C7400052E0F52A84E0F82A28C098E0F92A25C0AA
:10C75000E0E1FE2A22C0F7FC29C0892F80538A30ED
:10C7600070F4F6FE05C0989C902C1124980E15C00C
:10C77000E89CE02C1124E80EF0E2FF2A0EC09E3265
:10C7800029F4F6FC6BC140E4F42A07C09C3619F486
:10C7900050E8F52A02C0983649F4F20123FD95913C
:10C7A00023FF91912F01992309F0B8CF892F855448
:10C7B000833018F08052833038F444E050E0A40E07
:10C7C000B51E5FE359830FC0933631F0933779F08C
:10C7D000933509F056C020C0F5018081898342E07D
:10C7E00050E0A40EB51E610101E010E012C0F50199
:10C7F000C080D180F6FC03C06FEF7FEF02C0692DCF
:10C8000070E042E050E0A40EB51EC6010E944165F2
:10C810008C015FE7F52214C0F501C080D180F6FCE1
:10C8200003C06FEF7FEF02C0692D70E042E050E07F
:10C83000A40EB51EC6010E9436658C0150E8F52A8B
:10C84000F3FE07C01AC080E290E0B3010E944C657D
:10C85000EA948E2D90E008171907A8F30EC0F60190
:10C86000F7FC8591F7FE81916F0190E0B3010E9482
:10C870004C65E110EA94015010400115110579F75B
:10C88000EAC0943611F0993669F5F7FE08C0F50153
:10C89000208131814281538184E090E00AC0F5011A
:10C8A000808191819C01442737FD4095542F82E07F
:10C8B00090E0A80EB91E9FE6F92257FF09C05095D7
:10C8C0004095309521953F4F4F4F5F4FE0E8FE2A4E
:10C8D000CA01B901A1012AE030E00E947865D82E92
:10C8E000D21840C0953729F41F2D1F7E2AE030E072
:10C8F0001DC01F2D197F9F3661F0903720F49835A9
:10C9000009F0ACC00FC0903739F0983709F0A6C0D5
:10C9100004C028E030E00AC0106114FD146020E17A
:10C9200030E004C014FD166020E132E017FF08C0BB
:10C93000F501608171818281938144E050E008C0FB
:10C94000F50180819181BC0180E090E042E050E0FF
:10C95000A40EB51EA1010E947865D82ED2188FE7CB
:10C96000F82EF122F6FE0BC05EEFF522D91438F452
:10C97000F4FE07C0F2FC05C08FEEF82202C01D2DA8
:10C9800001C0192DF4FE0DC0FE01ED0DF11D8081D9
:10C99000803319F499EEF92208C01F5FF2FE05C03A
:10C9A00003C08F2D867809F01F5F0F2DF3FC14C094
:10C9B000F0FE0FC01E1510F09D2C0BC09D2C9E0C80
:10C9C000911A1E2D06C080E290E0B3010E944C65D2
:10C9D0001F5F1E15C0F304C01E1510F4E11A01C03C
:10C9E000EE2404FF0FC080E390E0B3010E944C6589
:10C9F00002FF1DC001FD03C088E790E00EC088E57E
:10CA000090E00BC0802F867891F001FF02C08BE28E
:10CA100001C080E2F7FC8DE290E0B3010E944C651A
:10CA200006C080E390E0B3010E944C659A94D9144B
:10CA3000C0F3DA94F101ED0DF11D808190E0B301B6
:10CA40000E944C65DD20A9F706C080E290E0B301AA
:10CA50000E944C65EA94EE20C1F743CEF301668153
:10CA60007781CB012B96E2E10C940D66FC010590D9
:10CA7000615070400110D8F7809590958E0F9F1FE0
:10CA80000895FC016150704001900110D8F7809525
:10CA900090958E0F9F1F08950F931F93CF93DF9351
:10CAA0008C01EB018B8181FF1BC082FF0DC02E81A9
:10CAB0003F818C819D812817390764F4E881F981D1
:10CAC0000193F983E88306C0E885F985802F0995ED
:10CAD000892B31F48E819F8101969F838E8302C0C2
:10CAE0000FEF1FEFC801DF91CF911F910F910895B4
:10CAF000FA01AA27283051F1203181F1E8946F938F
:10CB00006E7F6E5F7F4F8F4F9F4FAF4FB1E03ED034
:10CB1000B4E03CD0670F781F891F9A1FA11D680FD2
:10CB2000791F8A1F911DA11D6A0F711D811D911D05
:10CB3000A11D20D009F468943F912AE0269F11247A
:10CB40003019305D3193DEF6CF010895462F4770DE
:10CB5000405D4193B3E00FD0C9F7F6CF462F4F7039
:10CB6000405D4A3318F0495D31FD4052419302D097
:10CB7000A9F7EACFB4E0A69597958795779567953D
:10CB8000BA95C9F700976105710508959B01AC013D
:10CB90000A2E06945795479537952795BA95C9F764
:10CBA000620F731F841F951FA01D089597FB092E08
:10CBB00005260ED057FD04D0D5DC0AD0001C38F471
:10CBC00050954095309521953F4F4F4F5F4F0895B9
:10CBD000F6F790958095709561957F4F8F4F9F4F99
:10CBE00008952F923F924F925F926F927F928F9211
:10CBF0009F92AF92BF92CF92DF92EF92FF920F93EC
:10CC00001F93CF93DF93CDB7DEB7CA1BDB0B0FB6F5
:10CC1000F894DEBF0FBECDBF09942A8839884888B2
:10CC20005F846E847D848C849B84AA84B984C88448
:10CC3000DF80EE80FD800C811B81AA81B981CE0F3F
:10CC4000D11D0FB6F894DEBF0FBECDBFED01089524
:04CC5000F894FFCF86
:10CC54000100408891D2E4ADB5B6BEBFFF48696714
:10CC6400682053636F72657300436C617373696307
:10CC74000054696D656400256325632563002537C9
:10CC84006C7500284F66662900284F6E29200042E3
:10CC94006C617A696E67204D616D6D6F74682047B1
:10CCA400616D6573004E657720486967682053633A
:10CCB4006F72652100456E74657220796F757220FC
:10CCC400696E697469616C733A004141410052753F
:10CCD40062792043727573682100506C6179204336
:10CCE4006C617373696300506C61792054696D657C
:0CCCF40064004D757369630001000000CE
:00000001FF
